:020000040800F2
:1000000000060020E1020008E3020008E302000805
:10001000E3020008E3020008E3020008E30200082C
:10002000E3020008E3020008E3020008D18A0008A6
:10003000E3020008E3020008E3020008E30200080C
:10004000E3020008E3020008E3020008E3020008FC
:10005000E3020008E30200087D7F0008A97F000892
:10006000D57F0008018000082D800008E302000809
:10007000E3020008E3020008E3020008E3020008CC
:10008000E3020008E3020008E3020008E3020008BC
:10009000E3020008E3020008E302000859800008B8
:1000A000E3020008E3020008E3020008E30200089C
:1000B000E3020008E3020008E3020008E30200088C
:1000C000E3020008E3020008E3020008E30200087C
:1000D000E3020008E3020008E3020008458100088B
:1000E000BD800008E3020008E3020008E302000804
:1000F000E3020008E3020008E3020008E30200084C
:10010000E3020008E302000881810008E30200081E
:10011000E302000859810008E3020008E302000836
:10012000E3020008E3020008E3020008E30200081B
:10013000E3020008E3020008E3020008E30200080B
:10014000E3020008E3020008E3020008E3020008FB
:10015000E3020008E3020008E3020008E3020008EB
:10016000E3020008E3020008E3020008E3020008DB
:10017000E3020008657C0008E3020008E3020008CF
:10018000E3020008E30200086D810008E3020008B2
:10019000E3020008E3020008E3020008E3020008AB
:1001A000E3020008E3020008E3020008E30200089B
:1001B000E3020008E3020008E3020008E30200088B
:1001C000E3020008E3020008E3020008E30200087B
:1001D000E3020008517C0008E3020008E302000883
:1001E000E3020008E3020008E3020008E30200085B
:1001F000E3020008E3020008E3020008E30200084B
:10020000E3020008E3020008E3020008E30200083A
:10021000E3020008E3020008E3020008E30200082A
:10022000E3020008E3020008E3020008E30200081A
:1002300031810008E3020008E3020008E30200083D
:10024000E3020008E3020008E3020008E3020008FA
:10025000E3020008E3020008E3020008E3020008EA
:10026000E3020008E3020008E3020008E3020008DA
:10027000E3020008E3020008E3020008E3020008CA
:10028000E3020008E3020008E3020008E3020008BA
:10029000E3020008E3020008E3020008E3020008AA
:1002A000E3020008E3020008E3020008E30200089A
:1002B000E3020008E3020008E3020008E30200088A
:1002C000E3020008E3020008E3020008E30200087A
:1002D000E3020008E3020008E3020008E30200086A
:1002E00002E000F000F8FEE772B6374880F30888B5
:1002F000364880F3098836483649086040F20000E5
:10030000CCF200004EF63471CEF200010860BFF36B
:100310004F8FBFF36F8F40F20000C0F2F0004EF637
:100320008851CEF200010860BFF34F8FBFF36F8F8B
:100330004FF00000E1EE100A4EF63C71CEF20001E3
:100340000860062080F31488BFF36F8F06F0F6FE76
:1003500006F0FEF84FF055301F491B4A91423CBF52
:1003600041F8040BFAE71D49184A91423CBF41F895
:10037000040BFAE71A491B4A1B4B9A423EBF51F83D
:10038000040B42F8040BF8E700201849184A914280
:100390003CBF41F8040BFAE706F00EFF06F05CF9EB
:1003A000144C154DAC4203DA54F8041B8847F9E7A6
:1003B00000F0C4F9114C124DAC4203DA54F8041B9E
:1003C0008847F9E706F0F6BE00060020002200206C
:1003D0000000000808ED00E00000002000060020FA
:1003E000E896000800220020D8220020D822002011
:1003F00020670020E0020008E0020008E002000898
:10040000E00200082DE9F04F2DED108AC1F80CD064
:10041000D0F80CD0BDEC108ABDE8F08F002383F338
:1004200011882846A047002005F084FEFEE705F06D
:10043000C3FD00DFFEE7000053B94AB9002908BF39
:1004400000281CBF4FF0FF314FF0FF3000F074B9AF
:10045000ADF1080C6DE904CE00F006F8DDF804E01B
:10046000DDE9022304B070472DE9F047089D0446FA
:100470008E46002B4DD18A42944669D9B2FA82F257
:1004800052B101FA02F3C2F1200120FA01F10CFA93
:1004900002FC41EA030E94404FEA1C48210CBEFBCB
:1004A000F8F61FFA8CF708FB16E341EA034306FB54
:1004B00007F199420AD91CEB030306F1FF3080F0E3
:1004C0001F81994240F21C81023E63445B1AA4B230
:1004D000B3FBF8F008FB103344EA034400FB07F7D2
:1004E000A7420AD91CEB040400F1FF3380F00A8113
:1004F000A74240F207816444023840EA0640E41B08
:1005000000261DB1D4400023C5E900433146BDE8B3
:10051000F0878B4209D9002D00F0EF800026C5E955
:10052000000130463146BDE8F087B3FA83F6002E6D
:100530004AD18B4202D3824200F2F980841A61EBE5
:10054000030301209E46002DE0D0C5E9004EDDE703
:1005500002B9FFDEB2FA82F2002A40F09280A1EBEB
:100560000C014FEA1C471FFA8CFE0126200CB1FB40
:10057000F7F307FB131140EA01410EFB03F0884239
:1005800008D91CEB010103F1FF3802D2884200F2C6
:10059000CB804346091AA4B2B1FBF7F007FB101158
:1005A00044EA01440EFB00FEA64508D91CEB0404F6
:1005B00000F1FF3102D2A64500F2BB800846A4EB51
:1005C0000E0440EA03409CE7C6F12007B34022FA3C
:1005D00007FC4CEA030C20FA07F401FA06F31C436B
:1005E000F9404FEA1C4900FA06F3B1FBF9F8200C78
:1005F0001FFA8CFE09FB181140EA014108FB0EF0BE
:10060000884202FA06F20BD91CEB010108F1FF3A0D
:1006100080F08880884240F28580A8F10208614419
:10062000091AA4B2B1FBF9F009FB101144EA014127
:1006300000FB0EFE8E4508D91CEB010100F1FF34D2
:100640006CD28E456AD90238614440EA0840A0FB6A
:100650000294A1EB0E01A142C846A64656D353D040
:100660005DB1B3EB080261EB0E0101FA07F722FA64
:1006700006F3F1401F43C5E9007100263146BDE88D
:10068000F087C2F12003D8400CFA02FC21FA03F3F0
:10069000914001434FEA1C471FFA8CFEB3FBF7F071
:1006A00007FB10360B0C43EA064300FB0EF69E4296
:1006B00004FA02F408D91CEB030300F1FF382FD22F
:1006C0009E422DD9023863449B1B89B2B3FBF7F6D7
:1006D00007FB163341EA034106FB0EF38B4208D9B0
:1006E0001CEB010106F1FF3816D28B4214D9023EF1
:1006F0006144C91A46EA004638E72E46284605E70F
:100700000646E3E61846F8E64B45A9D2B9EB0208DF
:1007100064EB0C0E0138A3E74646EAE7204694E76F
:100720004046D1E7D0467BE7023B614432E73046A2
:1007300009E76444023842E7704700BF38B500F06B
:10074000DDFB06F001FC054606F0EEFC0446E0B9D0
:10075000104B9D421BD001339D4241F2883504BFAE
:1007600001240025002006F0F9FB0CB100F07AF816
:1007700001F04CFB01F0F6F900F028FD08B100F0A3
:1007800071F8284600F01CF9F9E70025EAE705466C
:10079000E8E700BF010007B008B501F0AFF9A0F12C
:1007A00020035842584108BD07B541F21203022107
:1007B00001A8ADF8043001F0BFF903B05DF804FB07
:1007C00038B5302383F31188174803680BB105F05F
:1007D00095FD0023154A4FF47A71134805F084FD06
:1007E000002383F31188124C236813B12368013B63
:1007F0002360636813B16368013B63600D4D2B7820
:1008000033B963687BB9022001F072FA3223636066
:100810002B78032B07D163682BB9022001F068FA0B
:100820004FF47A73636038BDD8220020C1070008F6
:10083000F8230020F0220020084B187003280CD861
:10084000DFE800F008050208022001F043BA0220A8
:1008500001F030BA024B00225A607047F0220020AB
:10086000F8230020F8B5504B504A1C461968013156
:1008700000F0998004339342F8D162684C4B9A425D
:1008800040F291804B4B9B6803F1006303F500330A
:100890009A4280F08880002001F07EF90220FFF764
:1008A000CBFF454B0021D3F8E820C3F8E810D3F87C
:1008B0001021C3F81011D3F81021D3F8EC20C3F89D
:1008C000EC10D3F81421C3F81411D3F81421D3F881
:1008D000F020C3F8F010D3F81821C3F81811D3F89A
:1008E0001821D3F8802042F00062C3F88020D3F8AA
:1008F000802022F00062C3F88020D3F88020D3F853
:10090000802042F00072C3F88020D3F8802022F0CB
:100910000072C3F88020D3F8803072B64FF0E02325
:10092000C3F8084DD4E90004BFF34F8FBFF36F8FB6
:10093000224AC2F88410BFF34F8F536923F48033E7
:100940005361BFF34F8FD2F8803043F6E076C3F3A4
:10095000C905C3F34E335B0103EA060C29464CEA92
:1009600081770139C2F87472F9D2203B13F1200F5C
:10097000F2D1BFF34F8FBFF36F8FBFF34F8FBFF332
:100980006F8F536923F4003353610023C2F8503250
:10099000BFF34F8FBFF36F8F302383F311888546EA
:1009A00080F308882047F8BD0000020820000208F4
:1009B000FFFF0108002200200044025800ED00E083
:1009C0002DE9F04F93B0B44B2022FF2100900AA8EC
:1009D0009D6801F0C5F9B14A1378A3B90121B04867
:1009E00011700360302383F3118803680BB105F0A5
:1009F00085FC0023AB4A4FF47A71A94805F074FCDA
:100A0000002383F31188009B13B1A74B009A1A604F
:100A1000A64A1378032B03D000231370A24A536015
:100A20004FF0000A009CD3465646D146012001F003
:100A300051F924B19C4B1B68002B00F0268200204A
:100A400001F05CF80390039B002BF2DB012001F026
:100A500031F9039B213B1F2BE8D801A252F823F068
:100A6000E10A0008090B00089D0B00082D0A000888
:100A70002D0A00082D0A00082F0C0008FF0D0008A1
:100A8000190D00087B0D0008A30D0008C90D000812
:100A90002D0A0008DB0D00082D0A00084D0E000885
:100AA000810B00082D0A0008910E0008ED0A0008CD
:100AB000810B00082D0A00087B0D00082D0A000894
:100AC0002D0A00082D0A00082D0A00082D0A00082A
:100AD0002D0A00082D0A00082D0A00089D0B0008A9
:100AE0000220FFF759FE002840F0F981009B022107
:100AF00005A8BAF1000F08BF1C4641F21233ADF849
:100B0000143001F019F891E74FF47A7000F0F6FF15
:100B1000071EEBDB0220FFF73FFE0028E6D0013F77
:100B2000052F00F2DE81DFE807F0030A0D1013360F
:100B30000523042105A8059300F0FEFF17E004211A
:100B40005548F9E704215A48F6E704215948F3E7E4
:100B50004FF01C08404608F1040801F01FF804217A
:100B6000059005A800F0E8FFB8F12C0FF2D10120A4
:100B70004FF0000900FA07F747EA0B0B5FFA8BFB0F
:100B800001F03AF926B10BF00B030B2B08BF002440
:100B9000FFF70AFE4AE704214748CDE7002EA5D01B
:100BA0000BF00B030B2BA1D10220FFF7F5FD07463D
:100BB00000289BD00120002600F0EEFF0220FFF766
:100BC0003BFE1FFA86F8404600F0F6FF0446B0B13F
:100BD000039940460136A1F140025142514100F0D3
:100BE000FBFF0028EDD1BA46044641F21213022160
:100BF00005A83E46ADF8143000F09EFF16E72546E6
:100C00000120FFF719FE244B9B68AB4207D9284609
:100C100000F0C4FF013040F067810435F3E70025A0
:100C2000224BBA463E461D701F4B5D60A8E7002E62
:100C30003FF45CAF0BF00B030B2B7FF457AF02209C
:100C4000FFF7FAFD322000F059FFB0F10008FFF67F
:100C50004DAF18F003077FF449AF0F4A08EB0503C7
:100C6000926893423FF642AFB8F5807F3FF73EAFC0
:100C7000124BB845019323DD4FF47A7000F03EFF2C
:100C80000390039A002AFFF631AF039A0137019BC4
:100C900003F8012BEDE700BF00220020F423002021
:100CA000D8220020C1070008F8230020F0220020ED
:100CB00004220020082200200C220020F422002020
:100CC000C820FFF769FD074600283FF40FAF1F2D2E
:100CD00011D8C5F120020AAB25F003008449424532
:100CE000184428BF4246019201F014F8019AFF21EE
:100CF0007F4801F035F84FEAA803C8F387027C4922
:100D00002846019301F034F8064600283FF46DAF01
:100D1000019B05EB830533E70220FFF73DFD00282B
:100D20003FF4E4AE00F076FF00283FF4DFAE00278A
:100D3000B846704B9B68BB4218D91F2F11D80A9B2D
:100D400001330ED027F0030312AA134453F8203CBA
:100D500005934046042205A9043701F0B7F8804600
:100D6000E7E7384600F01AFF0590F2E7CDF8148067
:100D7000042105A800F0E0FE02E70023642104A896
:100D8000049300F0CFFE00287FF4B0AE0220FFF7FE
:100D900003FD00283FF4AAAE049800F031FF05904F
:100DA000E6E70023642104A8049300F0BBFE0028BA
:100DB0007FF49CAE0220FFF7EFFC00283FF496AED4
:100DC000049800F01FFFEAE70220FFF7E5FC002887
:100DD0003FF48CAE00F02EFFE1E70220FFF7DCFCD1
:100DE00000283FF483AE05A9142000F029FF074630
:100DF0000421049004A800F09FFE3946B9E7322090
:100E000000F07CFE071EFFF671AEBB077FF46EAEEE
:100E1000384A07EB0903926893423FF667AE022017
:100E2000FFF7BAFC00283FF461AE27F003074F44F8
:100E3000B9453FF4A5AE484609F1040900F0AEFEFD
:100E40000421059005A800F077FEF1E74FF47A70D1
:100E5000FFF7A2FC00283FF449AE00F0DBFE0028BB
:100E600044D00A9B01330BD008220AA9002000F0CD
:100E70007FFF00283AD02022FF210AA800F070FF4F
:100E8000FFF792FC1C4805F05BF913B0BDE8F08F4A
:100E9000002E3FF42BAE0BF00B030B2B7FF426AE92
:100EA0000023642105A8059300F03CFE07460028B6
:100EB0007FF41CAE0220FFF76FFC804600283FF451
:100EC00015AEFFF771FC41F2883005F039F905984D
:100ED00000F0DAFF46463C4600F08EFFA6E50646E7
:100EE0004EE64FF0000901E6BA467EE637467CE65C
:100EF000F422002000220020A0860100704700009C
:100F00007047000070470000704700002DE9F04175
:100F100000F58037044616463B7C5BB9C06810304C
:100F2000204400F0F7FEE5683544B5F5004FE56074
:100F300002D816B1BDE8F081DEB905F07F0605F1F3
:100F400010000021C6F180062044F6B232462E443D
:100F500000F006FFA06804F11008324600F10060BE
:100F6000414600F5003005F0B7FD30B901233B7470
:100F7000E0E74FF400463546ECE7A26805F11001C2
:100F8000404632442144A260E268521BE26000F015
:100F9000C1FE0220BDE8F04100F0AABE183000F00A
:100FA000E9BC000010B5044607F042FE204610BD23
:100FB00010B5044607F03CFE204610BDC3B280B217
:100FC000A3F14102052A02D8373800B27047613BCD
:100FD000052B94BF57383038F7E70000F8B50446C2
:100FE0001546084603220C4900F09EFE014688B9CA
:100FF00008346F1C15F91100FFF7E0FF064617F9DA
:1010000011000131FFF7DAFF102940EA061004F859
:10101000010BEFD1F8BD00BFA88D00082DE9F04FFE
:10102000ADF53F7D0746416801222AA802F042FE45
:10103000002840F087800646824681461125DFF869
:101040000C81DFF80CB101AB4FF4805241462AA865
:1010500002F090FF002875D1019AB2F5805F71D837
:10106000002A65D00446019A9442ECD2282D0FD074
:1010700008DC132D2DD01E2D39D0112D13D00134A5
:10108000A4B2F0E7322D2DD0372D2FD02D2DF6D153
:101090003B68121B08EB040138461B692D25984755
:1010A000BDF80440EBE7121B022A09D9594608EBA8
:1010B000040000F039FE18B902342825A4B2DEE796
:1010C00018F804303A2B3DD00A2B1CBFA14613253B
:1010D000D5E718F804300A2B34D03A2B04BFA246C7
:1010E0003225CCE718F80430202BC8D0264618F853
:1010F00004300A2B1AD1AAEB090208EB090102A855
:1011000011254F2A28BF4F2207F03AFEA21B08EBF9
:10111000060116A84F2A28BF4F2207F031FE3B6870
:1011200016AA02A9DB6838469847A8E71E25A6E755
:101130003B68384604491B69984701200DF53F7DFF
:10114000BDE8F08F0020F9E7AA8E000800240020F7
:10115000AC8D000800F1180110B5044686B00846B1
:10116000019100F0F1FB2046FFF758FF60B10199B3
:1011700002A800F049FC102204F1080102A807F0BF
:101180007BFDB0FA80F0400906B010BD70B5044692
:101190000025EEB2304600F00FFD58B10021304678
:1011A000013500F019FD08B9002070BD022000F0E3
:1011B0009FFDEEE72046FFF731FF0028F4D004F54D
:1011C0008034207C80F00100EFE70000F0B5C9B06A
:1011D00005F0D2FE00F0A8FE18B90025284649B057
:1011E000F0BD69462A4802F087FF00284BD1294C00
:1011F000204602F0B1FF284802F0AEFF274802F077
:10120000ABFF2146224803F023F80028E5D17020E7
:1012100007F010FD064610B1214B446003603368AF
:1012200030469B689847054600282ED01A4F19482B
:10123000394603F00DF805460028CED1194807F0CD
:10124000F9FC044638B1184B4760036000F5803361
:10125000C0E902551D74236820469B6898470546DF
:1012600028B10E490C4802F0F3FF0028B5D13368CD
:1012700030465B6898471CB1236820465B689847F6
:1012800000F03AFEAAE70025FAE70446EFE700BFC0
:10129000B08D0008C08D0008D78D0008ED8D0008C6
:1012A000108E0008140001002C8E00082DE9F04F6C
:1012B000D44A8DB00B68D0F804A001931A44036897
:1012C000D14E1A44D1F81C90DFF8B4C3DFF8B4B3A0
:1012D000D0E90234634003EA0A03634013444A68D6
:1012E00002920AEB7363029CC84A2244C4682244F7
:1012F00084688AEA04051D40654015448A680392A3
:1013000003EB3555039CC24A2244846822448AEA8E
:1013100003042C4084EA0A041444CA6805EBF4343C
:101320000492164483EA0502224056445A4032444D
:101330000E69059604EBB222059FB64E3E441E444C
:1013400085EA040313406B4033444E69069602EB72
:101350007363069FB04E3E442E4484EA02051D404E
:10136000654035448E69079603EB3555079FAB4EB4
:101370003E44264482EA03042C4054403444A84EA0
:101380004E4405EBF434164483EA050222405A40E9
:1013900032440E6A089604EBB222089FA14E3E44E6
:1013A0001E4485EA040313406B4033444E6A099699
:1013B00002EB7363099F9C4ED1F830E03E44D1F8B4
:1013C0003880F3442E4484EA02051D4065403544CC
:1013D0008E6AA6F5244703EB35550A964F3F2744FE
:1013E00082EA03042C4054403C44CF6A0B9705EB3F
:1013F000F4340B9E8D4F3744029E174483EA050256
:1014000022405A403A448A4F774404EBB2221F44A8
:1014100085EA040313406B403B444F6BBC4402EB32
:101420007363654484EA020C0CEA030C8CEA040C36
:101430006544DFF854C2C44403EB3555A44482EA42
:1014400003042C4054406444D1F83CC0794905EB76
:10145000F4346144114483EA050222405A400A44AC
:10146000754904EBB2223144079E194484EA020311
:101470002B4063400B44714902EBF36331440B9EF4
:101480000D4482EA03012140514029446C4D03EB95
:10149000F1513544019E254483EA010414405C4027
:1014A0002C44684D01EBB4443544069E154481EA52
:1014B00004021A404A402A44634D04EB3232354458
:1014C0000A9E1D4484EA02030B4063402B445F4D97
:1014D00002EBF3633544059E0D4482EA030121408B
:1014E000514029445A4D03EBF1516544254483EAA8
:1014F000010414405C402C44564D01EBB444354487
:10150000099E154481EA04021A404A402A44524D79
:1015100004EB32323544049E1D4484EA02030B403E
:1015200063402B444D4D02EBF36345440D4482EA86
:101530000301214051402944494D03EBF151354409
:10154000089E2C4483EA010515405D402C44454D1E
:1015500001EBB4443544039E2A4481EA04051D404E
:101560004D402A44404D04EB32323D442B4484EA42
:10157000020593440D4065402B443C4D02EBF36360
:101580003544069E294482EA0305254055402944F6
:10159000374D03EBF1514D442C4483EA01051540CE
:1015A0005D40254401EBB54581EA050404EA0302E8
:1015B0004A405A44A6F5B82B089E05EB3232ABF2EE
:1015C000BE6B54405B4423442A4C344402EB3373D7
:1015D0000B9E0C4485EA020159402144264C3444B8
:1015E00003EB7151029E254482EA03044C402544DA
:1015F000224C444401EB3545144483EA01026A401D
:10160000224443E078A46AD7EECEBDC156B7C7E8FE
:10161000DB702024AF0F7CF52AC68747134630A81D
:10162000019546FDD8988069AFF7448BBED75C8999
:101630002211906B2108B44962251EF640B340C0C8
:10164000515A5E26AAC7B6E95D102FD6531444023C
:1016500081E6A1D8C8FBD3E7E6CDE121D60737C3A1
:10166000870DD5F4ED145A4505E9E3A9F8A3EFFC7D
:10167000D9026F6781F6718722619D6D0C38E5FD97
:10168000937198FD8A4C2A8D8E4379A6934C3444ED
:1016900005EB7222059E1C4481EA05035340234456
:1016A0008F4C344402EB33730A9E0C4485EA0201EA
:1016B000594021448B4C4C4403EB7151254482EA40
:1016C00003044C402C44884D354401EB3444019EC6
:1016D000154483EA010262402A44844D3D4404EBF0
:1016E00072221D4481EA040353402B44804D35444B
:1016F00002EB3373049E294484EA02055D402944C9
:101700007C4D354403EB7151079E254482EA030466
:101710004C402C44784D354401EB3444099E2A4416
:1017200083EA010565401544744A324404EB75258B
:10173000039E134481EA04026A401A44704B7344C6
:1017400005EB32720B4484EA0501514019446D4B9C
:10175000634402EB71511C4485EA02034B401C4474
:10176000694B334401EB3444019E1D4482EA01037A
:1017700063402B44654D04EB73233544069E1544AA
:1017800063EA010262402A44614D03EBB2624D44B8
:1017900062EA040929445F4D89EA03094544494442
:1017A0002C445D4D02EBB1513544049E61EA0308BF
:1017B0001D4488EA0208444401EB744464EA0203CD
:1017C0004B402B44554D04EBF323754463EA010E63
:1017D00015448EEA040E0EEB0502514D03EBB26286
:1017E000354462EA040E29440A9D8EEA030EA5F5EB
:1017F00080164C4D7144A6F6833602EBB151264457
:1018000061EA030454403444029E01EB74443544BD
:1018100064EA02061D444E407319089E424D04EBD3
:10182000F323354463EA01061544664072193F4DBF
:1018300003EBB262654462EA040629443C4D5E4013
:101840003144079E02EBB151354461EA03062C4452
:10185000384D56403D443444059E1D4401EB7444CC
:1018600064EA02034B402B44334D04EBF32335442D
:101870000B9E154463EA010262402A442F4D03EB9C
:10188000B2623544039E0D4462EA04015940294482
:101890002B4D02EBB15135442A4E254461EA030435
:1018A00054402C44099D01EB74442E4464EA020523
:1018B0001E4485EA01039D1903681A440AEB0403D8
:1018C00003EBF5230260436083681C44C36819443A
:1018D0008460C1600DB0BDE8F08F00BF44EABEA4D3
:1018E000A9CFDE4B604BBBF670BCBFBEC67E9B284B
:1018F000FA27A1EA8530EFD4051D880439D0D4D960
:10190000E599DBE6F87CA21F6556ACC4442229F4B5
:1019100097FF2A43A72394AB39A093FCC3595B6577
:1019200092CC0C8FD15D84854F7EA86FE0E62CFEB3
:10193000144301A3A111084E827E53F735F23ABD3C
:10194000BBD2D72A91D386EB094B036003F18833CE
:10195000436003F12943A3F59613A3F68B638360D9
:10196000A3F18833C3600023C0E90433704700BF8C
:10197000012345672DE9F8431446026905460E46E2
:10198000E300C2F3C50800F118079B18036122BFEA
:1019900043690133436112F4FC7F436903EB5473E1
:1019A000436114D0C8F1400907EB08004C4504D24C
:1019B0002246BDE8F84307F06FB9403C4A464E4422
:1019C00007F06AF9444439462846FFF76FFCA04601
:1019D00006EB0409B8F13F0FA9EB08010AD9402230
:1019E000384607F059F939462846A8F14008FFF76C
:1019F0005DFCEFE7A1096FF03F02384602FB0142B0
:101A000006EB8111D5E7000070B50B6901F11805EF
:101A100006460C46C3F3C503EA18501C8022EA545C
:101A2000C3F13F02072A1FD8002100F099F9294687
:101A30002046FFF73BFC38220021284600F090F9B1
:101A4000236929462046236563696365FFF72EFCF9
:101A500021461022304607F01FF920465822002167
:101A6000BDE8704000F07CB9C3F137020021E5E722
:101A70002DE9F84F4FF47A7306460D46002402FB19
:101A800003F7DFF85080DFF8509098F900305FFAE4
:101A900084FA5A1C01D0A34210D159F824002A46D6
:101AA00031460368D3F820B03B46D847854205D17C
:101AB000074B012083F800A0BDE8F88F0134042C07
:101AC000E3D14FF4FA7004F03BFB0020F4E700BFD1
:101AD00044340020102200201422002070B5044657
:101AE0004FF47A76412C254628BF412506FB05F0A8
:101AF00004F026FB641BF5D170BD0000002307B580
:101B0000024601210DF107008DF80730FFF7B0FF05
:101B100020B19DF8070003B05DF804FB4FF0FF30E3
:101B2000F9E700000A46042108B5FFF7A1FF80F09D
:101B30000100C0B2404208BD074B0A4630B41978D4
:101B4000064B53F82140014623682046DD69044BCB
:101B5000AC4630BC604700BF443400201422002053
:101B6000A086010070B50A4E00240A4D04F058FF0B
:101B7000308028683388834208D904F04DFF2B68F1
:101B800004440133B4F5003F2B60F2D370BD00BFB5
:101B9000463400200034002005F010B800F1006049
:101BA00000F500300068704700F10060920000F519
:101BB000003004F091BF0000054B1A68054B1B88EC
:101BC0009B1A834202D9104404F026BF00207047BC
:101BD000003400204634002038B50446074D29B1B2
:101BE00028682044BDE8384004F02EBF286820440F
:101BF00004F018FF0028F3D038BD00BF00340020E7
:101C00000020704700F1FF5000F58F10D0F8000859
:101C100070470000064991F8243033B100230822B0
:101C2000086A81F82430FFF7BFBF0120704700BF6A
:101C300004340020014B1868704700BF0010005C9E
:101C4000194B01380322084470B51D68174BC5F3C2
:101C50000B042D0C1E88A6420BD15C680A46013C81
:101C6000824213460FD214F9016F4EB102F8016B94
:101C7000F6E7013A03F10803ECD181420B4602D2A8
:101C80002C2203F8012B0424094A1688AE4204D101
:101C9000984284BF967803F8016B013C02F104027C
:101CA000F3D1581A70BD00BF0010005C2422002040
:101CB0006C8E0008022804D1054B4FF400129A6183
:101CC00070470128FCD1024B4FF40022F7E700BF18
:101CD00000100258022803D1044B20229A61704759
:101CE0000128FCD1014B0822F8E700BF0010025880
:101CF000022805D1064A536983F0200353617047D7
:101D00000128FCD1024A536983F00803F6E700BFBB
:101D100000100258002310B5934203D0CC5CC45489
:101D20000133F9E710BD0000013810B510F9013F8B
:101D30003BB191F900409C4203D11AB10131013A03
:101D4000F4E71AB191F90020981A10BD1046FCE78B
:101D500003460246D01A12F9011B0029FAD1704736
:101D600002440346934202D003F8011BFAE770478E
:101D70002DE9F8431F4D14460746884695F8242060
:101D800052BBDFF870909CB395F824302BB9202219
:101D9000FF2148462F62FFF7E3FF95F824004146F4
:101DA000C0F1080205EB8000A24228BF2246D6B24D
:101DB0009200FFF7AFFF95F82430A41B17441E4490
:101DC0009044E4B2F6B2082E85F82460DBD1FFF728
:101DD00021FF0028D7D108E02B6A03EB820383425E
:101DE000CFD0FFF717FF0028CBD10020BDE8F88344
:101DF0000120FBE704340020024B1A78024B1A70D2
:101E0000704700BF4434002010220020F8B5194C60
:101E1000194803F083FC2146174803F0ABFC246803
:101E20004FF47A70154ED4F89020154DD2F804383E
:101E3000114F43F00203C2F80438FFF74FFE20466B
:101E4000104903F0A5FDD4F890200424D2F80438FA
:101E500023F00203C2F804384FF4E133336055F83D
:101E6000040BB84202D0314603F0B6FB013CF6D178
:101E7000F8BD00BF68950008F04800202C34002011
:101E800014220020709500080C4B70B50C4D0446D0
:101E90001E780C4B55F826209A420DD00A4B002193
:101EA00018221846FFF75CFF0460014655F826002B
:101EB000BDE8704003F090BB70BD00BF443400200B
:101EC00014220020F04800202C34002030B50A44B1
:101ED000084D91420DD011F8013B5840082340F3C2
:101EE0000004013B2C4013F0FF0384EA5000F6D1BC
:101EF000EFE730BD2083B8ED10B5084C012208494A
:101F0000002001F0B3FE23783BB1064803F0DCFA71
:101F1000044803F00FFB0023237010BD4834002059
:101F20007C8E0008A43600201D482DE9F041036D89
:101F30002BB901224FF48051503005F067F8194E4B
:101F400033780BB1FFF7D8FF0324174F4FF0000889
:101F5000134D15492846C7F8048003F0DDFA2846DA
:101F600003F016F948B1013C284603F0E3FA14F0F7
:101F7000FF04EED1204634700FE00C4901220C48DA
:101F800001F074FE014618B1284603F09DFAEAE715
:101F9000084800F011F801203070BDE8F08100BF62
:101FA000A4360020483400203C2200207C8E00080B
:101FB0004C340020808E00080FB4002004B070471D
:101FC0000068704703460068596870470B0A017043
:101FD00043700B0C090E8370C1707047110A0270B8
:101FE00003714170110C120E8170C2701A0A427195
:101FF0001A0C1B0E8271C37170470000C36A02394C
:10200000023B8B4283BF4389006C01FB030000202D
:1020100070470000C2F307238A76CB760378032B40
:1020200001BF120C0A75120A4A75704700F10B01C4
:102030000022D30143EA520310F8012B52FA83F332
:102040008842DAB2F5D110467047000010B54178E9
:1020500004460020013102464901022A16BFA35C52
:10206000032203EBC03302F101021EBF9BB203EB5C
:10207000500398B29142F0D810BD000002684AB1F6
:10208000134613F8011B1F290DD93A29F9D1911CC8
:102090008B4202D04FF0FF3070471278302AF9D1CE
:1020A000036000207047014B187870479836002075
:1020B00038B50D46044618B9092000232B6038BDF9
:1020C0000368002BF8D01A78002AF5D08188DA88C6
:1020D0009142F1D1587804F0BFF910F00100EBD132
:1020E0002368EBE738B50D4640F25231144602F052
:1020F000B9F9FF2807D9012C0BD9030A022468700B
:102100002B70204638BD30B1002CFAD00124287045
:10211000F7E70024F5E70446F3E700002DE9F8436C
:102120000026D0F8008005460C468E76836B002B87
:102130004AD098F80030042B4BD13346354640271F
:1021400020E0B7F5187F80F0C480F90606F101069B
:1021500008BF0237D05B02372BB900F5205292B28C
:10216000B2F5006F0DD305F11A01C5F1FF0240EA87
:1021700003402144FFF7B6FF002800F0AA80054481
:1021800000200346D8F8102092F82310B142D8D886
:10219000002B40F09E80002D00F09B800023254402
:1021A000AB766373D8F81020137903F03701DB06A0
:1021B00021730BD402F13800FFF704FFC4E90001DA
:1021C00093896381D3892381BDE8F8830020014688
:1021D000F4E7C36C01335ED1EA6B00232E26551E53
:1021E000184615F8011F013020290CD0052908BF19
:1021F000E521092804D10B2B9EBFE71801337E731C
:10220000E718013379730B28EBD1E11800204873EC
:10221000A17E00294BD1002B40D06FF00C0604F1B9
:102220000D000825361B331810F8011B002938D083
:102230002E298BB24AD0A3F14101192903D8117B71
:102240000D4200D020330373EDE7B9F1000F05D143
:1022500000F520539BB2B3F5006F0BD307F11A01C1
:10226000C7F1FF0240EA09402144FFF73BFF48B1B4
:102270000744002002368146D8F80C30985B0028CD
:10228000E3D13846B9F1000F4FF0000218BF00202B
:1022900023189A76A0E7B1463746EDE73F23A376A9
:1022A0000123234400219976137B03B96373D37A06
:1022B00002F11C0003F03F0323730023FFF780FEAD
:1022C00020606360D38A6381138B7CE710250B4603
:1022D000B9E73F230125A37660E7000038B505463E
:1022E000002435F8020B08B9204638BD02F0EEF89C
:1022F0006308C2B203EBC43312FA83F39AB2C0F399
:10230000072303EB520303EBC2339CB2E9E700005F
:1023100037B5C37804461BB90025284603B030BD45
:1023200000F14C01826C01234078019104F0BAF86D
:10233000054680B9A36BE070A06C226BC31A934270
:10234000EAD2A3780199022BE6D1024401236078F6
:1023500004F0A8F8E1E70125DFE7000038B5836C59
:1023600005460C468B4210D0FFF7D2FF60B92246DB
:10237000012305F14C01687804F070F800281CBFB7
:102380004FF0FF340120AC6438BD0020FCE70000B2
:1023900038B500230446C3704FF0FF338364FFF762
:1023A000DDFF00284BD1B4F84A524AF655239D422E
:1023B00007D10B22254904F14C0006F05DFC0028F2
:1023C0003FD094F84C30EB2B03D01833DBB2012B09
:1023D0002ED84AF655239D4206D108221C4904F105
:1023E0009E0006F049FC48B3B4F85730B3F5007FBF
:1023F0001ED194F85930DBB15A1E1A4218D1B4F8E4
:102400005A30ABB194F85C30013B012B10D8B4F8D2
:102410005D306BB1B4F85F307F2B06D804F16C00EF
:10242000FFF7CEFDB0F5803F02D3B4F8623053B968
:102430004AF6552085420CBF0220032038BD0420F7
:10244000FCE70120FAE70020F8E700BFAC8E0008A7
:10245000B88E000802392DE9F04701F007044FF06B
:10246000010A466C05460AFA04F41746984606EB3C
:102470001136C1F3C809E4B2314628460136FFF7E8
:102480006DFF18B10120BDE8F087994605EB090200
:1024900092F84C30234214BF01210021414513D052
:1024A0006340013F82F84C3085F803A0EBD0640014
:1024B00014F0FF04EAD109F1010301244FF00009EF
:1024C000B3F5007FE1D1D7E70220DCE7012902461E
:1024D000F8B50C4640F28C800668F36A8B4240F2F5
:1024E00087803378013B032B00F28280DFE803F022
:1024F0000229384B04EB5405B16B304601EB5521F2
:10250000FFF72CFF10B14FF0FF30F8BD6F1CC5F383
:102510000805B16B3046354401EB572195F84C5016
:10252000FFF71CFF0028EED1C7F30807E3073E447E
:1025300096F84C0045EA00204CBF0009C0F30B00A0
:10254000E3E7B16B304601EB1421FFF707FF0028EA
:10255000D9D1640004F4FF742644B6F84C00D4E7E3
:10256000B16B304601EBD411FFF7F8FE0028CAD159
:10257000A40006F14C0004F4FE742044FFF720FD93
:1025800020F07040C1E7D0E90430D57953EA00016A
:1025900001D0916801B95DBB9168022DA4EB0101E6
:1025A0000DD1013B728940F1FF305B0A43EAC05311
:1025B000B3FBF2F399421BD81CD0601CA5E7032D96
:1025C00002D193698B42F8D8D3699BB9B16B30467D
:1025D00001EBD411FFF7C2FE002894D1A0004C36C5
:1025E00000F4FE703044FFF7EBFC20F000408CE775
:1025F00001208AE76FF0004087E70000F8B5066821
:1026000004460D463378042B0CBF4FF080524FF434
:1026100000128A4201D80220F8BDCA06FBD18268A6
:102620000163D2B9022B13D83389B3EB551FF2D90A
:10263000F36BA363A36B6263002BECD003EB552316
:102640004C36C5F308050020A3633544E563E3E792
:10265000F36BC271002BE7D01A4677897F02BD4227
:10266000114604D23046FFF7C9FCA063E2E72046DA
:10267000FFF72CFF431C024606D00128CBD9F36A92
:102680008342C8D9ED1BEAE70120C5E701292DE9FE
:10269000F04706460C46174608D9C36A8B4205D94F
:1026A0000378022B62D003D8012B22D0022552E0FE
:1026B000033B012BFAD8816B01EBD411FFF74EFEDF
:1026C0000546002847D1A40006F14C0304F4FE742B
:1026D0001C443378042B07D0204627F07047FFF7BF
:1026E0006FFC00F07040074339462046FFF76EFC50
:1026F0002FE001EB5108816B01EB5821FFF72EFE13
:10270000054640BB14F0010406F14C0908F1010A2A
:10271000C8F3080808BFFBB230461FBF19F80830DD
:1027200003F00F023B0103F0F00318BF134309F855
:1027300008300123B16BF37001EB5A21FFF70EFE55
:10274000054640B9CAF3080A44B1C7F3071709F8A8
:102750000A700123F3702846BDE8F08719F80A30A3
:10276000C7F3032723F00F031F43F0E7816B01EB4F
:102770001421FFF7F3FD05460028ECD1640006F1B3
:102780004C0304F4FF741F551919C7F307274F7042
:10279000DFE70000F8B504460E461746E3690BB9BB
:1027A0001846F8BD012BA6EB0305206814BFAA1C30
:1027B0003A46691CFFF76AFF0028F2D1E369013B42
:1027C000E361EBE701292DE9F84306460C4617467D
:1027D000056802D80220BDE8F883EB6A8B42F9D97C
:1027E0007AB9A14621463046A046FFF76FFE04465F
:1027F000B0B92B78042B02D1002F43D1F771002000
:10280000E9E72B78042B02D1C379022BE9D04FF0F2
:10281000FF3239462846FFF739FF0028E1D0DAE7D2
:102820000128D7D0421C01D10120D4E72B78042BFA
:1028300019D1EA6AAB69023A93421CD308F101024A
:10284000A2420CD02B78042B08D10023A2EB090262
:1028500049462846FFF7FEFD0028BCD1A146EB6A99
:10286000A342BFD8C5E7002241462846FFF70EFF26
:102870000028DED0AFE70133AB612B7943F00103D1
:102880002B71DBE7F3798BB9B468BC4202D1022328
:10289000F371B4E721463046FFF718FE012899D9B5
:1028A000431CC1D001348442EFD0A8E7032BA6D14A
:1028B000B368BB42A3D8B2691344BB429FD3E6E7D7
:1028C00070B5C3790446032B06D181688369CD189E
:1028D000A94203D10023E371002070BD4E1C206883
:1028E0003246FFF7D3FE0028F7D13146F0E700006B
:1028F0002DE9F74305460191FFF70AFD044600283C
:1029000049D105F14C09019928464FF40072FFF7AF
:1029100075FB2146A86407464846FFF721FA6C89F3
:102920006402B4F5004F28BF4FF40044B4F5007FB3
:102930002FD9204604F022FA804630B122460021E9
:10294000640A0026FFF70CFA09E06408EEE7234664
:10295000BA194146687803F0A5FD18B926446B8979
:102960009E42F4D3404604F019FA6889801B18BFD0
:10297000012003B0BDE8F08301366B899E42F4D29A
:102980000123BA194946687803F08CFD0028F3D07A
:10299000EBE70026F1E70120EBE70000F8B504467D
:1029A000FFF7B6FC0546002842D12378032B37D128
:1029B0002779012F34D104F14C0601464FF40072FF
:1029C0003046FFF7CDF955234122722184F84A326F
:1029D000AA2304F50D7084F84F2084F84B3252235B
:1029E00084F8301284F84C3084F84D30612384F838
:1029F000311284F84E3084F83332A16984F83222DF
:102A0000FFF7E4FA616904F50E70FFF7DFFA626B15
:102A10003B46314601326078A26403F043FD2571E4
:102A200000226078114603F061FD003818BF0120D4
:102A3000F8BD000000232DE9F0430B6085B00F4680
:102A40001546FFF71BFB061EC0F2B281804B53F800
:102A50002640002C00F0AE813C6005F0FE05237896
:102A60006BB1607803F0F8FCC70708D41DB110F013
:102A7000040500D00A25284605B0BDE8F0830023F0
:102A8000F0B22370607003F0D3FCC10700F19481B1
:102A90000DB14207EED400212046FFF779FC022851
:102AA00040F099806E4604F2122304F2522132461D
:102AB00018461033FFF784FA42F8040B8B42F7D123
:102AC000002556F8041B00297DD02046FFF760FC46
:102AD000012879D80128A26C40F0C08004F1570386
:102AE00004F18C0113F8015B002D7BD18B42F9D1ED
:102AF000B4F8B430B3F5807F74D194F8B830092BB2
:102B000070D104F19400FFF75DFA4FF0FF3317180E
:102B100041F10001BB4275EB010363D304F1A00056
:102B2000FFF74EFA94F8BA302063012BA37059D105
:102B300094F8B99003FA09F91FFA89F36381002B1D
:102B400050D0444B04F1A800FFF73AFA06469842E9
:102B500048D8831C626304F1A400E362FFF730FAF3
:102B600000EB020804F19C00C4F84080FFF728FA4B
:102B700010441FFA89F2A06306FB02F313EB08036B
:102B800045EB05029F4271EB02032BD32E4604F165
:102B9000AC00FFF715FAE06365B96389B34221D948
:102BA000E16B2046FFF72AFA81192046FFF7D6FB92
:102BB00098B90136631993F84C30812B14D0203525
:102BC000C5F30805E8E703200135042D7FF479AF4C
:102BD000042807D101E0042801D101254BE7012891
:102BE0007FF678AF0D2546E705F1140004F14C0699
:102BF0003044FFF7E5F901280546F3D9E36A83423B
:102C0000F0D96189821E236C02FB01336364A16BDE
:102C1000204601EBD511FFF7A1FB0028DDD105F01F
:102C20007F0006EB8000FFF7CBF9431C03D0013592
:102C3000A842ECD0D6E70425C4E90500064A257071
:102C400000251388E56101339BB21380E38012E70E
:102C50009C360020FDFFFF7FA0360020B4F85730DF
:102C6000B3F5007FBED1B4F8626026B904F17000FC
:102C7000FFF7A6F9064694F85C302663591EA37048
:102C80000129AFD894F859506581002DAAD0691E4A
:102C90002942A7D1B4F85D8018F00F0FA4F808807E
:102CA000A0D1B4F85F0018B904F16C00FFF788F9FF
:102CB000B4F85A10002995D006FB03FE01EB181C4E
:102CC000F44460458ED3A0EB0C00A842B0FBF5F3B2
:102CD00088D33E48834285D84FF6F57083426DD93C
:102CE00003259F1C114402EB0C03032DE762626372
:102CF000A16323644CD1B4F8763053EA08037FF41F
:102D000071AFBB0004F17800FFF75AF9E06303F2FA
:102D1000FF13B6EB532FFFF465AF4FF0FF33032DD6
:102D2000C4E905334FF08003237187D1B4F87C30B8
:102D3000012B83D1511C2046FFF710FB00287FF4A4
:102D40007DAFB4F84A224AF6552320719A427FF4A7
:102D500075AF1F4B04F14C00FFF732F998427FF436
:102D60006DAF03F1FF5304F50C70FFF729F903F57C
:102D70000053203398427FF461AF04F50D70FFF7E4
:102D80001FF9A06104F50E70FFF71AF9606155E7AD
:102D9000B8F1000F3FF426AF7144022D4FEA47030C
:102DA000E1631EBFD91907F0010303EB5103AEE73E
:102DB0000B2560E60C255EE603255CE640F6F5751E
:102DC000AB428CBF022501258BE700BFF5FFFF0F4B
:102DD000525261412DE9F84F07460568884649B9C6
:102DE0006E69C6B1EB6AB34298BF0126AB69A3B95D
:102DF000002405E0FFF76AFB0128044603D80124FC
:102E00002046BDE8F88F421C00F0D280EB6A834276
:102E1000F6D84646EAE70126E8E72A78EB6A042A6C
:102E200040F08380A6F1020A023B4FF0010B9A4565
:102E300028BF4FF0000AD146696C284601EB1931D2
:102E4000FFF78CFA00283BD109F00703EA6AC9F3BF
:102E5000C8010BFA03F3901EDBB26A184C4609F165
:102E6000010992F84C20814502EA030233BF5B005E
:102E700000234FF40071DBB228BF9946B2B9023487
:102E8000631E0333BCD80123214628461A46FFF7A8
:102E9000E1FA0228B3D0012800F08A80B8F1000FCF
:102EA00013D10223FB710028A9D130E0CA450AD012
:102EB000002BD2D10131B1F5007FBDD20123CCE787
:102EC0004FF0FF34DCE70024DAE7FB79022B07D16F
:102ED000731CA342E7D0BB68F31ABB610323FB71E9
:102EE00008F10102FB69A24205D113B10133FB6174
:102EF000D9E70223FBE70BB90123FB6122464146D8
:102F00003846FFF747FC00284FD10123FB61EA6AEE
:102F1000AB69023A6C6193429CBF03F1FF33AB6132
:102F20002B7943F001032B716AE7464514D1741CD9
:102F30003846A34298BF02242146FFF7C7FA01286A
:102F40003FF45DAF431C33D0E0B16B69012B03D973
:102F5000EA6A934238BF1E4634460134EB6AA34204
:102F600003D8012E7FF644AF022421463846FFF7EE
:102F7000ADFA48B101283FF442AF013018D0B44255
:102F8000EBD135E7002CE7D04FF0FF322146284641
:102F9000FFF77CFB48B9B8F1000FB8D02246414694
:102FA0002846FFF773FB0028B1D001287FF427AF34
:102FB0004FF0FF3424E700002DE9F843066804468B
:102FC000076B894633782037042B0CBF4FF08053B2
:102FD0004FF40013BB429CBF00238363836B73B128
:102FE000C7F30808B8F1000F3CD10133416B83638C
:102FF00039B93389B3EB571F34D80023A3630420B6
:103000000AE07389013B13EA57232BD1FFF75EFADD
:103010000128054602D80220BDE8F883421C01D1F0
:103020000120F9E7F36A834216D8B9F1000FE4D022
:10303000616B2046FFF7CEFE0546C8B10128EAD0F5
:10304000431CEDD001463046FFF752FC0028E7D183
:10305000E37943F00403E371294630466563FEF7E4
:10306000CDFFA0634C36002027634644E663D3E7D8
:103070000720D1E7F8B50E46002104460768FFF7A0
:10308000BDFA98B90546A16B3846FFF767F968B9EC
:103090003A78E36B042A1B780CD11B060ED5054643
:1030A00001212046FFF788FF0028ECD0042808BF44
:1030B000072006E0E52B01D0002BF0D10135B54209
:1030C000EED1F8BDC16C4B1C2DE9F04104460568FA
:1030D000066B1FD1E5274FF00108A16B2846FFF7CB
:1030E0003DF998B92A78E36B042A09BF1A781F7052
:1030F00002F07F021A7085F80380236BB3420DD271
:1031000000212046FFF758FF0028E6D0042808BF1A
:10311000022003E0FFF772FA0028DBD0BDE8F0815F
:103120002DE9F04105460068A96B0669FFF716F91D
:10313000044620B9EB6B1A78852A03D00224204676
:10314000BDE8F081324603F1200153F8040B8B42B5
:1031500042F8040BF9D1777801377F01A7F16003BA
:10316000B3F5007FEAD800212846FFF725FF0428A1
:103170000446E3D00028E2D1A96B2868FFF7EEF8F7
:1031800004460028DBD1EB6B1A78C02AD6D106F1B1
:10319000200203F1200153F8040B8B4242F8040B88
:1031A000F9D196F823300F222C33B3FBF2F3B7EBAF
:1031B000431FC3D34FF0400800212846FFF7FCFE11
:1031C00004280446BAD00028B9D1A96B2868FFF7B3
:1031D000C5F804460028B2D1EB6B1A78C12AADD1EC
:1031E000B8F5187F09D206EB080203F1200153F865
:1031F000040B8B4242F8040BF9D108F12008474533
:10320000DAD8B8F5187F9AD83046FEF71FFF7388D2
:10321000834294D092E700000B68002210B503604F
:1032200004460B6A83604B6AC261C37123F0FF03DB
:10323000896AC0E90432C164FFF7E0F920B9204689
:10324000BDE81040FFF76CBF10BD0000F8B5036883
:10325000054601271C692046FEF7F8FEA070000A0B
:103260006678E0702846E96CFFF7C8F920B10228BB
:1032700028BF0220C0B2F8BDA96B2868FFF76EF81E
:103280000028F4D1EB6B04F1200254F8041B9442A3
:1032900043F8041BF9D12B68DF70002EE7D0002122
:1032A0002846013EFFF788FEE0E700002DE9F843DD
:1032B0004FF0FF0806460768042445464FF6FF799D
:1032C000B16B11B9002C73D063E03846FFF746F8B4
:1032D000044600285DD1F06B0378002B6ED03A785D
:1032E000042A11D1852B4DD1336B3046F364FFF79F
:1032F00017FF044600284CD13B691B7903F03F03BC
:10330000B3712046BDE8F883C27AE52B02F03F0294
:10331000B27143D02E2B41D022F0200108293DD09C
:103320000F2A40D1590637D503F0BF05336B90F80B
:103330000D80F364437B434530D1428B72BB0378ED
:103340000D21FC6823F04003DFF874E0013B4B43A0
:1033500001211EF801CB30F80CC009B3FF2B1DD89A
:1033600024F813C06146013301320D2AF1D10278ED
:10337000520605D521B1FF2B10D8002224F81320C6
:10338000013DEDB200213046FFF716FE044600284D
:1033900096D00023B363B4E7AB42CBD0FF25F1E76F
:1033A000CC45E1D0FAE72DB9FEF740FE404501D10A
:1033B0000024A6E74FF0FF33F364A2E70424E8E714
:1033C000548F00082DE9F04F002187B00446D0F853
:1033D0000090FFF713F9804670B999F80030042B7C
:1033E00033D1D9F80C00FEF779FF07462046FFF7E6
:1033F0005DFF054620B18046404607B0BDE8F08F2E
:10340000D9F810309A8CBA42F0D193F823B0402604
:103410005D4506D1D9F80C3033F81530002BE5D1D5
:10342000EAE7F106D9F8103008BF0236985B01F0E0
:103430004DF8D9F80C30824633F8150001F046F803
:103440008245D3D102360135E2E74FF0FF0A4FF053
:10345000FF3B5546C4F84CB0A16B4846FEF77EFFD3
:1034600000285CD1E66B3778002F77D0F27AE52F11
:1034700002F03F03A37103D0120704D50F2B04D031
:10348000C4F84CB04FE00F2B54D194F84B30580691
:103490003FD4790645D5236B07F0BF0796F80DA0FA
:1034A000E364737B53453ED1738B002B3BD135785E
:1034B0000121D9F80C3005F03F0501930D23013DA2
:1034C0005D43284B13F8012BB25A71B3FF2D0593BE
:1034D00029D81046049200F0F9FF6B1C0390029368
:1034E000019B33F8150000F0F1FF039981421AD1D6
:1034F000049A029D1146059B1B4A9342E2D1337800
:103500005A0604D519B1019B33F815305BB97D1EFD
:10351000EDB200212046FFF74FFD00289CD08046E9
:103520006AE7BD42BDD0FF25F3E74FF6FF70824248
:10353000E2D0F8E72DB93046FEF778FD50453FF46C
:103540005BAF94F84B30DB079AD40B2204F14001B7
:10355000304605F091FB002892D14DE74FF004086A
:103560004AE700BF548F0008618F00082DE9F04F33
:1035700090F84BB099B004461BF0A00540F068816C
:103580000668F26832F81530002B4AD13378042BE4
:1035900040F087800F230E352046B5FBF3F5A91CBC
:1035A000FFF768FD8146002877D1236B0135A3EB37
:1035B0004515E3795A07E56435D523F00403204621
:1035C000E371FFF77DF950BB4FF0FF32616B20468E
:1035D000FFF7E0F818BBA3682BB3214604A8FFF758
:1035E0001BFEE0B970894FF40071D4E90423E0FBBD
:1035F00001233069C4E904233830FEF7EFFC306959
:10360000D4E904232830FEF7E9FCE379326904A801
:1036100043F0010382F82130FFF718FE18B181460C
:103620003BE00135AEE7D6E90354402200212046B5
:10363000FEF796FB8523012140222370C0234FF023
:10364000C10C04EB010884F8203000231E469E467E
:10365000571C04F802C0F0B2023204F807E021B1AE
:1036600035F8131009B10133DBB20F0AA15408F881
:1036700002700232D706F2D135F813700136002FEE
:10368000E6D184F82330831C28466370FEF726FEBB
:1036900084F82400000A84F82500484619B0BDE8E3
:1036A000F08F04F140070DF1100A1BF0010F97E8AD
:1036B00007008AE8070000F0D38040234FF001089C
:1036C00084F84B30BC46F368B8F1050F9AE8070060
:1036D000ACE803002CF8022B4FEA12428CF80020D1
:1036E00059D9981E424630F8021F002942D10DF1E7
:1036F0000F0C072102F00F0E914612090EF1300057
:10370000392888BF0EF1370001390CF8010902D0C1
:10371000B9F10F0FEED818AB7E205A1802F8580CEA
:1037200038460022914206D010F801CB02F1010E7A
:10373000BCF1200F31D104F13F0C072902F1010245
:1037400097BF18AB20205818013198BF10F8580CBB
:10375000072A0CF80200F0D92046FFF733FE814615
:10376000002878D108F10108B8F1640FAAD14FF010
:10377000070992E74FF0100C01F0010E49080EEB1B
:103780004202D30344BF82F4883282F02102BCF1AA
:10379000010CF1D1A7E74246A9E77246C2E7216BC7
:1037A0002046A1EB4511FEF729FF814600287FF452
:1037B00074AF4FF6FF783846FEF738FC0190A16BE6
:1037C0003046FEF7CBFD814600287FF466AFE36B01
:1037D000E9B2019A4FF00D0CD6F80CE05A734FF095
:1037E0000F02DFF8E0A0DA724A1E18730CFB02F237
:1037F00084469876D87640451AF8019B0CF1010C66
:1038000018BF3EF8120003EB090B18BF013203F892
:1038100009004FEA1029002808BF4046BCF10D0FEF
:103820008BF80190E7D1404502D03EF812200AB94A
:1038300041F040011970012300212046F370FFF789
:10384000BBFB814600287FF428AF013DB7D11BE0C8
:103850004FF0060921E704287FF41FAF84F84BB02E
:103860001BF0020F20461BBF0C350D210125B5FBB7
:10387000F1F518BF01352946FFF7FCFB814600280A
:103880007FF40BAF013D8AD1A16B3046FEF766FD98
:10389000814600287FF401AF01462022E06BFEF74D
:1038A0005FFAE36B03CF18605960BA7839889A726F
:1038B000198194F84B30E26B03F018031373012362
:1038C000F370EAE6548F000810B504460A46343017
:1038D000FEF776FB886004F13800FEF773FBC2E95F
:1038E000040194F8213003F00203D3710023D36163
:1038F00010BD000003284B8B04BF8A8A43EA0243B1
:10390000184670472DE9F04F0B7899B00446894668
:103910002F2BD0F800B001D05C2B09D14A46137888
:10392000914601322F2BFAD05C2BF8D0002301E016
:10393000DBF81C30A3600023E3619BF80030042B0C
:103940001ED1A368E3B1DBF82030214604A823622E
:10395000DBF824306362DBF82830A362FFF75CFCFD
:103960000346002854D1DBF8102002F13800FEF79E
:1039700027FBC4E9040392F8213003F00203E3714A
:1039800099F800301F2B00F235818023002120465A
:1039900084F84B3019B0BDE8F04FFEF72FBE494612
:1039A0000B78894601312F2BFAD05C2BF8D01F2BD6
:1039B0008CBF00250425012F2FD113882E2B31D148
:1039C000002322F8173004F140029F428CBF2E21C1
:1039D000202101330B2B02F8011BF6D145F0200505
:1039E000204684F84B50FFF7EDFC94F84B3000284C
:1039F00000F0E78004280BD1990603F0040240F19F
:103A0000DC80002A00F0F6808023002084F84B3010
:103A100019B0BDE8F08F0425CDE7022F02D15388FD
:103A20002E2BCAD0911E87BB002322F81730002FFF
:103A300000F0118132F81300194601332028F9D023
:103A400009B92E2801D145F00305901E30F8173032
:103A50002E2B01D0013FF9D14FF020334FF0000A57
:103A60006364D0462364C4F847300823481C32F806
:103A700011600090F6B1202E03D02E2E0DD1B84249
:103A800010D045F003050099F0E731F81730202BEE
:103A900001D02E2BC8D1013FC5E79A4505D2009928
:103AA000B9423BD10B2B30D101E00B2B27D145F094
:103AB00003050B2394F84020E52A04BF052284F86F
:103AC0004020082B04BF4FEA88085FFA88F808F006
:103AD0000C030C2B03D008F00303032B01D145F09A
:103AE0000205A8073FF57CAF18F0010F18BF45F09D
:103AF000100518F0040F18BF45F0080570E700998D
:103B0000B94202D045F00305D4D84FEA88080B2308
:103B10004FF0080A00975FFA88F8B4E77F2E15D9AE
:103B2000304640F25231CDE9022345F002030193C1
:103B300000F098FC10F0800F0646DDE9022316D055
:103B400000F07F0646498E5D019D46B331464548EB
:103B5000CDE9012305F0FEF8DDE90123F8B9A6F16E
:103B6000410189B219291ED848F0020810E0FF2847
:103B7000EAD9591E8A4503D345F003059A4682E7E0
:103B800004EB0A01000A0AF1010A019D81F84000D4
:103B900004EB0A010AF1010A81F8406073E745F07D
:103BA00003055F26F4E7A6F1610189B219299EBFDA
:103BB000203E48F00108B6B2EAE7002A08BF052017
:103BC00026E75A073FF524AFA379DB0645D59BF8D6
:103BD0000000042835D1A3682146E27923622369D5
:103BE000DBF8100023F0FF0313436362E36CA3626E
:103BF000FFF76AFE23680027DA6819F8010B00282E
:103C00003FF409AF40F25231009200F04BFC054600
:103C100008B31F28009A7FF6FEAE2F283FF4BFAEF0
:103C20005C283FF4BCAE7F2805D801460E4805F05D
:103C300091F8009A78B9FF2F0DD022F8175001376C
:103C4000DBE7216B0BF14C03C1F308011944FFF7CB
:103C500051FEA060CEE70620DAE60520D8E600BFD8
:103C6000D48E0008CD8E0008C48E00081FB5CDE9A3
:103C7000001003A814460391FEF700FA002815DB94
:103C80000B4A52F820300BB100211970019B0BB187
:103C90000021197042F820302CB1002201A9684699
:103CA000FEF7C8FE0446204604B010BD0B24FAE718
:103CB0009C3600202DE9F04798B0904605460191CA
:103CC000002800F0528102F03F0603A901A8324605
:103CD000FEF7B0FE002840F04681039B4FF48C6055
:103CE000049303F04BF80746002800F04081039B43
:103CF00000F500720199D86004A81A61FFF702FE6E
:103D0000044620B99DF95B30002BB8BF062418F09B
:103D10001C0F00F0CD80002C4CD0042C40D104A806
:103D2000FFF724FC044600283AD146F00806039B1E
:103D30001A78042A40F08380186929462B60FFF71F
:103D4000C3FD039B1E22002118690230FEF708F80C
:103D5000039C00211A2220692630FEF701F823690E
:103D600020221A71246903F027F801460122083441
:103D70002046FEF72BF9039B04A81B6983F821203A
:103D8000FFF764FA044658B9A96801B30246284609
:103D9000FEF718FDAB68039A0446013B5361B4B1CA
:103DA000384602F0FBFF0CB100232B60204618B010
:103DB000BDE8F0879DF8163013F0110F40F08480B5
:103DC00018F0040F40F0C98018F0080FAFD1039A23
:103DD00031071399936C48BF46F04006E964AB6421
:103DE0001078042872D1069B9DF817102B62089B4F
:103DF000106923F0FF030B4329466B62179BAB62EC
:103E0000FFF762FDDDF80CA00024002205F1500848
:103E1000BAF8063021464046C5F800A0AB80002322
:103E200085F8306085F831406C64C5E90E234FF4A5
:103E30000072FDF795FFB20653D40024B0E702F0FC
:103E4000BBFF0146009013980E30FEF7BFF81398A1
:103E500000991630FEF7BAF8039C13992078FFF703
:103E600049FD202300228046CB7220461399FEF79D
:103E7000D1F8139B002201211A775A779A77DA77C3
:103E8000039BD970B8F1000FA1D0414604A8D3F824
:103E90004890FEF797FC0446002881D149460398D4
:103EA000FEF75CFA039B044608F1FF30586176E7A1
:103EB000002C7FF475AF9DF81630DC064FD418F057
:103EC000020F84D0D80782D5072469E7FFF712FDD7
:103ED0000023A86001F11C00FEF772F86B612861F5
:103EE00090E7D5E9046956EA0903A6D0BAF80AA012
:103EF000A9684FEA4A2AC5E90E69B24574EB09037D
:103F00001BD300242964002C7FF44AAFC6F30803B6
:103F1000002B92D0039C2046FEF770F808B3760A77
:103F20000123414646EAC95682196A64607802F064
:103F300095FA041E18BF012432E72846FEF7C6FA98
:103F4000B6EB0A06014669F10009012803D9431CB2
:103F5000D3D10124D6E70224D4E7082420E704249F
:103F60001EE702241CE704461EE709241EE711246D
:103F70001CE700002DE9F04F994685B000238846E4
:103F800003A90446C9F800301646FEF791F8054625
:103F900080BB94F831506DBB94F8303013F00103BE
:103FA000009300F0A68004F1500AD4E90432D4E969
:103FB0000E011B1A62EB0102B34272F1000238BF1C
:103FC0001E46BEB1D4E90E10C1F30803002B40F029
:103FD0008280039B5A894B0A013A43EAC0531A4034
:103FE0001BD151EA000309D1A06801280DD8022590
:103FF00084F83150284605B0BDE8F08F216C20468A
:104000000192FEF763FA019AEFE7431C04D1012302
:10401000009D84F83130EDE72064DDF80CB0216CB0
:104020005846FDF7EBFF0028E1D0B6F5007F02EB24
:10403000000731D3BBF80A1002EB5620730A8842FE
:104040009BF8010088BF8B1A3A464146019302F063
:1040500005FA0028DBD194F93020019B002A0BDA05
:10406000606CC01B984207D24FF40072514608EBB7
:104070004020FDF74FFE019B5F02D9F80030F61B90
:10408000B8443B44C9F80030D4E90E32DB1942F1A0
:104090000002C4E90E3294E7626CBA421AD094F975
:1040A0003030002B0DDA012351469BF8010002F05D
:1040B000F9F90028ABD194F8303003F07F0384F88D
:1040C0003030039801233A465146407802F0C6F951
:1040D00000289CD16764A16B4046C1F30801C1F57B
:1040E00000775144B74228BF37463A46FDF712FEE3
:1040F000C3E707257EE7000070B596B00E460022A4
:10410000019002A901A8FEF795FC0446E0B94FF41E
:104110008C6002F033FE0546D8B1029B00F50072B8
:104120000199D86002A81A61FFF7ECFB044640B978
:104130009DF95330002B0ADB1EB1314602A8FDF772
:10414000EDFF284602F02AFE204616B070BD062478
:10415000F7E71124F8E7000070B5B8B0022201902B
:1041600003A901A8FEF766FC044608BB039B4FF4B5
:104170008C60109302F002FE0546002866D0039B77
:1041800000F500720199D86010A81A61FFF7BAFB18
:10419000044650B99DF88B30980655D4190653D46F
:1041A0009DF84630DA0706D50724284602F0F6FDCA
:1041B000204638B070BD039B04931878042814D1AE
:1041C00004A91869FFF780FB069E9DF84630DB06C0
:1041D00010D410A8FEF776FF04460028E5D156BBA0
:1041E0000398FEF7DBFB0446DFE71F99FFF782FB2E
:1041F0000646EAE7039BDA69B242D5D02493002150
:10420000269624A81B78042B01BFDDE90823CDE9FD
:1042100028239DF817308DF89730FEF7EFF9044604
:104220000028C2D124A8FFF741F804460028BBD0DB
:104230000428BAD1CDE70246314604A8FEF7C2FAF7
:1042400004460028B1D1CBE70624AEE71124AFE73E
:10425000F0B5BDB0CDE900106846FDF70FFF0222B2
:1042600003A901A8FEF7E6FB0446002841D1039B01
:104270004FF48C60149302F081FD0546002800F095
:10428000EE80039B00F5007214AE0199D8601A61AC
:104290003046FFF737FB044640BB9DF89B3013F0D8
:1042A000A00F40F0D880039B009F1A78042A68D1A1
:1042B0001B6904AC03F1400C1868083353F8041C64
:1042C0002246634503C21446F6D15022314628A83F
:1042D000FDF720FD394628A8FFF714FB0446002807
:1042E0004CD12A9A169B9A4206D00824284602F0FE
:1042F00055FD20463DB0F0BD349A209B9A42F4D142
:1043000028A8FFF733F904460028EFD1039B04AF38
:104310001B6993F801E093F823C09C8C3A4608335C
:1043200003CAB24243F8080C43F8041C1746F5D1FF
:10433000039B28A81B6983F801E0039B1A6982F894
:1043400023C01A6982F82440240A82F825401A6999
:104350001379D9065CBF43F020031371FEF776FF93
:1043600004460028C2D13046FEF7ACFE04460028C1
:10437000BCD10398FEF712FB0446B7E70428B5D179
:10438000BEE7239A04AB02F1200C1068083252F801
:10439000041C1C46624503C42346F6D15022314614
:1043A00028A8FDF7B7FC394628A8FFF7ABFA044662
:1043B00000284CD12A9A169B9A4296D1349A209B77
:1043C0009A4292D128A8FFF7D1F8044600288DD14F
:1043D00037990DF11D030DF12D0001F10D0253F878
:1043E000044B834242F8044BF9D11888012710800E
:1043F0009B7893709DF81B30039CDA0658BF43F0FE
:104400002003CB72E770CB7ADB06ACD5169A2A9BD9
:104410009A42A8D02078FFF76DFA01462046FDF7B2
:10442000EDFD0146C8B12046FDF798FF044600287F
:104430007FF45CAF039890F86D302E2B93D12A9ABD
:1044400000F16C01FDF7E6FD039BDF708BE70428AC
:104450007FF44CAFB6E7062448E7022446E7112470
:1044600047E700007F2810B501D880B210BDB0F535
:10447000803F13D240F2523399420FD108490022B3
:1044800031F8024B93B2844203D103F18000C0B2F1
:10449000ECE70132802AF3D11346F6E70020E5E786
:1044A000149200087F280DD940F25233994208D166
:1044B000FF2806D800F10040034B803833F8100085
:1044C00070470020704700BF14920008B0F5803F8D
:1044D000F0B522D21F4A83B21F49B0F5805F28BFD2
:1044E0000A46141D34F8042C2146AAB1934213D372
:1044F00034F8025C2E0AEFB252FA85F5A84222DAAD
:10450000082E09D8DFE806F0050A10121416181A4A
:104510001C00801A34F810301846F0BD981A00F0CC
:1045200001001B1A9BB2F7E7103BFBE7203BF9E7C2
:10453000303BF7E71A3BF5E70833F3E7503BF1E789
:10454000A3F5E353EEE70434002ECBD101EB470291
:10455000C7E700BF648F000858910008084BC26A83
:10456000994228BF1946836C50688B4210B506D912
:104570005A1E4C0002EB4103B3FBF4F3184410BD88
:1045800020BCBE0001F001038A0748BF43F00203CC
:104590004A0748BF43F008030A0748BF43F0040333
:1045A000CA0648BF43F010038A06426B48BF43F077
:1045B000200313434363704710B5074C204600F0B7
:1045C0009FFF064B0022C4E91023054BA364054B53
:1045D000E363054BE36410BDA436002000240248C9
:1045E00000B4C404F8360020F8380020C36A0BB9C0
:1045F000104BC3620379012B11D10F4B98420ED19E
:104600000E4BD3F8DC2042F40072C3F8DC20D3F860
:10461000042142F40072C3F80421D3F80431436C3E
:1046200000221A65DA621A605A605A624FF0FF324D
:104630009A63704714930008A4360020004402587F
:104640000379012B1BD0436C00221A65DA621A60D1
:104650005A605A624FF0FF329A63094B98420ED16A
:10466000084BD3F8DC2022F40072C3F8DC20D3F826
:10467000042122F40072C3F80421D3F804317047F6
:10468000A43600200044025810B5446C0649FFF7D8
:1046900065FF6060236842F2107043F003032360FB
:1046A000BDE8104001F04CBD801A06000129F8B5A4
:1046B000466C0B4F09D175680A493D40FFF74EFF24
:1046C000054345F480557560F8BD746806493C4063
:1046D000FFF744FF044344F480547460F4E700BFE0
:1046E00000ECFFFF80F0FA0240787D01436C00226D
:1046F0005A601A6070470000426C0129536823F425
:10470000404304D0022905D001B95360704743F4F7
:104710008043FAE743F40043F7E70000436C41F4B9
:1047200080519A60D9605A6B1206FCD580229A6338
:104730007047000010B541F48851446CA260E160FC
:10474000616B11F04502FBD0A26311F0040203D0AB
:10475000FFF718FF012010BD616910461960FAE7E4
:1047600010B541F48851446CA260E160616B11F0B6
:104770004502FBD0A26311F0050203D0FFF702FF50
:10478000012010BD616910461960FAE773B5134640
:1047900004460E46302282F31188426CD26B32B14D
:1047A0004FF0FF314030019301F0D6FC019B606C6B
:1047B00000220265C263C262456B15F4807504D1A4
:1047C00085F31188012002B070BD4FF0FF31816385
:1047D00082F31188012E06D90C21204602B0BDE8D3
:1047E0007040FFF7BDBF1046EDE7000073B5446CA5
:1047F0000E4600250192616BA1632565E562FFF716
:10480000C1FE012E07D9019B2A460C2102B0BDE84A
:104810007040FFF7A5BF02B070BD000010B541F4B5
:104820009851446CA260E160616B11F04502FBD0CD
:10483000A26311F03F0203D0FFF7A4FE012010BDD8
:10484000216A10461960E1695960A169996061693E
:10485000D960F4E72DE9F74304460191006D01A901
:104860001746984602F0EAFB064600284AD0626CDA
:104870002046DDF804905568C5F3090501356B0045
:10488000A56CB5FBF3F54FF47A73B5FBF3F55D4317
:10489000556200F0FBFD50BB636C4FF0FF32012509
:1048A0004146C3F8589020461D659A634FF49572AF
:1048B000DA6342F207029F62DA62E36C0A9AFFF758
:1048C0004FFFA0B9E26C104B11680B407BB9294631
:1048D0002046FFF75BFF054648B92E463A46019948
:1048E000206D02F0D3FB304603B0BDE8F0833A46BA
:1048F0000199206D02F0CAFBE26C01212046FFF70E
:1049000075FFF0E70126EEE708E0FFFD2DE9F7432C
:104910001F46436C01924FF47A725D6804468846E4
:10492000C5F3090501356E00856CB5FBF6F5B5FBE1
:10493000F2F555435D6200F0A9FD20B1012528463E
:1049400003B0BDE8F0837E0201A9206D324602F07B
:1049500075FB05460028F1D0636C019AD4F84C90A1
:104960009A6501221A654FF0FF329A634FF49572EF
:10497000DA639E62236BDB064B4658BF4FEA48283A
:10498000012F42461BD912212046FFF7E9FEC0B98C
:10499000D9F80020104B13409BB9636C42F293028C
:1049A00039462046DA62E26CFFF7F0FE804640B9F5
:1049B00032460199206D454602F068FBBFE71121A0
:1049C000E2E732460199206D02F060FBE26C394665
:1049D0002046FFF70BFFB2E708E0FFFD2DE9F341AA
:1049E0001F46436C01924FF47A725D680446884614
:1049F000C5F3090501356E00856CB5FBF6F5B5FB11
:104A0000F2F555435D6200F041FD20B101252846D5
:104A100002B0BDE8F0817E0201A9206D324602F0AD
:104A200043FB05460028F1D0636C019A9A65012288
:104A30001A654FF0FF329A634FF48D72DA639E620B
:104A4000236BE66CDB06334658BF4FEA4828012F3C
:104A5000424619D919212046FFF782FEB0B93268C3
:104A60000F4B134093B9636C42F2910239462046D2
:104A7000DA62E26CFFF78AFE064638B901993546DC
:104A8000206D02F03DFBC2E71821E4E70199206D9B
:104A900002F036FBE26C39462046FFF7A7FEB6E788
:104AA00008E0FFFD12F0030F2DE9F04107460C4628
:104AB00015461E4617D00E44B44202D10020BDE870
:104AC000F0810123FA6B21463846FFF71FFF0028CB
:104AD000F5D128464FF40072F96B05F500750134E5
:104AE000FDF718F9E8E7BDE8F041FFF70FBF000058
:104AF00012F0030F2DE9F04107460C4615461E46FD
:104B000017D00E44B44202D10020BDE8F0812946FE
:104B10004FF40072F86B05F50075FDF7FBF8012303
:104B2000FA6B21463846FFF759FF0028EDD10134D2
:104B3000E8E7BDE8F041FFF751BF000000207047F3
:104B4000302310B583F311880024436C4030214694
:104B5000DC6301F00FFB84F3118810BD0268436829
:104B60001143016003B1184770470000024A1368FF
:104B700043F0C0031360704700480040024A1368C6
:104B800043F0C0031360704700500040024A1368AE
:104B900043F0C0031360704700780040064BD3F821
:104BA000E8200243C3F8E820D3F810211043C3F8EB
:104BB0001001D3F8103170470044025837B5274C24
:104BC000274D204600F0FCFC04F114000094002363
:104BD0004FF40072234900F097F94FF40072224914
:104BE00004F138000094214B00F010FA204BC4E986
:104BF0001735204C204600F0E3FC04F1140000942B
:104C000000234FF400721C4900F07EF94FF400724B
:104C10001A4904F138000094194B00F0F7F9194BC8
:104C2000C4E91735184C204600F0CAFC04F1140002
:104C300000234FF400721549009400F065F9144BFD
:104C40004FF40072134904F13800009400F0DEF9CB
:104C5000114BC4E9173503B030BD00BFFC3800204C
:104C600000E1F505403A0020404000206D4B00086F
:104C70000048004068390020403C002040420020AD
:104C80007D4B000800500040D4390020403E0020F9
:104C90008D4B0008404400200078004038B5264D78
:104CA0000446037C002918BF0D46012B06D1234B77
:104CB000984230D14FF48020FFF770FF2A68236EAE
:104CC000E16D03EB5203A566B3FBF2F36A681004CF
:104CD00042BF23F0070003F0070343EA4003CB6021
:104CE000AB6843F040034B60EB6843F001038B601B
:104CF00042F4967343F001030B604FF0FF330B62F5
:104D0000510505D512F0102211D0B2F1805F10D0FC
:104D100084F8643038BD0A4B984205D0094B98425C
:104D2000CCD14FF08040C7E74FF48010C4E77F2319
:104D3000EEE73F23ECE700BF1C930008FC3800209F
:104D400068390020D43900202DE9F047C66D0546AA
:104D50003768F469210734621AD014F0080118BFCB
:104D60004FF48071E20748BF41F02001A3074FF0E4
:104D7000300348BF41F04001600748BF41F0800167
:104D800083F31188281DFFF7E9FE002383F31188C0
:104D9000E2050AD5302383F311884FF48061281D82
:104DA000FFF7DCFE002383F311884FF030094FF04A
:104DB000000A14F0200838D13B0616D54FF0300910
:104DC00005F1380A200610D589F31188504600F005
:104DD00051F9002836DA0821281DFFF7BFFE27F019
:104DE00080033360002383F31188790614D56206AB
:104DF00012D5302383F31188D5E913239A4208D1C1
:104E00002B6C33B127F040071021281DFFF7A6FEB9
:104E10003760002383F31188E30618D5AA6E13695F
:104E2000ABB15069BDE8F047184789F31188736A40
:104E3000284695F86410194000F0DCFB8AF31188CD
:104E4000F469B6E7B06288F31188F469BAE7BDE89F
:104E5000F0870000F8B51546826804460B46AA4262
:104E600000D28568A1692669761AB5420BD2184628
:104E70002A46FCF74FFFA3692B44A3612846A36889
:104E80005B1BA360F8BD0CD9AF1B18463246FCF77C
:104E900041FF3A46E1683044FCF73CFFE3683B449D
:104EA000EBE718462A46FCF735FFE368E5E7000024
:104EB00083689342F7B50446154600D28568D4E965
:104EC0000460361AB5420BD22A46FCF723FF636909
:104ED0002B4463612846A3685B1BA36003B0F0BD4D
:104EE0000DD93246AF1B0191FCF714FF01993A46E8
:104EF000E0683144FCF70EFFE3683B44E9E72A46EB
:104F0000FCF708FFE368E4E710B50A440024C36136
:104F1000029B8460C16002610362C0E90000C0E9D5
:104F2000051110BD08B5D0E90532934201D1826860
:104F300082B98268013282605A1C42611970002174
:104F4000D0E904329A4224BFC368436101F02CF9CE
:104F5000002008BD4FF0FF30FBE7000070B53023A4
:104F600004460E4683F31188A568A5B1A368A2691B
:104F7000013BA360531CA36115782269934224BFAF
:104F8000E368A361E3690BB120469847002383F3EC
:104F90001188284607E03146204601F0F5F8002840
:104FA000E2DA85F3118870BD2DE9F74F04460E460D
:104FB00017469846D0F81C904FF0300A8AF31188B3
:104FC0004FF0000B154665B12A4631462046FFF7E3
:104FD00041FF034660B94146204601F0D5F800285C
:104FE000F1D0002383F31188781B03B0BDE8F08F64
:104FF000B9F1000F03D001902046C847019B8BF305
:105000001188ED1A1E448AF31188DCE7C160C36180
:10501000009B82600362C0E905111144C0E90000F1
:1050200001617047F8B504460D461646302383F3F8
:105030001188A768A7B1A368013BA36063695A1CE4
:1050400062611D70D4E904329A4224BFE36863614F
:10505000E3690BB120469847002080F3118807E0F0
:105060003146204601F090F80028E2DA87F31188F3
:10507000F8BD0000D0E9052310B59A4201D182683D
:105080007AB982680021013282605A1C82611C78E0
:1050900003699A4224BFC368836101F085F8204602
:1050A00010BD4FF0FF30FBE72DE9F74F04460E46E9
:1050B00017469846D0F81C904FF0300A8AF31188B2
:1050C0004FF0000B154665B12A4631462046FFF7E2
:1050D000EFFE034660B94146204601F055F800282E
:1050E000F1D0002383F31188781B03B0BDE8F08F63
:1050F000B9F1000F03D001902046C847019B8BF304
:105100001188ED1A1E448AF31188DCE70379052B18
:1051100005BF836A002001204B6004BF4FF4007379
:105120000B60704770B55D1E866A04460D44B5423B
:1051300005D9436B43F080034363012070BD06250E
:105140000571FFF7AFFC05232371F7E770B55D1E0E
:10515000866A04460D44B54205D9436B43F080038B
:105160004363012070BD07250571FFF7C1FC0523CE
:105170002371F7E738B505790446052D05D10823D5
:105180000371FFF7DBFC257138BD0120FCE700004F
:105190000323F0B5037185B00446FFF775FA0022CA
:1051A00020461146FFF7BAFA4FF4D57203AB082137
:1051B0002046FFF7D5FA0246B8B901232363039BC3
:1051C000C3F30323012B09D103AB37212046FFF79B
:1051D000C7FA18B9A44B039A1340ABB12046012576
:1051E000FFF784FA0223237137E103AB0022372152
:1051F0002046FFF7B5FA28B99B4A039B1A40002ABC
:1052000000F0A78002232363236B03F00F03022B1C
:1052100040F0A9806425954E42F2107000F090FF96
:1052200003AB324601212046FFF784FA0028D5D18E
:10523000039B002B80F293805A0003D5236B43F02D
:1052400010032363002204F1080302212046FFF724
:10525000E5FA02460028C1D104F1380303212046B3
:10526000FFF77EFA0028B9D104F11805A26B0921D5
:1052700020462B46FFF7D2FA0028AFD102ABA26B33
:1052800007212046FFF76CFA06460028A6D1236BBB
:1052900003F00F03022B40F08F807E227F212846EF
:1052A00003F0A2F9012840F28780E76B42F2107008
:1052B00000F046FF08234FF400723946204600965E
:1052C000FFF7C8FA002889D1384603F0DBF9236BD1
:1052D000A06203F00F03022B72D103AB644A0621D4
:1052E0002046FFF73DFA002871D15F49039B194022
:1052F000B1FA81F149092046FFF7D8F902AB4FF422
:10530000007210212046FFF72BFA054600287FF493
:1053100065AF554E029B33427FF460AF236B13F0B1
:105320000E0F03F00F0273D0022A7FF457AFE36A27
:105330001978012900F09480022900F09380002957
:1053400000F089804B4F2046FFF7D6F903AB3A4671
:1053500076E0114620462263FFF7E0F954E7013D6D
:105360007FF45AAF3AE7444D6426444A3E4F012B3E
:1053700018BF154603AB002237212046FFF7F0F98E
:1053800000287FF42BAF039B3B427FF427AF03AB96
:105390002A4629212046FFF7CDF900287FF41EAFC9
:1053A000039B002BFFF648AF013E3FF417AF42F2DC
:1053B000107000F0C5FEDDE7284603F037F986E7F8
:1053C0007E227F212846E66B03F00EF908B9002102
:1053D00091E7002340223146204600930623FFF741
:1053E00039FA0028F3D1B3895BBA9B07EFD5244B78
:1053F00040223146204600930623FFF72BFA00286F
:10540000E5D1317C01F00F010F3918BF012172E79E
:10541000E36A1978F9B101297FF4E0AE2046FFF77D
:105420006BF903ABA26B37212046FFF799F90028EF
:105430007FF4D4AE039B33427FF4D0AE03AB0222A1
:1054400006212046FFF78CF900287FF4C7AE039BA6
:1054500033427FF4C3AE05232371284605B0F0BD67
:10546000084F70E7084F6EE708E0FFFD0080FFC0BF
:105470000001B9030000B7030080FF500000108056
:10548000F1FFFF800001B7030002B70337B5044600
:105490000C4D01ABA26B0D212046FFF761F978B9E5
:1054A000019B2B420BD1C3F34323042B08D0053BB4
:1054B000022B04D84FF47A7000F042FEE9E7012095
:1054C00003B030BD08E0FFFD70B53023054683F31F
:1054D000118803790024022B03D184F3118820461C
:1054E00070BD0423037184F311880226FFF7CEFFF9
:1054F00004462846FFF7FAF82E71F0E7FFF75CB88C
:10550000044B03600123037100234363C0E90A33A2
:10551000704700BF3493000810B53023044683F36E
:105520001188C162FFF762F802230020237180F323
:10553000118810BD10B53023044683F31188FFF79E
:105540007FF800230122E362227183F3118810BDEA
:10555000026843681143016003B1184770470000B7
:105560001430FFF721BD00004FF0FF331430FFF778
:105570001BBD00003830FFF797BD00004FF0FF3330
:105580003830FFF791BD00001430FFF7E7BC000092
:105590004FF0FF311430FFF7E1BC00003830FFF767
:1055A00041BD00004FF0FF323830FFF73BBD000037
:1055B000012914BF6FF0130000207047FFF7FEBAF7
:1055C000044B036000234360C0E9023301230374EA
:1055D000704700BF5893000810B53023044683F38A
:1055E0001188FFF75BFB02230020237480F31188EE
:1055F00010BD000038B5C36904460D461BB904212F
:105600000844FFF7A5FF294604F11400FFF78AFCC0
:10561000002806DA201D4FF40061BDE83840FFF78E
:1056200097BF38BD026843681143016003B1184752
:105630007047000013B5406B00F58054D4F8A438CF
:105640001A681178042914D1017C022911D1197921
:10565000012312898B4013420BD101A94C3002F077
:10566000F1FED4F8A4480246019B2179206800F09D
:10567000DFF902B010BD0000143002F073BE00006C
:105680004FF0FF33143002F06DBE00004C3002F0DA
:1056900045BF00004FF0FF334C3002F03FBF000029
:1056A000143002F041BE00004FF0FF31143002F020
:1056B0003BBE00004C3002F011BF00004FF0FF3243
:1056C0004C3002F00BBF00000020704710B500F511
:1056D0008054D4F8A4381A681178042917D1017CB1
:1056E000022914D15979012352898B4013420ED1DA
:1056F000143002F0D3FD024648B1D4F8A4484FF468
:10570000407361792068BDE8104000F07FB910BD9A
:10571000406BFFF7DBBF0000704700007FB5124B06
:1057200001250426044603600023057400F1840269
:1057300043602946C0E902330C4B029014300193B8
:105740004FF44073009602F085FD094B04F6944235
:10575000294604F14C000294CDE900634FF44073F4
:1057600002F04CFE04B070BD809300081157000891
:10577000355600080A68302383F311880B790B3300
:1057800042F823004B79133342F823008B7913B18D
:105790000B3342F8230000F58053C3F8A41802230A
:1057A0000374002080F311887047000038B5037F30
:1057B000044613B190F85430ABB90125201D0221E5
:1057C000FFF730FF04F114006FF00101257700F0BE
:1057D000F7FC04F14C0084F854506FF00101BDE86F
:1057E000384000F0EDBC38BD10B50121044604304E
:1057F000FFF718FF0023237784F8543010BD000012
:1058000038B504460025143002F03CFD04F14C008C
:10581000257702F00BFE201D84F854500121FFF77C
:1058200001FF2046BDE83840FFF750BF90F88030B8
:1058300003F06003202B06D190F881200023212A59
:1058400003D81F2A06D800207047222AFBD1C0E9BE
:105850001D3303E0034A426707228267C3670120C2
:10586000704700BF4422002037B500F58055D5F8B9
:10587000A4381A68117804291AD1017C022917D199
:105880001979012312898B40134211D100F14C0484
:10589000204602F08BFE58B101A9204602F0D2FD4D
:1058A000D5F8A4480246019B2179206800F0C0F891
:1058B00003B030BD01F10B03F0B550F8236085B0A3
:1058C00004460D46FEB1302383F3118804EB8507AF
:1058D000301D0821FFF7A6FEFB6806F14C005B694E
:1058E0001B681BB1019002F0BBFD019803A902F0F7
:1058F000A9FD024648B1039B2946204600F098F8CE
:10590000002383F3118805B0F0BDFB685A69126863
:10591000002AF5D01B8A013B1340F1D104F180022B
:10592000EAE70000133138B550F82140ECB13023DC
:1059300083F3118804F58053D3F8A42813685279AF
:1059400003EB8203DB689B695D6845B10421601845
:10595000FFF768FE294604F1140002F0A9FC204676
:10596000FFF7B4FE002383F3118838BD70470000B1
:1059700001F0B8BC01234022002110B5044600F814
:10598000303BFCF7EDF90023C4E9013310BD000002
:1059900010B53023044683F311882422416000218E
:1059A0000C30FCF7DDF9204601F0BEFC022300209C
:1059B000237080F3118810BD70B500EB810305469C
:1059C00050690E461446DA6018B110220021FCF727
:1059D000C7F9A06918B110220021FCF7C1F93146BE
:1059E0002846BDE8704001F0A5BD00008368202274
:1059F000002103F0011310B5044683601030FCF75A
:105A0000AFF92046BDE8104001F020BEF0B40125FA
:105A100000EB810447898D40E4683D43A4694581DA
:105A200023600023A2606360F0BC01F03DBE000073
:105A3000F0B4012500EB810407898D40E4683D4303
:105A40006469058123600023A2606360F0BC01F0FB
:105A5000B3BE000070B50223002504462422037063
:105A60002946C0F888500C3040F8045CFCF778F9FF
:105A7000204684F8705001F0F1FC63681B6823B184
:105A800029462046BDE87040184770BD0378052BB5
:105A900010B504460AD080F88C30052303704368A3
:105AA0001B680BB1042198470023A36010BD0000C0
:105AB0000178052906D190F88C20436802701B6894
:105AC00003B118477047000070B590F87030044675
:105AD00013B1002380F8703004F18002204601F0F9
:105AE000D9FD63689B68B3B994F8803013F0600502
:105AF00035D00021204602F0CBF80021204602F0EC
:105B0000BBF863681B6813B106212046984706233B
:105B100084F8703070BD204698470028E4D0B4F86F
:105B20008630A26F9A4288BFA36794F98030A56F30
:105B3000002B4FF0300380F20381002D00F0F28043
:105B4000092284F8702083F3118800212046D4E9CB
:105B50001D23FFF76DFF002383F31188DAE794F824
:105B6000812003F07F0343EA022340F20232934292
:105B700000F0C58021D8B3F5807F48D00DD8012B27
:105B80003FD0022B00F09380002BB2D104F18802A9
:105B900062670222A267E367C1E7B3F5817F00F085
:105BA0009B80B3F5407FA4D194F88230012BA0D123
:105BB000B4F8883043F0020332E0B3F5006F4DD003
:105BC00017D8B3F5A06F31D0A3F5C063012B90D8DF
:105BD0006368204694F882205E6894F88310B4F8D5
:105BE0008430B047002884D0436863670368A367A4
:105BF0001AE0B3F5106F36D040F6024293427FF4BC
:105C000078AF5C4B63670223A3670023C3E794F874
:105C10008230012B7FF46DAFB4F8883023F002039B
:105C2000A4F88830C4E91D55E56778E7B4F88030FA
:105C3000B3F5A06F0ED194F88230204684F88A30F4
:105C400001F06AFC63681B6813B101212046984784
:105C5000032323700023C4E91D339CE704F18B0365
:105C600063670123C3E72378042B10D1302383F328
:105C700011882046FFF7BAFE85F311880321636877
:105C800084F88B5021701B680BB12046984794F81C
:105C90008230002BDED084F88B30042323706368BD
:105CA0001B68002BD6D0022120469847D2E794F8F3
:105CB000843020461D0603F00F010AD501F0DCFCFC
:105CC000012804D002287FF414AF2B4B9AE72B4B0A
:105CD00098E701F0C3FCF3E794F88230002B7FF4DF
:105CE00008AF94F8843013F00F01B3D01A062046A1
:105CF00002D501F0E5FFADE701F0D6FFAAE794F881
:105D00008230002B7FF4F5AE94F8843013F00F014D
:105D1000A0D01B06204602D501F0BAFF9AE701F099
:105D2000ABFF97E7142284F8702083F311882B4689
:105D30002A4629462046FFF769FE85F31188E9E6E1
:105D40005DB1152284F8702083F31188002120466C
:105D5000D4E91D23FFF75AFEFDE60B2284F87020DC
:105D600083F311882B462A4629462046FFF760FE1A
:105D7000E3E700BFB0930008A8930008AC930008C5
:105D800038B590F870300446002B3ED0063BDAB2AE
:105D90000F2A34D80F2B32D8DFE803F0373131081F
:105DA000223231313131313131313737856FB0F80D
:105DB00086309D4214D2C3681B8AB5FBF3F203FB05
:105DC00012556DB9302383F311882B462A46294694
:105DD000FFF72EFE85F311880A2384F870300EE059
:105DE000142384F87030302383F311880023204675
:105DF0001A461946FFF70AFE002383F3118838BDBF
:105E0000C36F03B198470023E7E70021204601F064
:105E10003FFF0021204601F02FFF63681B6813B18C
:105E20000621204698470623D7E7000010B590F8D2
:105E300070300446142B29D017D8062B05D001D872
:105E40001BB110BD093B022BFBD80021204601F0FD
:105E50001FFF0021204601F00FFF63681B6813B18C
:105E6000062120469847062319E0152BE9D10B237C
:105E700080F87030302383F3118800231A461946C6
:105E8000FFF7D6FD002383F31188DAE7C3689B6927
:105E90005B68002BD5D1C36F03B19847002384F80A
:105EA0007030CEE70023826880F8243083691B6855
:105EB00099689142FBD25A68036042601060586052
:105EC000704700000023826880F8243083691B68D3
:105ED00099689142FBD85A6803604260106058602C
:105EE0007047000008B50846302383F3118891F805
:105EF0002430032B05D0042B0DD02BB983F311884C
:105F000008BD8B6A00221A604FF0FF338362FFF7EF
:105F1000C9FF0023F2E7D1E9003213605A60F3E7CA
:105F2000034610B51B68984203D09C688A68944267
:105F3000F8D25A680B604A601160596010BD0000C9
:105F4000FFF7B0BF064BD96881F8240018680268D3
:105F500053601A600122D86080F82420FAF752BA00
:105F6000404600200C4B30B5DD684B1C87B0044622
:105F70000FD02B46094A684600F0B6F92046FFF7D5
:105F8000E1FF009B13B1684600F0B8F9A86A07B0BA
:105F900030BDFFF7D7FFF9E740460020E55E000877
:105FA000044B1A68DB6890689B68984294BF002095
:105FB0000120704740460020094B10B51C68D86886
:105FC000226853601A600122DC6084F82420FFF705
:105FD00079FF01462046BDE81040FAF713BA00BF2A
:105FE00040460020044B1A68DB6892689B689A421E
:105FF00001D9FFF7E1BF70474046002038B50123C3
:10600000084C00252370656002F06AFB02F090FBEB
:106010000549064802F066FC0223237085F31188C7
:1060200038BD00BFE8480020B89300084046002073
:1060300000F09AB9EFF3118020B9EFF30583302215
:1060400082F311887047000010B530B9EFF3058472
:10605000C4F3080414B180F3118810BDFFF7C2FF28
:1060600084F31188F9E70000034A516853685B1A0A
:106070009842FBD8704700BF001000E08B604B6374
:106080000023CA6100F128020B6302230A618B849A
:106090000123886181F8263001F11003C26A4A6148
:1060A0001360C36201F12C030846CB627047000005
:1060B000D0E90131026841F8183CA1F19C0338395C
:1060C000CB60036941F8243C436941F8203C034B11
:1060D00041F8043CC3680248FFF7D0BF1D04000824
:1060E0004046002008B5FFF7E3FFBDE80840FFF792
:1060F00027BF000038B50E4BDC6804F12C05A06208
:10610000E06AA8420FD194F826303BB994F82530C4
:106110009B0702BFD4E9043213605A600F20BDE828
:106120003840FFF70FBF0368E362FFF709FFE7E7B7
:1061300040460020302383F31188FFF7DBBF0000C7
:1061400008B50146302383F311880820FFF70AFFC2
:10615000002383F3118808BD054BDB6821B1036080
:1061600098620320FFF7FEBE4FF0FF30704700BF7C
:106170004046002003682BB1002202601846996255
:10618000FFF7DEBE70470000064BDB6839B142689E
:1061900018605A60136043600420FFF7E3BE4FF0BD
:1061A000FF307047404600200368984206D01A68C6
:1061B0000260506018469962FFF7C2BE7047000047
:1061C00038B504460D462068844200D138BD0368C6
:1061D00023605C608562FFF7B3FEF4E7036810B5E7
:1061E0009C68A2420CD85C688A600B604C6021609D
:1061F000596099688A1A9A604FF0FF33836010BD26
:10620000121B1B68ECE700000A2938BF0A2170B591
:1062100004460D460A26601902F05CFA02F044FAC0
:10622000041BA54203D8751C04462E46F3E70A2E2C
:1062300004D90120BDE8704002F01CBC70BD000014
:10624000F8B5144B0D460A2A4FF00A07D96103F13D
:106250001001826038BF0A2241601969144601604A
:1062600048601861A81802F025FA02F01DFA431BD5
:106270000646A34206D37C1C28192746354602F061
:1062800029FAF2E70A2F04D90120BDE8F84002F00C
:10629000F1BBF8BD40460020F8B506460D4602F0B9
:1062A00003FA0F4A134653F8107F9F4206D12A463D
:1062B00001463046BDE8F840FFF7C2BFD169BB6870
:1062C000441A2C1928BF2C46A34202D92946FFF7AD
:1062D0009BFF224631460348BDE8F840FFF77EBFEA
:1062E0004046002050460020C0E90323002310B49C
:1062F0005DF8044B4361FFF7CFBF000010B5194CA8
:10630000236998420DD08168D0E9003213605A6049
:106310009A680A449A60002303604FF0FF33A36138
:1063200010BD0268234643F8102F5360002202601C
:1063300022699A4203D1BDE8104002F0C5B99368C2
:1063400081680B44936002F0AFF92269E1699268B9
:10635000441AA242E4D91144BDE81040091AFFF7DB
:1063600053BF00BF404600202DE9F047DFF8BC8056
:1063700008F110072C4ED8F8105002F095F9D8F813
:106380001C40AA68031B9A423ED814444FF00009EF
:10639000D5E90032C8F81C4013605A60C5F8009077
:1063A000D8F81030B34201D102F08EF989F3118888
:1063B000D5E9033128469847302383F311886B6968
:1063C000002BD8D002F070F96A69A0EB040982466C
:1063D0004A450DD2022002F04DFB0022D8F81030C1
:1063E000B34208D151462846BDE8F047FFF728BF21
:1063F000121A2244F2E712EB09092946384638BF3F
:106400004A46FFF7EBFEB5E7D8F81030B34208D0A4
:106410001444C8F81C00211AA960BDE8F047FFF732
:10642000F3BEBDE8F08700BF504600204046002084
:1064300010B560B9074804790368053C9B6818BF2C
:106440000124984708B144F00404204610BD0124FB
:10645000FBE700BFA4360020FFF7EABF2DE9F047B5
:10646000884617469A460446B0B90D4E3579052D33
:1064700005D003240DE0013D15F0FF050ED0326874
:10648000534639463046D2F814904246C847002851
:10649000F1D12046BDE8F0870424FAE70124F8E7AB
:1064A000A43600202DE9F047884617469A46044650
:1064B000B0B90D4E3579052D05D003240DE0013D11
:1064C00015F0FF050ED03268534639463046D2F8F3
:1064D00018904246C8470028F1D12046BDE8F08711
:1064E0000424FAE70124F8E7A436002037B50C4667
:1064F000154670B951B101290BD1074869460368A7
:106500001B6A984710B9019B04462B60204603B0D4
:1065100030BD0424FAE700BFA436002000207047F5
:10652000FEE70000704700004FF0FF3070470000AA
:106530004B6843608B688360CB68C3600B694361C1
:106540004B6903628B6943620B680360704700000C
:1065500008B53C4B40F2FF713B48D3F888200A4312
:10656000C3F88820D3F8882022F4FF6222F00702C3
:10657000C3F88820D3F88820D3F8E0200A43C3F872
:10658000E020D3F808210A43C3F808212F4AD3F8A2
:1065900008311146FFF7CCFF00F5806002F11C01C5
:1065A000FFF7C6FF00F5806002F13801FFF7C0FF7A
:1065B00000F5806002F15401FFF7BAFF00F580603A
:1065C00002F17001FFF7B4FF00F5806002F18C0169
:1065D000FFF7AEFF00F5806002F1A801FFF7A8FF0A
:1065E00000F5806002F1C401FFF7A2FF00F58060B2
:1065F00002F1E001FFF79CFF00F5806002F1FC0171
:10660000FFF796FF02F58C7100F58060FFF790FFB1
:1066100001F0EAFB0E4BD3F8902242F00102C3F8DE
:106620009022D3F8942242F00102C3F8942205226A
:10663000C3F898204FF06052C3F89C20054AC3F875
:10664000A02008BD0044025800000258CC93000866
:1066500000ED00E01F00080308B501F0E7FDFFF7BB
:10666000CDFC104BD3F8DC2042F04002C3F8DC2014
:10667000D3F8042122F04002C3F80421D3F80431F6
:10668000094B1A6842F008021A601A6842F00402C4
:106690001A6000F03DFD00F035FBBDE8084000F059
:1066A000B5B800BF004402580018024801207047E6
:1066B000002070477047000002290CD0032904D045
:1066C0000129074818BF00207047032A05D805484C
:1066D00000EBC2007047044870470020704700BFBD
:1066E000CC950008542200208095000870B59AB01F
:1066F00005460846144601A900F0C2F801A8FBF7B8
:1067000027FB431C0022C6B25B001046C5E90034DB
:1067100023700323023404F8013C01ABD1B20234EC
:106720008E4201D81AB070BD13F8011B013204F873
:10673000010C04F8021CF1E708B5302383F311883B
:106740000348FFF791F8002383F3118808BD00BFC9
:10675000F048002090F8803003F01F02012A07D192
:1067600090F881200B2A03D10023C0E91D3315E0E6
:1067700003F06003202B08D1B0F884302BB990F8D7
:106780008120212A03D81F2A04D8FFF74FB8222AD4
:10679000EBD0FAE7034A426707228267C36701200A
:1067A000704700BF4B22002007B5052917D8DFE846
:1067B00001F0191603191920302383F31188104AA8
:1067C00001210190FFF7F8F8019802210D4AFFF727
:1067D000F3F80D48FFF714F8002383F3118803B092
:1067E0005DF804FB302383F311880748FEF7DEFFD2
:1067F000F2E7302383F311880348FEF7F5FFEBE758
:106800002095000844950008F048002038B50C4D4C
:106810000C4C2A460C4904F10800FFF767FF05F10C
:10682000CA0204F110000949FFF760FF05F5CA72BA
:1068300004F118000649BDE83840FFF757BF00BF14
:10684000C861002054220020009500080A95000825
:106850001595000870B5044608460D46FBF778FA12
:10686000C6B22046013403780BB9184670BD3246D3
:106870002946FBF759FA0028F3D10120F6E700007A
:106880002DE9F84F05460C46FBF762FA2C49C6B2D3
:106890002846FFF7DFFF08B10236F6B2294928463D
:1068A000FFF7D8FF08B11036F6B2632E0DD8DFF827
:1068B0009080DFF89090244FDFF894A0DFF894B038
:1068C0002E7846B92670BDE8F88F29462046BDE8E7
:1068D000F84F02F04DBA252E2ED107224146284608
:1068E000FBF722FA70B9DBF800300735093444F8B9
:1068F000093CDBF8043044F8053C9BF8083004F808
:10690000013CDDE7082249462846FBF70DFA98B915
:10691000A21C0E4B197802320909C95D02F8041C49
:1069200013F8011B01F00F015345C95D02F8031C68
:10693000F0D118340835C3E7013504F8016BBFE71F
:10694000EC95000815950008FE95000800E8F11F79
:106950000CE8F11FF4950008BFF34F8F044B1A6940
:106960005107FCD1D3F810215207F8D1704700BF6E
:106970000020005208B50D4B1B78ABB9FFF7ECFFB8
:106980000B4BDA68D10704D50A4A5A6002F1883203
:106990005A60D3F80C21D20706D5064AC3F8042161
:1069A00002F18832C3F8042108BD00BF266400202C
:1069B000002000522301674508B5114B1B78F3B93D
:1069C000104B1A69510703D5DA6842F04002DA60C9
:1069D000D3F81021520705D5D3F80C2142F040021C
:1069E000C3F80C21FFF7B8FF064BDA6842F001024A
:1069F000DA60D3F80C2142F00102C3F80C2108BD83
:106A000026640020002000520F289ABF00F5806005
:106A100040040020704700004FF400307047000031
:106A2000102070470F2808B50BD8FFF7EDFF00F5D1
:106A300000330268013204D104308342F9D10120CD
:106A400008BD0020FCE700000F2838B505463FD8F8
:106A5000FFF782FF1F4CFFF78DFF4FF0FF33072832
:106A60006361C4F814311DD82361FFF775FF030279
:106A700043F02403E360E36843F08003E3602369A9
:106A80005A07FCD42846FFF767FFFFF7BDFF4FF416
:106A9000003100F097FA2846FFF78EFFBDE8384036
:106AA000FFF7C0BFC4F81031FFF756FFA0F108038D
:106AB0001B0243F02403C4F80C31D4F80C3143F02A
:106AC0008003C4F80C31D4F810315B07FBD4D9E74C
:106AD000002038BD002000522DE9F84F05460C4635
:106AE000104645EA0203DE0602D00020BDE8F88F1A
:106AF00020F01F00DFF8BCB0DFF8BCA0FFF73AFFC2
:106B000004EB0008444503D10120FFF755FFEDE7F2
:106B100020222946204602F0AFF810B92035203453
:106B2000F0E72B4605F120021F68791CDDD1043304
:106B30009A42F9D105F178431B481C4EB3F5801FEA
:106B40001B4B38BF184603F1F80332BFD946D14674
:106B50001E46FFF701FF0760A5EB040C336804F144
:106B60001C0143F002033360231FD9F8007017F0B3
:106B70000507FAD153F8042F8B424CF80320F4D1C7
:106B8000BFF34F8FFFF7E8FE4FF0FF33202221467F
:106B900003602846336823F00203336002F06CF888
:106BA0000028BBD03846B0E7142100520C20005218
:106BB00014200052102000521021005210B5084C31
:106BC000237828B11BB9FFF7D5FE0123237010BD30
:106BD000002BFCD02070BDE81040FFF7EDBE00BFD9
:106BE000266400202DE9F04F0D4685B0814658B14E
:106BF00011F00D0614BF2022082211F008030193A2
:106C000004D0431E034269D0002435E0002E37D063
:106C100009F11F0121F01F094FF00108314F05F064
:106C20000403DFF8CCA005EA080BBBF1000F32D05B
:106C30007869C0072FD408F101080C37B8F1060FA6
:106C4000F3D19EB9284D4946A819019201F092FD51
:106C50000446002839D12036019AA02EF3D14946A6
:106C600001F088FD044600282FD1019A49461F48AB
:106C700001F080FD044660BB204605B0BDE8F08F02
:106C80000029C9D101462846029201F073FD04464D
:106C9000D8B9029AC0E713B178694107CBD5AC07E0
:106CA00002D578698007C6D5019911B178690107C5
:106CB000C1D549460AEB4810CDE9022301F05AFD3F
:106CC0000446DDE902230028B5D04A4600212046CB
:106CD00001E04A460021FBF743F8CDE70246002ECB
:106CE00096D199E710960008686400202864002077
:106CF000486400200021FFF775BF00000121FFF765
:106D000071BF000070B5144D0124144E40F2FF32E3
:106D100000210120FBF724F806EB441001342A6916
:106D200055F80C1F01F012FD062CF5D137254FF454
:106D3000C0542046FFF7E2FF014628B1224608482A
:106D4000BDE8704001F002BDC4EBC404013D4FEA50
:106D5000D404EED170BD00BF109600084864002036
:106D6000286400200421FFF73DBF00004843FFF7DF
:106D7000C1BF000008B101F06FBD7047B0F5805F82
:106D800010B5044607D8FFF7EDFF28B92046BDE847
:106D90001040FFF7AFBF002010BD0000FFF7EABFB3
:106DA00008B501F06FFE034AD2E90032C01842EB89
:106DB000010108BD08650020434BD3E900232DE9FC
:106DC000F34113437CD0FFF7EBFF404A0023002739
:106DD000F9F732FB06460D463D4A0023F9F72CFB36
:106DE0000023144630462946394AF9F725FB4FF46B
:106DF00061613C23ADF80170B4FBF1F5B4FBF3F62F
:106E000001FB154103FB16464624B1FBF3F1314B60
:106E1000F6B28DF8004098423CD84FF0640C4FF425
:106E2000C87EA30704F26C7225D1B2FBFCF30CFB05
:106E3000132313BBB2FBFEF30EFB1322B2FA82F351
:106E40005B0903F26D18621C8045D2B217D90FB1ED
:106E50008DF800400022204C4FF00C0C17460CFB24
:106E60000343D4B2013213F804C084450CD8A0EB1C
:106E70000C000127F5E70023E3E70123E1E7A0EB9E
:106E8000080014460127CCE70FB18DF80140431CE0
:106E90008DF802309DF80100431C9DF80000503829
:106EA000400640EA43509DF8023040EA034040EA81
:106EB000560040EAC52040EA411002B0BDE8F0812A
:106EC0004FF40410F9E700BF0865002040420F00AE
:106ED0008051010090230B00589600080244074B94
:106EE000D2B210B5904200D110BD441C00B253F88C
:106EF000200041F8040BE0B2F4E700BF5040005816
:106F00000E4B30B51C6F240405D41C6F1C671C6F1E
:106F100044F400441C670A4C02442368D2B243F490
:106F200080732360074B904200D130BD441C51F860
:106F3000045B00B243F82050E0B2F4E7004402588A
:106F4000004802585040005807B5012201A900200E
:106F5000FFF7C4FF019803B05DF804FB13B50446C6
:106F6000FFF7F2FFA04205D0012201A90020019401
:106F7000FFF7C6FF02B010BD10B56424013C4FF40A
:106F80007A70FFF7DDF814F0FF04F7D10C4B4FF4E3
:106F9000801214249A61A3F580634FF08052A3F508
:106FA0004063C3F8182C4FF400529A61013C4FF42F
:106FB0007A70FFF7C5F814F0FF04F7D110BD00BFD9
:106FC000001802580144BFF34F8F064B884204D388
:106FD000BFF34F8FBFF36F8F7047C3F85C02203051
:106FE000F4E700BF00ED00E00144BFF34F8F064B14
:106FF000884204D3BFF34F8FBFF36F8F7047C3F83E
:1070000070022030F4E700BF00ED00E070B50546E7
:1070100016460C4601201021FFF7A8FE2860467393
:107020003CB1204636B1FFF79DFE2B68186000B1D9
:107030009C6070BDFFF762FEF7E7000070B50E467A
:107040001546044600B30B6843608368934210D230
:1070500013B10068FFF78EFE637B28462BB1FFF764
:1070600081FE206020B9A06070BDFFF747FEF8E701
:10707000A560206805F11F01306021F01F01FFF7B6
:10708000A1FF01202073EFE70120EDE710B50446D2
:1070900040B10068884205D1606808B1FAF73AFE4D
:1070A0000023237310BD000070B50E46154604463C
:1070B00020B383689A4210D913B10068FFF75AFED3
:1070C000637B28462BB1FFF74DFE206020B9A060FE
:1070D00070BDFFF713FEF8E7A560316819B12A46C5
:1070E0002068FAF717FE206805F11F01306021F0D3
:1070F0001F01FFF779FF01202073E9E70120E7E78F
:1071000020B103688B4204BF002303737047000063
:10711000034B1A681AB9034AD2F8D0241A60704790
:10712000106500200040025808B5FFF7F1FF024B40
:107130001868C0F3806008BD1065002070B5BFF30B
:107140004F8FBFF36F8F1A4A0021C2F85012BFF35E
:107150004F8FBFF36F8F536943F400335361BFF315
:107160004F8FBFF36F8FC2F88410BFF34F8FD2F8E9
:10717000803043F6E074C3F3C900C3F34E335B01C0
:1071800003EA0406014646EA81750139C2F86052F5
:10719000F9D2203B13F1200FF2D1BFF34F8F536987
:1071A00043F480335361BFF34F8FBFF36F8F70BDD4
:1071B00000ED00E0FEE70000214B2248224A70B5B6
:1071C000904237D3214BC11EDA1C121A22F003025F
:1071D0008B4238BF00220021FAF7C2FD1C4A00236F
:1071E000C2F88430BFF34F8FD2F8803043F6E0749A
:1071F000C3F3C900C3F34E335B0103EA040601463F
:1072000046EA81750139C2F86C52F9D2203B13F17C
:10721000200FF2D1BFF34F8FBFF36F8FBFF34F8FAC
:10722000BFF36F8F0023C2F85032BFF34F8FBFF30D
:107230006F8F70BD53F8041B40F8041BC0E700BFFC
:10724000C0970008206700202067002020670020EA
:1072500000ED00E0074BD3F8D81021EA0001C3F895
:10726000D810D3F8002122EA0002C3F80021D3F895
:10727000003170470044025870B5D0E92443002221
:107280004FF0FF359E6804EB42135101D3F800091B
:10729000002805DAD3F8000940F08040C3F800095F
:1072A000D3F8000B002805DAD3F8000B40F080403B
:1072B000C3F8000B013263189642C3F80859C3F8AB
:1072C000085BE0D24FF00113C4F81C3870BD000019
:1072D000890141F02001016103699B06FCD4122061
:1072E000FEF7C2BE10B50A4C2046FEF743FB094B21
:1072F000C4F89030084BC4F89430084C2046FEF790
:1073000039FB074BC4F89030064BC4F8943010BDDD
:10731000146500200000084094960008B065002025
:1073200000000440A096000870B503780546012BC4
:107330005CD1434BD0F89040984258D1414B0E213C
:107340006520D3F8D82042F00062C3F8D820D3F8E3
:10735000002142F00062C3F80021D3F80021D3F8E5
:10736000802042F00062C3F88020D3F8802022F011
:107370000062C3F88020D3F8803000F041FF324B28
:10738000E360324BC4F800380023D5F89060C4F8AD
:10739000003EC02323604FF40413A3633369002B22
:1073A000FCDA01230C203361FEF75EFE3369DB0754
:1073B000FCD41220FEF758FE3369002BFCDA0026BD
:1073C0002846A660FFF758FF6B68C4F81068DB68B2
:1073D000C4F81468C4F81C6883BB1D4BA3614FF04C
:1073E000FF336361A36843F00103A36070BD194BD1
:1073F0009842C9D1134B4FF08060D3F8D82042F0A7
:107400000072C3F8D820D3F8002142F00072C3F80C
:107410000021D3F80021D3F8802042F00072C3F895
:107420008020D3F8802022F00072C3F88020D3F8A7
:107430008030FFF70FFF0E214D209EE7064BCDE772
:10744000146500200044025840140040030020024C
:10745000003C30C0B0650020083C30C0F8B5D0F822
:107460009040054600214FF000662046FFF730FFB0
:10747000D5F8941000234FF001128F684FF0FF30C1
:10748000C4F83438C4F81C2804EB431201339F427B
:10749000C2F80069C2F8006BC2F80809C2F8080B0C
:1074A000F2D20B68D5F89020C5F8983063621023AB
:1074B0001361166916F01006FBD11220FEF7D4FDF9
:1074C000D4F8003823F4FE63C4F80038A36943F409
:1074D000402343F01003A3610923C4F81038C4F813
:1074E00014380B4BEB604FF0C043C4F8103B094B12
:1074F000C4F8003BC4F81069C4F80039D5F89830D6
:1075000003F1100243F48013C5F89820A362F8BD7C
:107510007096000840800010D0F8902090F88A10F3
:10752000D2F8003823F4FE6343EA0113C2F80038AE
:10753000704700002DE9F84300EB8103D0F890502C
:107540000C468046DA680FFA81F94801166806F0A1
:107550000306731E022B05EB41134FF0000194BF8D
:10756000B604384EC3F8101B4FF0010104F11003AC
:1075700098BF06F1805601FA03F3916998BF06F5AA
:10758000004600293AD0578A04F15801374349018F
:107590006F50D5F81C180B430021C5F81C382B1868
:1075A0000127C3F81019A7405369611E9BB3138AC2
:1075B000928B9B08012A88BF5343D8F898209818CB
:1075C00042EA034301F140022146C8F898002846E8
:1075D00005EB82025360FFF77BFE08EB8900C3686E
:1075E0001B8A43EA845348341E4364012E51D5F864
:1075F0001C381F43C5F81C78BDE8F88305EB491714
:10760000D7F8001B21F40041C7F8001BD5F81C185F
:1076100021EA0303C0E704F13F030B4A2846214651
:1076200005EB83035A60FFF753FE05EB4910D0F8D2
:10763000003923F40043C0F80039D5F81C3823EA98
:107640000707D7E70080001000040002D0F894205C
:107650001268C0F89820FFF70FBE00005831D0F82C
:10766000903049015B5813F4004004D013F4001F1C
:107670000CBF0220012070474831D0F890304901FA
:107680005B5813F4004004D013F4001F0CBF022019
:107690000120704700EB8101CB68196A0B68136009
:1076A0004B6853607047000000EB810330B5DD6824
:1076B000AA691368D36019B9402B84BF40231360B3
:1076C0006B8A1468D0F890201C4402EB4110013CF6
:1076D00009B2B4FBF3F46343033323F0030343EA37
:1076E000C44343F0C043C0F8103B2B6803F00303CE
:1076F000012B0ED1D2F8083802EB411013F4807F31
:10770000D0F8003B14BF43F0805343F00053C0F85F
:10771000003B02EB4112D2F8003B43F00443C2F8B5
:10772000003B30BD2DE9F041D0F8906005460C4695
:1077300006EB4113D3F8087B3A07C3F8087B08D55A
:10774000D6F814381B0704D500EB8103DB685B68AF
:107750009847FA071FD5D6F81438DB071BD505EB79
:107760008403D968CCB98B69488A5A68B2FBF0F6B1
:1077700000FB16228AB91868DA6890420DD2121AF4
:10778000C3E90024302383F3118821462846FFF7FC
:107790008BFF84F31188BDE8F081012303FA04F222
:1077A0006B8923EA02036B81CB68002BF3D021465F
:1077B0002846BDE8F041184700EB81034A0170B547
:1077C000DD68D0F890306C692668E66056BB1A44D4
:1077D0004FF40020C2F810092A6802F00302012ABF
:1077E0000AB20ED1D3F8080803EB421410F4807FDC
:1077F000D4F8000914BF40F0805040F00050C4F8A5
:10780000000903EB4212D2F8000940F00440C2F82C
:1078100000090122D3F8340802FA01F10143C3F848
:10782000341870BD19B9402E84BF402020602068F4
:107830001A442E8A8419013CB4FBF6F440EAC44091
:1078400040F00050C6E700002DE9F843D0F8906002
:1078500005460C464F0106EB4113D3F8088918F092
:10786000010FC3F808891CD0D6F81038DB0718D5EB
:1078700000EB8103D3F80CC0DCF81430D3F800E03F
:10788000DA68964530D2A2EB0E024FF000091A607A
:10789000C3F80490302383F31188FFF78DFF89F339
:1078A000118818F0800F1DD0D6F834380126A64074
:1078B000334217D005EB84030134D5F89050D3F848
:1078C0000CC0E4B22F44DCF8142005EB0434D2F8E9
:1078D00000E05168714514D3D5F8343823EA060620
:1078E000C5F83468BDE8F883012303FA01F203897F
:1078F00023EA02030381DCF80830002BD1D098473B
:10790000CFE7AEEB0103BCF81000834228BF03466B
:10791000D7F8180980B2B3EB800FE3D89068A0F1D4
:10792000040959F8048FC4F80080A0EB09089844B2
:10793000B8F1040FF5D818440B4490605360C8E7C1
:107940002DE9F84FD0F8905004466E69AB691E409F
:1079500016F480586E6103D0BDE8F84FFEF77AB890
:10796000002E12DAD5F8003E9B0705D0D5F8003E70
:1079700023F00303C5F8003ED5F80438204623F071
:107980000103C5F80438FEF793F8370505D52046FE
:10799000FFF772FC2046FEF779F8B0040CD5D5F855
:1079A000083813F0060FEB6823F470530CBF43F450
:1079B000105343F4A053EB6031071BD56368DB68B9
:1079C0001BB9AB6923F00803AB612378052B0CD1FD
:1079D000D5F8003E9A0705D0D5F8003E23F0030302
:1079E000C5F8003E2046FEF763F86368DB680BB11C
:1079F00020469847F30200F1BA80B70226D5D4F8A2
:107A0000909000274FF0010A09EB4712D2F8003B93
:107A100003F44023B3F5802F11D1D2F8003B002BA3
:107A20000DDA62890AFA07F322EA0303638104EBA1
:107A30008703DB68DB6813B1394620469847013776
:107A4000D4F89430FFB29B689F42DDD9F00619D577
:107A5000D4F89000026AC2F30A1702F00F0302F48E
:107A6000F012B2F5802F00F0CA80B2F5402F09D194
:107A700004EB8303002200F58050DB681B6A974209
:107A800040F0B0803003D5F8185835D5E90303D558
:107A900000212046FFF746FEAA0303D50121204618
:107AA000FFF740FE6B0303D502212046FFF73AFEA5
:107AB0002F0303D503212046FFF734FEE80203D548
:107AC00004212046FFF72EFEA90203D505212046FA
:107AD000FFF728FE6A0203D506212046FFF722FEA3
:107AE0002B0203D507212046FFF71CFEEF0103D52B
:107AF00008212046FFF716FE700340F1A780E90732
:107B000003D500212046FFF79FFEAA0703D50121D8
:107B10002046FFF799FE6B0703D502212046FFF7A9
:107B200093FE2F0703D503212046FFF78DFEEE06B7
:107B300003D504212046FFF787FEA80603D50521BB
:107B40002046FFF781FE690603D506212046FFF790
:107B50007BFE2A0603D507212046FFF775FEEB05BD
:107B600074D520460821BDE8F84FFFF76DBED4F864
:107B700090904FF0000B4FF0010AD4F894305FFA68
:107B80008BF79B689F423FF638AF09EB4713D3F85A
:107B9000002902F44022B2F5802F20D1D3F8002929
:107BA000002A1CDAD3F8002942F09042C3F80029D9
:107BB000D3F80029002AFBDB3946D4F89000FFF700
:107BC00087FB22890AFA07F322EA0303238104EBE5
:107BD0008703DB689B6813B13946204698470BF151
:107BE000010BCAE7910701D1D0F80080072A02F102
:107BF00001029CBF03F8018B4FEA18283FE704EB12
:107C0000830300F58050DA68D2F818C0DCF8082049
:107C1000DCE9001CA1EB0C0C00218F4208D1DB68D1
:107C20009B699A683A449A605A683A445A6029E7CC
:107C300011F0030F01D1D0F800808C4501F1010152
:107C400084BF02F8018B4FEA1828E6E7BDE8F88FF9
:107C500008B50348FFF774FEBDE8084000F070BFA8
:107C60001465002008B50348FFF76AFEBDE8084028
:107C700000F066BFB0650020D0F8903003EB4111F2
:107C8000D1F8003B43F40013C1F8003B70470000FB
:107C9000D0F8903003EB4111D1F8003943F40013D0
:107CA000C1F8003970470000D0F8903003EB411163
:107CB000D1F8003B23F40013C1F8003B70470000EB
:107CC000D0F8903003EB4111D1F8003923F40013C0
:107CD000C1F8003970470000064BD3F8DC2002439E
:107CE000C3F8DC20D3F804211043C3F80401D3F80F
:107CF00004317047004402583A4B4FF0FF31D3F83B
:107D0000802062F00042C3F88020D3F8802002F087
:107D10000042C3F88020D3F88020D3F88420C3F831
:107D20008410D3F884200022C3F88420D3F8840080
:107D3000D86F40F0FF4040F4FF0040F4DF4040F0D7
:107D40007F00D867D86F20F0FF4020F4FF0020F4B8
:107D5000DF4020F07F00D867D86FD3F888006FEA43
:107D600040506FEA5050C3F88800D3F88800C0F341
:107D70000A00C3F88800D3F88800D3F89000C3F84D
:107D80009010D3F89000C3F89020D3F89000D3F867
:107D90009400C3F89410D3F89400C3F89420D3F857
:107DA0009400D3F89800C3F89810D3F89800C3F85B
:107DB0009820D3F89800D3F88C00C3F88C10D3F82F
:107DC0008C00C3F88C20D3F88C00D3F89C00C3F847
:107DD0009C10D3F89C10C3F89C20D3F89C3000F082
:107DE000D7B900BF0044025808B50122534BC3F86D
:107DF0000821534BD3F8F42042F00202C3F8F420D8
:107E0000D3F81C2142F00202C3F81C210222D3F84D
:107E10001C314C4BDA605A689104FCD54A4A1A600E
:107E200001229A60494ADA6000221A614FF4404206
:107E30009A61444B9A699204FCD51A6842F48072A4
:107E40001A603F4B1A6F12F4407F04D04FF4803217
:107E50001A6700221A671A6842F001021A60384B4A
:107E60001A685007FCD500221A611A6912F038020C
:107E7000FBD1012119604FF0804159605A67344AA3
:107E8000DA62344A1A611A6842F480321A602C4B62
:107E90001A689103FCD51A6842F480521A601A6875
:107EA0009204FCD52C4A2D499A6200225A63196328
:107EB00001F57C01DA6301F2E71199635A64284AFB
:107EC0001A64284ADA621A6842F0A8521A601C4BF7
:107ED0001A6802F02852B2F1285FF9D148229A615B
:107EE0004FF48862DA6140221A621F4ADA641F4A3C
:107EF0001A651F4A5A651F4A9A6532231E4A136043
:107F0000136803F00F03022BFAD10D4A136943F0F3
:107F100003031361136903F03803182BFAD14FF0F0
:107F20000050FFF7D9FE4FF08040FFF7D5FE4FF02D
:107F30000040BDE80840FFF7CFBE00BF0080005101
:107F4000004402580048025800C000F0020000013E
:107F50000000FF0100889008222040006302090110
:107F6000470E0508DD0BBF012000002000000110B6
:107F70000910E00000010110002000524FF0B04253
:107F800008B5D2F8883003F00103C2F8883023B175
:107F9000044A13680BB150689847BDE8084000F0E8
:107FA000CFBD00BF986600204FF0B04208B5D2F8B0
:107FB000883003F00203C2F8883023B1044A936882
:107FC0000BB1D0689847BDE8084000F0B9BD00BFCC
:107FD000986600204FF0B04208B5D2F8883003F020
:107FE0000403C2F8883023B1044A13690BB1506905
:107FF0009847BDE8084000F0A3BD00BF9866002088
:108000004FF0B04208B5D2F8883003F00803C2F848
:10801000883023B1044A93690BB1D0699847BDE811
:10802000084000F08DBD00BF986600204FF0B042C0
:1080300008B5D2F8883003F01003C2F8883023B1B5
:10804000044A136A0BB1506A9847BDE8084000F033
:1080500077BD00BF986600204FF0B04310B5D3F84D
:10806000884004F47872C3F88820A30604D5124A25
:10807000936A0BB1D06A9847600604D50E4A136B19
:108080000BB1506B9847210604D50B4A936B0BB18B
:10809000D06B9847E20504D5074A136C0BB1506CBE
:1080A0009847A30504D5044A936C0BB1D06C98474C
:1080B000BDE8104000F044BD986600204FF0B0438A
:1080C00010B5D3F8884004F47C42C3F888206205D8
:1080D00004D5164A136D0BB1506D9847230504D58E
:1080E000124A936D0BB1D06D9847E00404D50F4A46
:1080F000136E0BB1506E9847A10404D50B4A936ED2
:108100000BB1D06E9847620404D5084A136F0BB1C7
:10811000506F9847230404D5044A936F0BB1D06F76
:108120009847BDE8104000F00BBD00BF98660020E6
:1081300008B50348FCF704FDBDE8084000F000BDA9
:10814000A436002008B50348FCF7FEFDBDE8084052
:1081500000F0F6BCFC38002008B50348FCF7F4FD3D
:10816000BDE8084000F0ECBC6839002008B50348C1
:10817000FCF7EAFDBDE8084000F0E2BCD43900207D
:1081800008B500F03FFDBDE8084000F0D9BC000094
:10819000062108B5084600F033F80621072000F054
:1081A0002FF80621082000F02BF80621092000F006
:1081B00027F806210A2000F023F80621172000F0F6
:1081C0001FF80621282000F01BF809217A2000F072
:1081D00017F809217C2000F013F80721322000F065
:1081E0000FF80C21272000F00BF80C21352000F0AF
:1081F00007F80C215220BDE8084000F001B800004B
:10820000090100F16043012203F56143C9B283F81B
:10821000001300F01F039A4043099B0003F16043E1
:1082200003F56143C3F880211A60704708B5FFF772
:1082300063FD00F0AFFCFDF7C1F9FDF75FF9FDF755
:1082400097FBFDF769FAFEF735FABDE8084000F044
:1082500029BA000030B50433039C0172002104FBED
:108260000325C160C0E90653049B0363059BC0E975
:108270000000C0E90422C0E90842C0E90A114363D2
:1082800030BD00000022416AC260C0E90411C0E9AB
:108290000A226FF00101FDF793BF0000D0E904321C
:1082A000934201D1C2680AB9181D70470020704777
:1082B000036919600021C2680132C260C2691344B7
:1082C00082699342036124BF436A0361FDF76CBF77
:1082D00038B504460D46E3683BB162690020131DC2
:1082E0001268A3621344E36207E0237A33B9294694
:1082F0002046FDF749FF0028EDDA38BD6FF0010098
:10830000FBE70000C368C269013BC36043691344D3
:1083100082699342436124BF436A436100238362BD
:10832000036B03B11847704770B53023044683F3DD
:108330001188866A3EB9FFF7CBFF054618B186F370
:108340001188284670BDA36AE26A13F8015B934264
:10835000A36202D32046FFF7D5FF002383F31188E1
:10836000EFE700002DE9F84F04460E461746984601
:108370004FF0300989F311880025AA46D4F828B0B7
:10838000BBF1000F09D141462046FFF7A1FF20B104
:108390008BF311882846BDE8F88FD4E90A12A7EBC1
:1083A000050B521A934528BF9346BBF1400F1BD9CA
:1083B000334601F1400251F8040B914243F8040B9B
:1083C000F9D1A36A403640354033A362D4E90A2389
:1083D0009A4202D32046FFF795FF8AF31188BD42E7
:1083E000D8D289F31188C9E730465A46F9F792FC8A
:1083F000A36A5E445D445B44A362E7E710B5029C58
:108400000433017203FB0421C460C0E90613002396
:10841000C0E90A33039B0363049BC0E90000C0E981
:108420000422C0E90842436310BD0000026A6FF0F5
:108430000101C260426AC0E904220022C0E90A22A6
:10844000FDF7BEBED0E904239A4201D1C26822B929
:10845000184650F8043B0B60704700231846FAE7B3
:10846000C3680021C2690133C36043691344826950
:108470009342436124BF436A4361FDF795BE000008
:1084800038B504460D46E3683BB1236900201A1D48
:10849000A262E2691344E36207E0237A33B9294612
:1084A0002046FDF771FE0028EDDA38BD6FF00100BF
:1084B000FBE7000003691960C268013AC260C26943
:1084C000134482699342036124BF436A036100231A
:1084D0008362036B03B118477047000070B5302307
:1084E0000D460446114683F31188866A2EB9FFF7BC
:1084F000C7FF10B186F3118870BDA36A1D70A36A0F
:10850000E26A01339342A36204D3E169204604394D
:10851000FFF7D0FF002080F31188EDE72DE9F84F39
:1085200004460D46904699464FF0300A8AF311886A
:108530000026B346A76A4FB949462046FFF7A0FF79
:1085400020B187F311883046BDE8F88FD4E90A07D7
:108550003A1AA8EB0607974228BF1746402F1BD9A7
:1085600005F1400355F8042B9D4240F8042BF9D146
:10857000A36A40364033A362D4E90A239A4204D363
:10858000E16920460439FFF795FF8BF311884645D2
:10859000D9D28AF31188CDE729463A46F9F7BAFBD2
:1085A000A36A3D443E443B44A362E5E7D0E904238B
:1085B0009A4217D1C3689BB1836A8BB1043B9B1A63
:1085C0000ED01360C368013BC360C3691A4483695A
:1085D0009A42026124BF436A03610023836201233C
:1085E000184670470023FBE701F01F03F0B502F0C7
:1085F0001F0456095A1C0123B6EB511F50F8265090
:1086000003FA02F34FEA511703F1FF333DBF50F86D
:108610002720C4F12000134003EA05003BBF03FA02
:1086200000F225FA04F0E0401043F0BD70B57E2260
:108630007F210546FFF7D8FF18B1012819D0002087
:1086400070BD3E2249212846FFF7CEFF2F22044667
:1086500031212846FFF7C8FF064601345022023672
:1086600053212846B440FFF7BFFF093804FA00F051
:10867000E6E7302245212846FFF7B6FF01308002A9
:10868000DEE7000090F8D63090F8D7201B0403EB0B
:10869000026390F8D42090F8D500134403EB002037
:1086A0007047000000F084BA014B586A704700BF61
:1086B000000C0040034B002258631A610222DA606A
:1086C000704700BF000C0040014B0022DA60704789
:1086D000000C0040014B5863704700BF000C004085
:1086E000024B034A1A60034A5A60704764660020CE
:1086F0002067002000000220074B494210B55C684B
:10870000201A08401968821A8A4203D3A24201D86B
:108710005A6010BD0020FCE76466002008B53023D5
:1087200083F31188FFF7E8FF002383F3118808BD66
:108730000448054B03600023C0E901330C3000F00E
:1087400017B900BF6C6600201D870008CB1D083AD2
:1087500023F00703591A521A10B4D2080024C0E9B2
:10876000004384600C301C605A605DF8044B00F0DC
:10877000FFB800002DE9F74F364FCD1D8846002881
:1087800018BF0746082A4FEAD50538BF082207F167
:108790000C003C1D9146019000F02CF9019809F164
:1087A0000701C9F1000E2246246864B900F02CF9D3
:1087B0003B68CBB308224946E8009847044698B383
:1087C00040E9027830E004EB010CD4F804A00CEA94
:1087D0000E0C0AF10106ACF1080304EBC6069E423A
:1087E000E1D9A6EB0C0CB5EBEC0F4FEAEC0BDAD8A9
:1087F0009C421DD204F10802AB45A3EB02024FEAF2
:10880000E202626009D9691CED4303EBC1025D44D9
:108810005560256843F8315022601C46C3F8048037
:1088200044F8087B00F0F0F8204603B0BDE8F08F74
:10883000AA45216802D111602346EEE7013504EB19
:10884000C50344F8351003F10801761AF6105E608E
:108850001360F1E76C66002073B50446A0F10805CB
:1088600050F8080C54F8043C061D0C3007330190F6
:10887000DB0844F8043C00F0BDF8334601989E4202
:108880001A6801D0AB4228D20AB1954225D244F8E9
:10889000082C54F8042C1D60013254F8081C05EB18
:1088A000C206B14206D14E68324444F8042C0A682C
:1088B00044F8082C5E68711C03EBC1018D4207D19E
:1088C00054F8042C013232445A6054F8082C1A60CF
:1088D00002B0BDE8704000F097B81346CFE7000043
:1088E000FEE7000070B51E4B0025044686B05860B8
:1088F0000E460563816300F0FBF804F12803A560D0
:108900006563C4E90A3304F11003C4E904334FF08A
:10891000FF33C4E90044C4E90635FFF7C5FE2B4622
:10892000024604F13C012046C4E9082380230D4A95
:108930006567FDF7A3FB7368E0600B4A03620123E0
:10894000009280F824306846F26801923269CDE9DD
:108950000223064BCDE90435FDF7C4FB06B070BD1C
:10896000E8480020B4960008AC960008E1880008AA
:108970000023C0E9000083600361704770B51C4BA1
:1089800005468468DE685CB3B44213D103690133E1
:10899000036170BDA36094F8243083B1062B15D118
:1089A000A06A2146D4E9003213605A60FDF7B8FA94
:1089B000A36A9C68B368A2689A42EBD306E0D4E944
:1089C0000032204613605A60FDF7BAFA2846314655
:1089D000FDF7A6FAB5620620BDE87040FDF7B2BA11
:1089E0000369866001330361336BC3603063D0E792
:1089F0004046002008B5302383F31188FFF7BEFFFF
:108A0000002383F3118808BD194BD96883688B4212
:108A100010B520D1302383F311880269013A026135
:108A2000B2B90468C368A0420B631ED04A6B9BB9FD
:108A300001238A60036103681A68026050601A6B40
:108A40008360C26018631846FDF77AFAFDF7CAFA28
:108A5000002383F3118810BD1C68A34203D0A468CF
:108A6000A24238BF2246DB68E1E78260F0E700BF40
:108A700040460020024A536B18435063704700BFC2
:108A80004046002070B5104E82B0FDF7D3FA05467F
:108A9000FFF70AFE326803469042336037BF0B4A45
:108AA0000A495168146836BF0131D1E9004151606B
:108AB0000419284641F100010191FDF7C5FA20464D
:108AC000019902B070BD00BF8C6600209066002046
:108AD000EFF30983054968334A6B22F001024A63C8
:108AE00083F30988002383F31188704700EF00E0C7
:108AF000302080F3118862B60D4B0E4AD96821F4FC
:108B0000E0610904090C0A430B49DA60D3F8FC2040
:108B100042F08072C3F8FC20084AC2F8B01F116806
:108B200041F0010111602022DA7783F822007047BA
:108B300000ED00E00003FA0555CEACC5001000E0E2
:108B4000302310B583F311880E4B5B6813F4006378
:108B500014D0F1EE103AEFF309844FF08073683CC3
:108B6000E361094BDB6B236684F30988FDF718FA90
:108B700010B1064BA36110BD054BFBE783F31188D1
:108B8000F9E700BF00ED00E000EF00E02F0400086F
:108B9000320400080023054A19460133102BC2E9AC
:108BA000001102F10802F8D1704700BF986600205A
:108BB000114BD3F8E82042F00802C3F8E820D3F8BC
:108BC000102142F00802C3F810210C4AD3F81031EA
:108BD000D36B43F00803D363C722094B9A624FF06B
:108BE000FF32DA6200229A615A63DA605A60012227
:108BF0005A611A60704700BF004402580010005CC0
:108C0000000C0040094A08B51169D3680B40D9B27D
:108C10009B076FEA0101116107D5302383F31188A7
:108C2000FDF706FA002383F3118808BD000C00400D
:108C3000FEF7A0B8012838BF012010B50446204631
:108C4000FEF758F830B900F007F808B900F00CF852
:108C50008047F4E710BD0000024B1868BFF35B8F3C
:108C6000704700BF1867002008B5062000F056F8CE
:108C70000120FDF755FC000010B501390244904277
:108C800001D1002005E0037811F8014FA34201D083
:108C9000181B10BD0130F2E7884210B501EB020449
:108CA00002D98442234607D8431EA14208D011F8B6
:108CB000012B03F8012FF8E7024401468A4200D154
:108CC00010BD13F8014D02F8014DF7E71F2938B523
:108CD00004460D4604D9162303604FF0FF3038BD1B
:108CE000426C12B152F821304BB9204600F030F8F6
:108CF0002A4601462046BDE8384000F017B8012B4F
:108D00000AD0591C03D1162303600120E7E7002491
:108D100042F82540284698470020E0E7024B0146EC
:108D20001868FFF7D3BF00BF7422002038B5074D85
:108D300000230446084611462B60FDF7F5FB431C53
:108D400002D12B6803B1236038BD00BF1C6700202F
:108D5000FDF7E4BBC9B2034610F8012B1AB18A42F1
:108D6000F9D118467047002918BF0023F9E7000021
:108D7000034611F8012B03F8012B002AF9D17047A3
:108D800010B50139034632B111F8014F03F8014B18
:108D9000013A002CF7D11A440021934200D110BDB2
:108DA00003F8011BF9E700004D4435002D2D0A00A2
:108DB0002F6172647570696C6F742E6162696E00E8
:108DC0002F6172647570696C6F742D766572696657
:108DD000792E6162696E002F6172647570696C6FC3
:108DE000742D666C6173682E6162696E002F61720A
:108DF000647570696C6F742D666C61736865642E40
:108E00006162696E000000000000000000000000C8
:108E1000090F0008A50F000855110008DD0F000814
:108E20009D0F00080000000000000000050F000872
:108E3000B10F00088D110008010F00080D0F000888
:108E400053544D333248373F3F3F0053544D333234
:108E5000483733782F3732780053544D3332483700
:108E600034332F3735332F373530000001105A0097
:108E70000310590001205800032056002F00000065
:108E80005375636365737366756C6C79206D6F756C
:108E90006E746564205344436172642028736C6F60
:108EA00077646F776E3D2575290A0000EB76904553
:108EB000584641542020200046415433322020207F
:108EC000000000002A3A3C3E7C223F7F002B2C3BD6
:108ED0003D5B5D0043554541414141434545454961
:108EE000494941414592924F4F4F5555594F554F22
:108EF0009C4F9E9F41494F55A5A5A6A7A8A9AAABDF
:108F0000ACADAEAFB0B1B2B3B4414141B8B9BABB88
:108F1000BCBDBEBFC0C1C2C3C4C54141C8C9CACB24
:108F2000CCCDCECFD1D145454549494949D9DADBE8
:108F3000DCDD49DF4FE14F4F4F4FE6E8E85555552F
:108F40005959EEEFF0F1F2F3F4F5F6F7F8F9FAFB10
:108F5000FCFDFEFF01030507090E10121416181C74
:108F60001E00000061001A03E0001703F800070369
:108F7000FF000100780100013001320106013901D2
:108F800010014A012E017901060180014D004302C2
:108F900081018201820184018401860187018701A8
:108FA00089018A018B018B018D018E018F01900156
:108FB0009101910193019401F601960197019801A5
:108FC00098013D029B019C019D0120029F01A0018F
:108FD000A001A201A201A401A401A601A701A70169
:108FE000A901AA01AB01AC01AC01AE01AF01AF0117
:108FF000B101B201B301B301B501B501B701B801C7
:10900000B801BA01BB01BC01BC01BE01F701C0013E
:10901000C101C201C301C401C501C401C701C80126
:10902000C701CA01CB01CA01CD011001DD01010058
:109030008E01DE011201F3010300F101F401F401DC
:10904000F8012801220212013A020900652C3B02B4
:109050003B023D02662C3F024002410241024602B1
:109060000A015302400081018601550289018A01EB
:1090700058028F015A0290015C025D025E025F029B
:109080009301610262029401640265026602670252
:10909000970196016A02622C6C026D026E029C01BD
:1090A000700271029D01730274029F0176027702C1
:1090B000780279027A027B027C02642C7E027F02B3
:1090C000A60181028202A90184028502860287022A
:1090D000AE014402B101B20145028D028E028F023F
:1090E00090029102B7017B030300FD03FE03FF031F
:1090F000AC0304008603880389038A03B1031103C8
:10910000C2030200A303A303C4030803CC030300A8
:109110008C038E038F03D8031801F2030A00F903AE
:10912000F303F403F503F603F703F703F903FA0374
:10913000FA033004200350041007600422018A045B
:109140003601C1040E01CF040100C004D004440163
:1091500061052604000000007D1D0100632C001E37
:109160009601A01E5A01001F0806101F0606201FA8
:109170000806301F0806401F0606511F0700591F2A
:10918000521F5B1F541F5D1F561F5F1F601F080685
:10919000701F0E00BA1FBB1FC81FC91FCA1FCB1FDD
:1091A000DA1FDB1FF81FF91FEA1FEB1FFA1FFB1F57
:1091B000801F0806901F0806A01F0806B01F0400A5
:1091C000B81FB91FB21FBC1FCC1F0100C31FD01F87
:1091D0000206E01F0206E51F0100EC1FF31F01005D
:1091E000FC1F4E2101003221702110028421010058
:1091F0008321D0241A05302C2F04602C0201672C07
:109200000601752C0201802C6401002D260841FF07
:109210001A030000C700FC00E900E200E400E000DF
:10922000E500E700EA00EB00E800EF00EE00EC00EC
:10923000C400C500C900E600C600F400F600F20054
:10924000FB00F900FF00D600DC00F800A300D80006
:10925000D7009201E100ED00F300FA00F100D10027
:10926000AA00BA00BF00AE00AC00BD00BC00A10067
:10927000AB00BB0091259225932502252425C10032
:10928000C200C000A9006325512557255D25A20015
:10929000A5001025142534252C251C2500253C254A
:1092A000E300C3005A25542569256625602550250D
:1092B0006C25A400F000D000CA00CB00C80031012A
:1092C000CD00CE00CF0018250C2588258425A600CA
:1092D000CC008025D300DF00D400D200F500D500FB
:1092E000B500FE00DE00DA00DB00D900FD00DD0085
:1092F000AF00B400AD00B1001720BE00B600A7005B
:10930000F700B800B000A800B700B900B300B20081
:10931000A025A00001000000000000000096000051
:10932000000000000000000000000000000000003D
:109330000000000000000000AD660008B1660008F3
:1093400091510008C9540008255100084D510008EA
:10935000755100080D510008000000007D550008FF
:1093600069550008A5550008915500089D5500084D
:10937000895500087555000861550008B155000869
:10938000000000009556000881560008BD560008F0
:10939000A9560008B5560008A15600088D560008C9
:1093A00079560008C95600080000000001000000BE
:1093B0000000000063300000B493000800000000CB
:1093C00000000000B8460020E84800200000802A85
:1093D00000020000AAAAAAAA00000024FFFF0000C1
:1093E0000000000000A00A00000200A00000000031
:1093F000AAAAAAAA00010050FFFF0000000009006D
:10940000000000990000000600000000AAAAAAAA15
:1094100000000001FFFF0000000000000000080045
:1094200020A00A0000000000AAAAAAAA1040050075
:10943000FFFF0000000800BB77000000401402009E
:1094400028000000AAAAAAAA00000100FFFF00004D
:1094500000000000070000000020000100000000E4
:10946000AAAAAAAA00100000FFFF0000000000073F
:10947000000000000041800000000000AAAAAAAA83
:1094800000404000FFFF00000000000000A00000BE
:109490000004004000000000AAAAAAAA000400409C
:1094A000FFFF0000000000000000000000011500A8
:1094B00000000000AAAAAAAA00011500FFFF0000F0
:1094C000000000000000000000000000000000009C
:1094D000AAAAAAAA00000000FFFF000000000000E6
:1094E000000000000000000000000000AAAAAAAAD4
:1094F00000000000FFFF000000000000000000006E
:109500004172647550696C6F740025424F4152443A
:10951000252D424C002553455249414C2500000061
:109520000200000000000000B5580008255900089E
:109530004000400098610020A86100200200000067
:109540000000000003000000000000006D5900084A
:109550000000000010000000B861002000000000C2
:10956000010000000000000014650020010102005D
:10957000A9670008B9660008556700083967000840
:10958000430000008895000809024300020100C062
:109590003209040000010202010005240010010547
:1095A00024010001042402020524060001070582AB
:1095B000030800FF09040100020A0000000705017A
:1095C0000240000007058102400000001200000078
:1095D000D495000812011001020000400912415701
:1095E00000020102030100000403090425424F4167
:1095F000524425005069786861776B3658003031E5
:109600003233343536373839414243444546000019
:1096100000000020000002000200000000000030F6
:109620000000040008000000000000240000080002
:10963000040000000004000000FC00000200000024
:109640000000043000800000080000000000003826
:1096500000000100010000001F1C1F1E1F1E1F1F15
:109660001E1F1E1F1F1D1F1E1F1E1F1F1E1F1E1F12
:1096700000000000C95A0008815D00082D5E000846
:10968000400040004C6600204C66002001000000B5
:109690005C6600208000000040010000080000001F
:1096A00000010000001000000800000069646C6503
:1096B000000000006D61696E002C04380404380855
:1096C0000C10141C20242526000000000000640457
:1096D0000100040000000000000C001028303400DD
:1096E000886DFF7F010000003500000000000000D1
:1096F00000001E0000000000FF000000F0480020F5
:10970000D439002068390020FC3800200000000017
:10971000408E0008830400004B8E000850040000B7
:10972000598E0008010000000000000000960000B3
:10973000000008009600000000080000040000007F
:10974000E895000800000000000000000000000094
:10975000000000000000000000000000782200204F
:1097600000000000000000000000000000000000F9
:1097700000000000000000000000000000000000E9
:1097800000000000000000000000000000000000D9
:1097900000000000000000000000000000000000C9
:020000040801F1
:020000040802F0
:1000000000060024E90D0208514712088103020886
:10001000CD461208C5461208C9461208EB0D020863
:10002000EB0D0208EB0D0208EB0D0208CD0A1908D2
:10003000EB0D0208EB0D0208EB0D0208EB0D0208B8
:10004000EB0D0208EB0D0208EB0D0208EB0D0208A8
:10005000EB0D0208EB0D0208CD9F1908F99F190856
:1000600025A0190851A019087DA01908F51919082B
:100070001D1A1908491A1908751A1908A11A190818
:10008000C91A1908F51A1908DD151908E5341208F6
:10009000CD351208553512083D361208A9A01908A9
:1000A000EB0D0208EB0D0208EB0D0208EB0D020848
:1000B00035A21908EB0D020845A2190851231908A9
:1000C000C523190839241908AD241908053A190857
:1000D000193A190895A11908A9A11908BDA119086B
:1000E0000DA11908EB0D0208EB0D02086DA219080D
:1000F00081A2190895A21908A9A21908211B19089B
:10010000EB0D0208EB0D020859A219082D3A190847
:10011000D1A11908E5A11908EB0D0208EB0D0208A1
:100120004D1B1908751B1908A11B1908CD1B1908AF
:10013000F91B1908CD2A1908EB0D0208EB0D02086E
:10014000EB0D0208EB0D0208EB0D0208EB0D0208A7
:10015000211C19084D1C1908791C1908F9A1190846
:100160002125190895251908EB0D0208EB0D020849
:10017000EB0D0208199C1908EB0D0208EB0D0208A3
:10018000EB0D0208EB0D02080DA2190821A21908B7
:10019000EB0D0208413A1908EB0D0208EB0D0208BD
:1001A000EB0D0208EB0D0208EB0D0208EB0D020847
:1001B000EB0D0208EB0D0208EB0D020809261908E9
:1001C0007D261908EB0D0208EB0D0208EB0D020865
:1001D000EB0D0208059C1908EB0D0208EB0D020857
:1001E000EB0D0208EB0D0208EB0D0208EB0D020807
:1001F000EB0D0208EB0D0208EB0D0208EB0D0208F7
:10020000EB0D0208EB0D0208EB0D0208EB0D0208E6
:10021000EB0D0208EB0D0208EB0D0208EB0D0208D6
:10022000EB0D0208EB0D0208EB0D0208EB0D0208C6
:1002300081A11908EB0D0208EB0D0208FD15190844
:10024000EB0D0208A5171908CD171908F917190899
:1002500025181908511819087D181908A91819081E
:10026000D5181908EB0D0208EB0D0208EB0D02087A
:10027000EB0D0208EB0D0208EB0D0208EB0D020876
:10028000EB0D0208EB0D0208EB0D0208EB0D020866
:10029000EB0D0208EB0D0208EB0D0208EB0D020856
:1002A000EB0D0208EB0D0208EB0D0208EB0D020846
:1002B000EB0D0208EB0D0208EB0D0208EB0D020836
:1002C000EB0D0208EB0D0208EB0D0208EB0D020826
:1002D000EB0D0208EB0D0208EB0D0208EB0D020816
:1002E0005D4B0208C1880208D1D10208F14203081F
:1002F000A9B503081988040801E60408157505085E
:10030000C1020708D17E0908C185090835300A08ED
:10031000D1B00A0869B90A08F5BC0A0821470B08D8
:10032000C1720B08F5810B0841230C0819DD0C087C
:10033000ED080E0809BD0E0885CC0E08B939120863
:100340001D3F1208D15E1208B1091408F15B1408B0
:10035000FDB11408E505150851C816089D241708B5
:10036000E1411708C184170861A8170865D9170863
:1003700081E61708912318089D2D18080000000039
:10038000EFF30383EFF30982EFF30881DFF814D072
:100390002DE9FE4F684600F0FDFFBDE8FE4F8D469B
:1003A00070470000B4330024F1EE101AA0EC200ACC
:1003B00001607047A0EC108A704700BF81F00041D7
:1003C00002E000BF83F0004330B54FEA41044FEA3A
:1003D000430594EA050F08BF90EA020F1FBF54EAD5
:1003E000000C55EA020C7FEA645C7FEA655C00F071
:1003F000E2804FEA5454D4EB5555B8BF6D420CDD42
:100400002C4480EA020281EA030382EA000083EAC4
:10041000010180EA020281EA0303362D88BF30BD64
:1004200011F0004F4FEA01314FF4801C4CEA1131BA
:1004300002D0404261EB410113F0004F4FEA033319
:100440004CEA133302D0524263EB430394EA050FA4
:1004500000F0A780A4F10104D5F1200E0DDB02FA13
:100460000EFC22FA05F2801841F1000103FA0EF2A7
:10047000801843FA05F359410EE0A5F120050EF16D
:10048000200E012A03FA0EFC28BF4CF0020C43FA9E
:1004900005F3C01851EBE37101F0004507D54FF0AB
:1004A000000EDCF1000C7EEB00006EEB0101B1F5FB
:1004B000801F1BD3B1F5001F0CD349085FEA300041
:1004C0004FEA3C0C04F101044FEA445212F5800F4C
:1004D00080F09A80BCF1004F08BF5FEA500C50F1E9
:1004E000000041EB045141EA050130BD5FEA4C0CCC
:1004F000404141EB0101013C28BFB1F5801FE9D229
:1005000091F0000F04BF01460020B1FA81F308BF4B
:100510002033A3F10B03B3F120020CDA0C3208DD17
:1005200002F1140CC2F10C0201FA0CF021FA02F1F2
:100530000CE002F11402D8BFC2F1200C01FA02F162
:1005400020FA0CFCDCBF41EA0C019040E41AA2BF87
:1005500001EB0451294330BD6FEA04041F3C1CDA4F
:100560000C340EDC04F11404C4F1200220FA04F06F
:1005700001FA02F340EA030021FA04F345EA030119
:1005800030BDC4F10C04C4F1200220FA02F001FADB
:1005900004F340EA0300294630BD21FA04F029465D
:1005A00030BD94F0000F83F4801306BF81F48011F6
:1005B0000134013D4EE77FEA645C18BF7FEA655C69
:1005C00029D094EA050F08BF90EA020F05D054EA3B
:1005D000000C04BF1946104630BD91EA030F1EBF40
:1005E0000021002030BD5FEA545C05D14000494144
:1005F00028BF41F0004130BD14F580043CBF01F537
:10060000801130BD01F0004545F0FE4141F470011C
:100610004FF0000030BD7FEA645C1ABF19461046F7
:100620007FEA655C1CBF0B46024650EA013406BFF8
:1006300052EA033591EA030F41F4002130BD00BFB7
:1006400090F0000F04BF0021704730B54FF4806474
:1006500004F132044FF000054FF0000150E700BFF5
:1006600090F0000F04BF0021704730B54FF4806454
:1006700004F1320410F0004548BF40424FF0000141
:100680003EE700BF42004FEAE2014FEA31014FEA84
:1006900002701FBF12F07F4393F07F4F81F06051D3
:1006A000704732F07F4208BF704793F07F4F04BF1E
:1006B00041F40021704730B54FF4607401F00045FB
:1006C00021F000411CE700BF50EA010208BF70475B
:1006D00030B54FF000050AE050EA010208BF70474C
:1006E00030B511F0004502D5404261EB41014FF4B5
:1006F000806404F132045FEA915C3FF4D8AE4FF0BD
:1007000003025FEADC0C18BF03325FEADC0C18BF9F
:10071000033202EBDC02C2F1200300FA03FC20FAF0
:1007200002F001FA03FE40EA0E0021FA02F114443D
:10073000BDE600BF80F0004002E000BF81F0004154
:1007400042001FBF5FEA410392EA030F7FEA226C77
:100750007FEA236C6AD04FEA1262D2EB1363C1BF07
:10076000D218414048404140B8BF5B42192B88BF76
:10077000704710F0004F40F4000020F07F4018BF99
:10078000404211F0004F41F4000121F07F4118BFB9
:10079000494292EA030F3FD0A2F1010241FA03FC61
:1007A00010EB0C00C3F1200301FA03F100F0004349
:1007B00002D5494260EB4000B0F5000F13D3B0F111
:1007C000807F06D340084FEA310102F10102FE2A80
:1007D00051D2B1F1004F40EBC25008BF20F00100F0
:1007E00040EA03007047490040EB0000013A28BF8F
:1007F000B0F5000FEDD2B0FA80FCACF1080CB2EB12
:100800000C0200FA0CF0AABF00EBC250524218438F
:10081000BCBFD0401843704792F0000F81F4000134
:1008200006BF80F400000132013BB5E74FEA410307
:100830007FEA226C18BF7FEA236C21D092EA030F73
:1008400004D092F0000F08BF0846704790EA010FED
:100850001CBF0020704712F07F4F04D1400028BF1A
:1008600040F00040704712F100723CBF00F50000FC
:10087000704700F0004343F0FE4040F40000704732
:100880007FEA226216BF08467FEA236301464202DE
:1008900006BF5FEA412390EA010F40F480007047F1
:1008A0004FF0000304E000BF10F0004348BF404297
:1008B0005FEA000C08BF704743F0964301464FF0D3
:1008C00000001CE050EA010208BF70474FF000032F
:1008D0000AE000BF50EA010208BF704711F0004370
:1008E00002D5404261EB41015FEA010C02BF844640
:1008F0000146002043F0B64308BFA3F18053A3F59F
:100900000003BCFA8CF2083AA3EBC25310DB01FAE5
:1009100002FC634400FA02FCC2F12002BCF1004F69
:1009200020FA02F243EB020008BF20F001007047FA
:1009300002F1200201FA02FCC2F1200250EA4C004E
:1009400021FA02F243EB020008BF20EADC70704794
:100950007BB972B90029BEBF00204FF0004106E00C
:1009600008BF00281CBF6FF000414FF0FF3000F0BF
:1009700039BAADF1080C6DE904CE002909DB002B72
:100980001ADB00F0C7F8DDF804E0DDE9022304B06B
:100990007047404261EB4101002B1BDB00F0BAF8CD
:1009A000DDF804E0DDE9022304B0404261EB4101DF
:1009B000524263EB43037047524263EB430300F040
:1009C000A9F8DDF804E0DDE9022304B0404261EB60
:1009D00041017047524263EB430300F09BF8DDF89E
:1009E00004E0DDE9022304B0524263EB43037047A5
:1009F00053B94AB9002908BF00281CBF4FF0FF3186
:100A00004FF0FF3000F0EEB9ADF1080C6DE904CE07
:100A100000F080F8DDF804E0DDE9022304B070475F
:100A200030B1012390FAA0F0B0FA80F0184470477A
:100A300008460029FBD02123F4E700BF430803F058
:100A40005533C01A830803F0333300F033301844B1
:100A500000EB101000F00F3000EB002000EB004026
:100A6000000E704708B502460B4643EC172BB5EE57
:100A7000C07BF1EE10FA03D4BDE8084000F02AB8BC
:100A8000B1EE477B51EC170B00F024F8404261EBCC
:100A9000410108BD9FED0B6B07EE900A9FED0B5BCC
:100AA000B7EEE77A27EE066BBCEEC66BB8EE464BA8
:100AB000A4EE457BFCEEC77B16EE101A17EE900AEB
:100AC000704700BF000000000000F03D0000000083
:100AD0000000F0419FED0B6B41EC170B9FED0B5BA2
:100AE00027EE066BBCEEC66BB8EE464BA4EE457B1C
:100AF000FCEEC77B16EE101A17EE900A704700BF87
:100B0000AFF30080000000000000F03D0000000096
:100B10000000F0412DE9F047089D04468E46002B69
:100B20004DD18A42944669D9B2FA82F252B101FAA1
:100B300002F3C2F1200120FA01F10CFA02FC41EAB1
:100B4000030E94404FEA1C48210CBEFBF8F61FFA36
:100B50008CF708FB16E341EA034306FB07F19942D1
:100B60000AD91CEB030306F1FF3080F01F81994284
:100B700040F21C81023E63445B1AA4B2B3FBF8F05E
:100B800008FB103344EA034400FB07F7A7420AD9E5
:100B90001CEB040400F1FF3380F00A81A74240F20D
:100BA00007816444023840EA0640E41B00261DB178
:100BB000D4400023C5E900433146BDE8F0878B42AD
:100BC00009D9002D00F0EF800026C5E9000130466C
:100BD0003146BDE8F087B3FA83F6002E4AD18B4246
:100BE00002D3824200F2F980841A61EB03030120F0
:100BF0009E46002DE0D0C5E9004EDDE702B9FFDEDC
:100C0000B2FA82F2002A40F09280A1EB0C014FEA86
:100C10001C471FFA8CFE0126200CB1FBF7F307FBE3
:100C2000131140EA01410EFB03F0884208D91CEB86
:100C3000010103F1FF3802D2884200F2CB80434623
:100C4000091AA4B2B1FBF7F007FB101144EA014402
:100C50000EFB00FEA64508D91CEB040400F1FF3191
:100C600002D2A64500F2BB800846A4EB0E0440EA7F
:100C700003409CE7C6F12007B34022FA07FC4CEA88
:100C8000030C20FA07F401FA06F31C43F9404FEA7B
:100C90001C4900FA06F3B1FBF9F8200C1FFA8CFE90
:100CA00009FB181140EA014108FB0EF0884202FAE4
:100CB00006F20BD91CEB010108F1FF3A80F08880A5
:100CC000884240F28580A8F102086144091AA4B262
:100CD000B1FBF9F009FB101144EA014100FB0EFEE3
:100CE0008E4508D91CEB010100F1FF346CD28E4512
:100CF0006AD90238614440EA0840A0FB0294A1EBA3
:100D00000E01A142C846A64656D353D05DB1B3EBFF
:100D1000080261EB0E0101FA07F722FA06F3F1402F
:100D20001F43C5E9007100263146BDE8F087C2F1D6
:100D30002003D8400CFA02FC21FA03F3914001434E
:100D40004FEA1C471FFA8CFEB3FBF7F007FB103687
:100D50000B0C43EA064300FB0EF69E4204FA02F433
:100D600008D91CEB030300F1FF382FD29E422DD986
:100D7000023863449B1B89B2B3FBF7F607FB1633BB
:100D800041EA034106FB0EF38B4208D91CEB01013B
:100D900006F1FF3816D28B4214D9023E6144C91ABB
:100DA00046EA004638E72E46284605E70646E3E6CB
:100DB0001846F8E64B45A9D2B9EB020864EB0C0ED5
:100DC0000138A3E74646EAE7204694E74046D1E7E4
:100DD000D0467BE7023B614432E7304609E7644492
:100DE000023842E7704700BF02E000F000F8FEE77B
:100DF00072B6374880F30888364880F30988364849
:100E00003649086040F20000CCF200004EF6347122
:100E1000CEF200010860BFF34F8FBFF36F8F40F237
:100E20000000C0F2F0004EF68851CEF200010860DA
:100E3000BFF34F8FBFF36F8F4FF00000E1EE100A4A
:100E40004EF63C71CEF200010860062080F3148853
:100E5000BFF36F8F78F1C0F876F158FD4FF0553041
:100E60001F491B4A91423CBF41F8040BFAE71D4958
:100E7000184A91423CBF41F8040BFAE71A491B4A51
:100E80001B4B9A423EBF51F8040B42F8040BF8E7A3
:100E900000201849184A91423CBF41F8040BFAE778
:100EA00078F1DCF876F172FE144C154DAC4203DAA1
:100EB00054F8041B8847F9E703F040FE114C124D2B
:100EC000AC4203DA54F8041B8847F9E778F1C4B858
:100ED00000060024002200240000020808ED00E0C3
:100EE000000000240006002418671F0800220024C8
:100EF000C0310024C0310024CC640224E002020886
:100F00007C0302087C0302087C0302082DE9F04FF1
:100F10002DED108AC1F80CD0D0F80CD0BDEC108AA1
:100F2000BDE8F08F002383F311882846A0470020F6
:100F300076F11AFAFEE776F109F800DFFEE7000025
:100F400070B54FF0FF0C4CF4E06C1CEA11541DBF5F
:100F50001CEA135594EA0C0F95EA0C0F00F0DEF82A
:100F60002C4481EA030621EA4C5123EA4C5350EA0F
:100F7000013518BF52EA033541F4801143F4801360
:100F800038D0A0FB02CE4FF00005E1FB02E506F0F1
:100F90000042E0FB03E54FF00006E1FB03569CF046
:100FA000000F18BF4EF0010EA4F1FF04B6F5007F4C
:100FB00064F5407404D25FEA4E0E6D4146EB0606BE
:100FC00042EAC62141EA55514FEAC52040EA5E5047
:100FD0004FEACE2EB4F1FD0C88BFBCF5E06F1ED8F1
:100FE000BEF1004F08BF5FEA500E50F1000041EB28
:100FF000045170BD06F0004646EA010140EA0200D5
:1010000081EA0301B4EB5C04C2BFD4EB0C0541EAF6
:10101000045170BD41F480114FF0000E013C00F30B
:10102000AB8014F1360FDEBF002001F0004170BD2F
:10103000C4F10004203C35DA0C341BDC04F1140448
:10104000C4F1200500FA05F320FA04F001FA05F2D4
:1010500040EA020001F0004221F0004110EBD370A1
:1010600021FA04F642EB06015EEA430E08BF20EACD
:10107000D37070BDC4F10C04C4F1200500FA04F370
:1010800020FA05F001FA04F240EA020001F0004102
:1010900010EBD37041F100015EEA430E08BF20EA75
:1010A000D37070BDC4F1200500FA05F24EEA020EBD
:1010B00020FA04F301FA05F243EA020321FA04F0EC
:1010C00001F0004121FA04F220EA020000EBD370A3
:1010D0005EEA430E08BF20EAD37070BD94F0000FA3
:1010E0000FD101F00046400041EB010111F4801FD7
:1010F00008BF013CF7D041EA060195F0000F18BF88
:10110000704703F00046520043EB030313F4801FC3
:1011100008BF013DF7D043EA0603704794EA0C0F7D
:101120000CEA135518BF95EA0C0F0CD050EA410693
:1011300018BF52EA4306D1D181EA030101F0004110
:101140004FF0000070BD50EA410606BF1046194638
:1011500052EA430619D094EA0C0F02D150EA013644
:1011600013D195EA0C0F05D152EA03361CBF104685
:1011700019460AD181EA030101F0004141F0FE4124
:1011800041F470014FF0000070BD41F0FE4141F4A8
:10119000780170BD4FEA410212F5001215D211D547
:1011A0006FF47873B3EB625212D94FEAC12343F064
:1011B000004343EA505311F0004F23FA02F018BFE6
:1011C000404270474FF00000704750EA013005D1AF
:1011D00011F0004008BF6FF0004070474FF0000072
:1011E000704700BF4FEA4102B2F1E04324BFB3F5BC
:1011F000001CDCF1FE5C0DD901F0004C4FEAC0028E
:101200004CEA5070B2F1004F40EB830008BF20F071
:101210000100704711F0804F21D113F13872BCBF2B
:1012200001F00040704741F480114FEA5252C2F180
:101230001802C2F1200C10FA0CF320FA02F018BFC9
:1012400040F001004FEAC1234FEAD32303FA0CFC1C
:1012500040EA0C0023FA02F34FEA4303CCE77FEAAB
:10126000625307D150EA01331EBF4FF0FE4040F4F5
:101270004000704701F0004040F0FE4040F40000A4
:10128000704700BF01F0FF01102A2BDB10F0070FA1
:1012900008D010F8013B013A8B422DD010F0070F17
:1012A00042B3F6D1F0B441EA012141EA014122F012
:1012B00007047FF000070023F0E80256083C85EAA7
:1012C000010586EA010685FA47F5A3FA87F586FA4D
:1012D00047F6A5FA87F68EB9EED1F0BC01F0FF0112
:1012E00002F0070232B110F8013B013A83EA010330
:1012F00013B1F8D10020704701387047002D06BFA8
:1013000035460338073815F0010F07D1013015F4C1
:10131000807F02BF013015F4C03F0130F0BC0138BE
:10132000704700BFEC46A0E8F05F4FF00000704748
:10133000B0E8F05FE546080008BF0120704700BF35
:1013400010F8012B11F8013B012A28BF9A42F7D06F
:10135000D01A7047034613F8012B002AFBD1181A44
:1013600001387047A8B110B504460AE000F096FABB
:1013700014F8041C54E903031B1AB3FBF1F200F048
:101380008DFA204654F80C3B082201210133EDD19F
:1013900010BD70472DE9F04F0023A7B00293C36A38
:1013A000009013F0040FD0E9002118BF0A46D906B7
:1013B0004FF0E021D3694CBF02F1200002F1680038
:1013C0000192DB0903F0040303430393D1F8883D42
:1013D00003F4A003B3F5A00F01D101230293936995
:1013E0004FF004094F4D4FF001081B884E4C03F499
:1013F0007F43A3F53E43B3FA83F35B09049329E0EB
:1014000000F040F9FFF7AEFF4FF0E023D3F8003DC6
:1014100003F47023B3F5402F0ED0444A4FF0FF334E
:1014200005A88DF81C90059214328DF8288006923C
:10143000CDE90833FFF796FF2B68A34206D03C4B5B
:101440000422012105A8059300F028FA00F070FBA2
:1014500000285ED103A82C6000F00CFC04220121BE
:10146000344800F01BFA0422012102A800F016FA09
:1014700010220121019800F011FA00982022012188
:101480000C3000F00BFA019804220121103000F01A
:1014900005FA0422012103A800F000FA01980C22A9
:1014A0000121143000F0FAF90C220121009800F01B
:1014B000F5F9029BDA07A3D5009BDB6ADB0622D491
:1014C00015A80DF1140AFEF775FFDDF804E0D44607
:1014D0000EF120060EF1600B3068103656F80C1C29
:1014E000674656F8082C0CF1100C56F8043C5E4583
:1014F0000FC7F1D1DEF860302593842250460121D8
:1015000000F0CCF97CE70DF1140A5046FEF74CFFD1
:10151000F3E7049B1BB1019A93690233936127B0EF
:10152000BDE8F08FC0310024ED55CEAC28ED00E0D1
:10153000ACCE55EDEC351A0838B535206D2573F174
:10154000C5FC144B144A4FF0FF34D3F890100D2013
:1015500041F48011C3F89010D3F8901021F4801159
:10156000C3F89010D3F89010D3F8E81041F480112C
:10157000C3F8E810D3F8101141F48011C3F810112A
:101580000121D3F81031054BD56014621060197039
:1015900038BD00BF0044025800500040EC33002426
:1015A000002953D02DE9F84F074689460026284DDB
:1015B000DFF8A480274C17F801AB2B784FEA1A12FA
:1015C00018F802B0002B3CD0C4F828B0E3695806E4
:1015D00004D477F1C7FCE3695906FAD50AF00F0A7B
:1015E0002B7818F80AA04BB3C4F828A0E3695A0670
:1015F00004D477F1B7FCE3695B06FAD50136B1454F
:1016000022D03107D7D12B784FF00D0BDFF84CA04B
:101610008BB1C4F828B0E3695A0604D477F1A2FC70
:10162000E3695B06FAD51AF801BFBBF1000FC2D01F
:101630002B78002BEDD1FFF77FFFEAE7FFF77CFF68
:10164000D2E7FFF779FFBFE7BDE8F88F704700BF2B
:10165000EC3300240050004074361A087C701B08DC
:10166000014B1868704700BFFCFF1F08014B024880
:10167000C01A7047E0761F08000020080048704735
:10168000E0761F08774943F69822774B09682DE9E1
:10169000F04F0A441B7883B0744F02EB030975F1D5
:1016A00053FB734B0446002800F0C8800225FF1A44
:1016B000DFF8E0810126DFF8CCB130E01846019177
:1016C00076F1CCFF0199002836D1206AAA460AF1AA
:1016D00001030AEB4A0E04F13C058944DBB20144E4
:1016E0000BEB8E0CB94503EB43034BF82E40CCF8C3
:1016F00004500AF102058CF808600BEB830CEDB284
:101700004BF823008CF80860CCF8041023D2204654
:1017100075F12AFB0446002835D04E2D33D8206AB7
:10172000404505D0211AE369002BC7D1AA46CEE770
:10173000504BA3EB0801F6E705EB450C01350BEB2D
:101740008C005FFA85FA0672E3694BF82C300D3392
:101750004360206ABBE74F2D63D94FF0FF3301226E
:10176000CBF8B4338BF8BC23CBF8B833424B1B789F
:101770002BB1424A424B12681B68CBE90023414817
:1017800003B0BDE8F08FB7EB0900E4D44E2DE2D8EA
:101790000AF1030A3C4EDFF800C15FFA8AFAA6EBB1
:1017A0000C03BAF14E0F514694BF0024012483422A
:1017B0002BDC05EB450503EB090201200BEB850350
:1017C0004BF825C05E601872BA1A12D48CB92F4833
:1017D00001EB41052E4BC41A944224DD1A440AF150
:1017E00001014BF825300BEB8503C9B25A60012289
:1017F0001A7201EB41054FF0FF3201210BEB85031B
:101800004BF8252019725A60B0E705EB4505012217
:1018100060440BEB85034BF825C01A723A465860BA
:10182000D2E72946E5E70AF1010101224BF825300C
:101830000BEB8503C9B258601A72DAE7FF1AB7EBEF
:1018400009000BD4104E4FF0030ADFF84CC00225FC
:10185000DFF830B05146A6EB0C03A8E70221DFF811
:1018600024B0C6E7DC330024B43300240000200891
:10187000E0761F080022002400220024E033002428
:10188000D833002404220024CC640224000008245D
:10189000D064022400060024C03100249A4B1B7837
:1018A0002DE9F04F824685B00E4693462BB9974BF3
:1018B0001B782BBB05B0BDE8F08F022900F0EE804D
:1018C000042900F0B580012900F0AE80904D2B78FE
:1018D0000D27DFF858828F4C7BB1A762E3695A0667
:1018E00004D477F13FFBE3695B06FAD518F8017F72
:1018F000002FDCD02B78002BEFD1FFF71DFEECE79B
:10190000854B4FF00009854A9B1A0093CB45D1D0F7
:10191000834F844C38682578031D009A2B449342EA
:1019200079D2202D51D0022E24D0042E0DD0012E9C
:10193000ECD12378DFF8F0815A1C22701AF80920C4
:1019400009F1010908F80320E0E7DFF8DC81002550
:10195000434620789AF80010421CE9400835D2B27C
:1019600008F80010202A227018D0202DF1D109F19A
:101970000109CBE725789AF80030DFF8AC8108F848
:1019800005300135EDB2202D257030D06B1C09F1EA
:1019900001092370002308F80530B7E738685F496C
:1019A00001920844194676F1E1FB39684FF00003D3
:1019B000019A203123705C4B3960002118467CF17C
:1019C000DBFF77F1CFFA584BCFE7544B2A46564905
:1019D000184476F1CBFB3B6800212A46203352485D
:1019E00021703B607CF1C8FF77F1BCFA9BE74B4B61
:1019F0002A4638684146184476F1B8FB3B68002116
:101A00002A462033404621703B607CF1B5FF77F1D8
:101A1000A9FA2578BAE7444A4FF0FF312023D16173
:101A2000237005B0BDE8F08F1146FFF7B9FD4DE713
:101A3000002A3FF44BAF02460027354D0DF10C084C
:101A400052F8043B334C0092039301910137042177
:101A50004046FFF7A5FDBB451ED0009ABE0752F8D1
:101A6000043B00920393F1D12A780D26DFF8BC9055
:101A70007AB1A662E369580604D477F173FAE36990
:101A80005906FAD519F8016F002EDFD02A78002AFE
:101A9000EFD1FFF751FDECE7019E18E7002A3FF474
:101AA00015AF024600271A4D0DF10C0832F8023B23
:101AB000184C0092ADF80C300191013702214046DC
:101AC000FFF76EFDBB45E7D0009A790732F8023B7D
:101AD0000092ADF80C30F0D12A780D26DFF84C904A
:101AE0007AB1A662E3695A0604D477F13BFAE36956
:101AF0005B06FAD519F8016F002EDED02A78002A8D
:101B0000EFD1FFF719FDECE7B533002400220024E4
:101B1000EC3300240050004000002008E0761F084D
:101B2000DC330024B4330024B83300247C701B0859
:101B3000F8B5324B1A782AB9314A1078F0B9012237
:101B40001A70F8BD2F4E0D252F4F304C3B7893B1B6
:101B5000A562E3695A0604D477F104FAE3695B06E7
:101B6000FAD516F8015F002DF0D1294B58680038DE
:101B700018BF0120F8BDFFF7DFFCE9E7254D264E31
:101B80002B68264C26481A1D3178241A0A44A24292
:101B900006D239BB9C421CD8002076F19DFBE4E7BD
:101BA000204A4FF0FF31D1612022327018442022A8
:101BB0001C4976F1DBFA2A6833780021194813446E
:101BC000202231702B607CF1D7FE77F1CBF92B68A6
:101BD000E0E7144920221448CB6176F1C7FA77F187
:101BE000C1F9D9E703F120029442DFD81F29DDD8DB
:101BF0000C4AD36120223270D8E700BFB5330024ED
:101C000000220024F0351A08EC3300240050004074
:101C1000E4330024DC330024B43300240000200823
:101C2000E0761F08B8330024E0FF1F080E4B1B7836
:101C300010B5B3B1642100200C4A0D4CD3699B064A
:101C4000FCD5536ADBB28B424FF0640101D0002017
:101C5000F4E70130C0B20E2801D0015DEEE70020AC
:101C600010BDFFF769FCE5E7EC33002400500040AD
:101C700000361A082DE9F04102680646EFF30581A7
:101C8000D9205369C9B202F123FD674B1B782BB9E8
:101C9000664C2378002B37D1BDE8F081644B0D27CB
:101CA000DFF8B081634D644C96E8030083E80300DD
:101CB0002B7833B3A762E3695F0604D477F152F956
:101CC000E3695806FAD518F8017F002FF0D1736840
:101CD0000BB32B784227DFF88081574C73B1A76292
:101CE000E369590604D477F13DF9E3695A06FAD558
:101CF00018F8017F1FB32B78002BF0D1FFF71CFCE5
:101D0000EDE7FFF719FCD5E73568002D47D1002333
:101D10002370BDE8F081DFF844814327464C2B78DF
:101D2000002B6AD0A762E3695B0604D477F11AF945
:101D3000E3695F06FAD518F8017F002FEFD1DFF8CD
:101D4000208120273C4C2B78002B53D0A762E369DD
:101D5000580604D477F106F9E3695906FAD518F85C
:101D6000017F002FEFD1FFF761FF2B78DFF8F480C0
:101D70000D27314C83B1A762E3695A0604D477F189
:101D8000F1F8E3695B06FAD518F8017F002F3FF4FC
:101D90007FAF2B78002BEED1FFF7CEFBEBE7284689
:101DA00076F15CFC0028B2D0284676F17FFC00F288
:101DB0001450854231D3214BA5F214521A602846A3
:101DC00076F18AFC05F5E053834220D81C4A136063
:101DD00000231C481C4A03601C481D49801A0B70D4
:101DE00002D10DE083420BD252F8041B04330131BF
:101DF000F8D08CE7FFF7A0FBA8E7FFF79DFB91E782
:101E000077F1B0F80120BDE8F04176F165BA2846D7
:101E100076F162FC0A4B1860DAE7284676F146FC58
:101E2000064B1860CBE700BFB53300240022002426
:101E3000E4330024EC33002400500040E03300245D
:101E4000D8330024DC330024E0761F08000020088B
:101E5000B433002410361A0818361A086C361A08DB
:101E600024361A087C701B08002070470368002283
:101E70001B681847F0B50D4683B040210646E4F0D4
:101E80003FFC18B1154F97F95A371BB9012420466A
:101E900003B0F0BD92F06CFF437A93B1104BB7F9E9
:101EA0005C27D3F89434B3F906309A42EEDD0D493D
:101EB0002A460D4B3046009140210024E4F028FCD6
:101EC000E5E792F055FF847A002CE7D1074B2A46CC
:101ED00040213046E4F01CFCD9E700BFF073002439
:101EE000F0930024AC361A0898361A0888361A0877
:101EF0002DE9F0410D469CB020210446E4F000FCA1
:101F0000002865D0694E96F95A37002B64D196F9AE
:101F10004937022B00F08880B6F81C3741F658325A
:101F2000A3F57A739BB2934277D8DFF8C88106F5A0
:101F3000F162D8F85C3492ED007AD3ED097AB4EE10
:101F4000E77AF1EE10FA61DCD3ED0B7A06F28C73CE
:101F500093ED007AB4EEE77AF1EE10FA56DCB6F9BA
:101F60005637002B40F39680A8F5405393F844224F
:101F70000D2A04D80123934013F4215F5BD14C4810
:101F800013F0BCFE01285DD04A4F97F8251911F0D7
:101F9000100178D1602204A803917CF1EDFC642348
:101FA00003AA4549D8F86404F0F082FE38B16423EE
:101FB000D8F85C0403AA4149EEF0F2F948B920468A
:101FC00003AC3F4B2A4620210094E4F0A1FB19E02A
:101FD00001201CB0BDE8F08106F50057B6F95C376A
:101FE000D7F89424B2F90A1003F10A02914203DDF2
:101FF00040F28D3293428ADC324B2A462021204621
:10200000E4F086FB00201CB0BDE8F0812E4B2A4690
:1020100020212046E4F07CFBF4E72C4B2A462021CB
:102020002046E4F075FBEDE7294B2A4620212046A7
:10203000E4F06EFB70E7274B2A4620212046E4F0AF
:1020400067FBDFE7D8F86804F3F0B6F848B3012877
:10205000184F9AD197F8A8342BB319211E4877F05E
:10206000F1FA00B3D6F8346719211B4877F020FB4A
:1020700086428ADD194E1A4B2A46202120460096B8
:10208000E4F046FBBEE7174B2A4620212046E4F049
:102090003FFBB7E7144B2A4620212046E4F038FBEB
:1020A000B0E7124EE7E7124EE5E700BFF0730024F9
:1020B000C0CD0024F0930024D0371A08E8371A085E
:1020C000D4371A08B8361A0804371A08F4361A082A
:1020D000CC361A0838371A08D84B0024A0371A080B
:1020E00058371A08B8371A0820371A0880371A08DC
:1020F00090371A08F0B3002470B500249AB060221B
:102100000E460546214602A801947CF135FC642266
:1021100001A90D48BEF088FF044640B99DF904307E
:1021200043B90A4B31460A4A2846E4F057FF204695
:102130001AB070BD284601AB054A3146E4F04EFFA7
:1021400020461AB070BD00BFEC950024EC371A0889
:102150005C011E082DE9F043DFF88491A5B0074625
:102160008846D9F80C391A68184613699847054605
:102170001CF090FF0021064660220CA80B917CF118
:10218000FBFB64230BAA294630461CF0F7F80446F3
:1021900098B34848BCF04EFB9DB997F91E30012B0F
:1021A0000FD010F0060F24D0A9F5C04018F010FA97
:1021B000034660B9404A414638461C46E4F00EFFEB
:1021C00017E03E4818F004FA0346002852D003A94D
:1021D00030461BF071FC18B19DF80D305B0650D4F1
:1021E000374D0023D5ED007AF5EEC07AF1EE10FA06
:1021F0000DDC204625B0BDE8F08338460BAB314AF4
:102200004146E4F0EBFE204625B0BDE8F0833046C1
:10221000089308AE09930A9307AB05AA04A9019392
:1022200006AB00961CF078FB30464AF045F8D5ED39
:10223000007AB4EEE70AF1EE10FA29DA9DED057A9C
:10224000F4EEC77AF1EE10FA28D99DED047AF4EE97
:10225000C77AF1EE10FA27D99DED067AF4EEC77A27
:10226000F1EE10FAC5D8184A41463846E4F0B6FEF9
:102270000024BEE7154A414638461C46E4F0AEFE4F
:10228000B7E7134A414638460024E4F0A7FEB0E71A
:10229000104A41463846E4F0A1FEE9E70E4A4146BD
:1022A0003846E4F09BFEE3E70C4A41463846E4F04A
:1022B00095FEDDE7BC75002428381A08F0330024A9
:1022C000687B002404381A08A8381A0810381A083D
:1022D00050381A0860381A0878381A0890381A08DE
:1022E000F093002470B50D469AB020210646E4F024
:1022F00007FA18B9012420461AB070BDFBF0ECFAB9
:1023000004460028F6D00021602202A801917CF149
:1023100033FB2046642201A9FBF0A6FA04460028FC
:10232000E8D101AB024A29463046E4F057FEE2E725
:102330005C011E0870B50D4C05460E46D4F80C39EC
:102340001A6818465369984710B10124204670BD99
:10235000A4F5C04018F050F904460028F5D1044A0D
:1023600031462846E4F03AFEF0E700BFF09300243F
:10237000CC381A08F0B583B007460E46E4F0FCF9F5
:10238000044610B9204603B0F0BD02213846E4F0FF
:10239000B7F905460028F5D01548F4F0DFFDC20571
:1023A000C0F30723C0F3002401D49B0703D42C46B9
:1023B000204603B0F0BD0E48F4F0DEFD0D4B9FED5E
:1023C0000E7A03F20C43D3ED007AF8EEE77A30EEA2
:1023D000670AF0EEC07AF4EEC77AF1EE10FAE6DDA5
:1023E000064B324602213846E4F092F9CAE700BFB4
:1023F00030B80024F0B300240000C842E0381A08C6
:1024000070B5054682B00E46E5F04AF81021044644
:102410002846E4F075F910B9204602B070BD0848AE
:10242000F4F09CFD10F00100F6D10446054B28465F
:1024300032461021E4F06CF9204602B070BD00BFB6
:1024400030B80024F4381A0870B506460D46E4F09A
:10245000BDFD044608B9204670BD80213046E4F039
:102460004FF90028F7D0074B93F8F13E13B9044613
:10247000204670BD044B2A46802130460024E4F0FB
:1024800047F9E8E7F093002408391A0838B50D4DEC
:102490000446D5F86804F2F08FFE012810D0D5F874
:1024A0006804F2F089FE022804D02046BDE83840D6
:1024B000E4F0A8B8044813F021FC0128F5D138BD98
:1024C000002038BDF0B30024C0CD0024F0B5114C7D
:1024D00085B00F460646D4F88C346A460093D4F88B
:1024E00090340193D4F894340293D4F8983403933D
:1024F000E5F0A8FD054639463046E4F0E3FA94F8E5
:102500000039284060F3C303C3F3C00084F80039E6
:1025100005B0F0BDF0930024F8B5264F04462648D8
:102520000D46BCF087F9D7F80C3906461A681846EC
:102530001369984716F0060F0ED168B9D7F84039DD
:10254000022B09D029462046FFF704FE68B3012379
:102550001A4A1846D371F8BD29462046E4F0DCFB40
:1025600018B329462046FFF7F5FDF0B108212046B3
:10257000E4F0C6F80028EAD0114830F0A5FC0028A5
:10258000E5D0104BB02193F8642601FB023203F52D
:102590008043B2F86E24B3F94A379A42D7DD0A4B2A
:1025A0002A4608212046E4F0B3F80023034A1846DF
:1025B000D371F8BDF0930024BC75002458D50024D5
:1025C00048370024F03300241C391A0870B588B04D
:1025D00006460D46E4F02CFD044610B9204608B02E
:1025E00070BD20213046E4F08BF80028F6D0194B5E
:1025F00093F8A425002AF1D093F880359B07EDD5F8
:1026000007AA06A91448B7F0E1F90028E6D09DED25
:10261000077ADFED127AB4EEE77AF1EE10FADDD840
:10262000DDED066AB7EEC77A2A463046FDEEE66A69
:102630000B4B202100249FED055BCDED006A8DED55
:10264000045B8DED027BE4F063F8C7E70000004017
:102650003333E33FF0B300248C7C00249A99193F74
:102660002C391A082DE9F04182B00D4606461CF0BF
:1026700011FD07461BF0B8F988B338461CF070FC12
:1026800078B1DFF8C8812946D8F80C0903689B693E
:1026900098470446A0B1B3685BBB204602B0BDE8D2
:1026A000F08127F00BFB90F8461327F03DFA044623
:1026B0000028E6D1584A01213046E4F08FFCECE7CF
:1026C000D8F80C0903681B6C9847544A034601214B
:1026D0003046E4F083FC204602B0BDE8F0810446B9
:1026E0004F4A30460121E4F079FC204602B0BDE8B3
:1026F000F08110213046E4F003F8E0B1D7ED937A91
:1027000097ED920A20EE270A79F1F0F9A8F5005327
:10271000DFED447AB3F91C3720EE270A9FED427AA9
:1027200007EE903A20EE070AF8EEE77AB4EEE70AF1
:10273000F1EE10FA67DC20213046E3F0E1FF18B13A
:1027400098F82539DB0656D440213046E3F0D8FF0F
:1027500058B1232D18BF012D01D0042D14D1D8F864
:102760000C090368DB6B984770B1304B304A1B682B
:10277000D86A0368DB69934233D12946304602B0F8
:10278000BDE8F041E4F054B9D8F894342948B3F9DD
:10279000083000EE103AB8EEC00A00F0AFFCB5EE1B
:1027A000C00AF1EE10FA12DCD8F80C0903685B6974
:1027B000984730B9D8F80C0903681B6898470B286C
:1027C000D3D1D8F89434B3F90830002BCDDD1A4CAE
:1027D00001221A4B4021009430460024E3F098FF78
:1027E0005BE7984701280146C7D1154A30460024C7
:1027F000E4F0F4FB51E7134B012220213046002482
:10280000E3F086FF49E7104B0122102130460024F7
:10281000E3F07EFF41E700BF6C391A0880391A08DF
:1028200058391A08E02E65420000C84250D20024F0
:10283000691E0208F0330024AC361A089C391A08C5
:10284000A8391A08B8371A0894391A08F0930024DE
:1028500070B50E460546FFF77DFC084B0446314631
:10286000D8712846FFF766FD034631462846002BFF
:1028700008BF0024E4F02CFD204070BD58D5002492
:102880002DE9F0439BB00D46044692F071FA2021E9
:1028900093F0E8FC002839D092F06AFA1F2193F0F7
:1028A000E1FC60B3594F2946594A2046E4F096FBB3
:1028B00097F80239002603F01403142B2ED1294671
:1028C0002046544A0026E4F089FB29462046E5F0DC
:1028D00045FD48BB01466022019002A87CF14CF8FE
:1028E000D7F830090DF104086421036842461B68DB
:1028F000984700284BD000201BB0BDE8F08392F031
:1029000037FAA52193F0AEFC0028CBD13F4F01262A
:1029100097F8023903F01403142BD0D0294620462F
:10292000E5F01CFD0028D5D04FF00009602202A878
:102930000DF104084946CDF804907CF11DF8D7F854
:1029400030096421424603681B689847F8B1002E9D
:10295000D1D0A3682BBB236829462F4A20469B6B06
:1029600093424AD1FFF7F6FB2C4B06462946D87115
:102970002046FFF7DFFC034629462046002B08BF10
:102980000026E4F0A5FC30401BB0BDE8F0832046F3
:102990004346234A2946E4F021FB00201BB0BDE852
:1029A000F08329462046FFF7A3FA2946064620462B
:1029B000FFF7A2FB97F8253906409B07F6B21ED415
:1029C00029462046FFF78EFC064029462046FFF7A1
:1029D00051FA064029462046FFF7ACFC294606403E
:1029E0002046E4F09BFC0346294620461E40E5F0C5
:1029F00097FB30401BB0BDE8F0839847C4E7094A15
:102A0000294620464E46E4F0E9FAD9E7F09300243F
:102A1000B8391A08D4391A085128020858D50024A0
:102A2000EC391A08BC381A08F8B5124DD5F8303907
:102A300093F8D54074B9104B07460E461B68986A48
:102A400003685B6B9847044670B131463846FFF720
:102A500017FF044695F800392046084A64F304132A
:102A6000947185F80039F8BD054A31463846E4F0DE
:102A7000B5FAEFE7F093002450D2002458D5002493
:102A8000F8391A082DE9F041554E3378C3B9554F3E
:102A90000124D7F83059347095F8D5501DB1284627
:102AA0003370BDE8F081E5F033FD054660B94E4A6C
:102AB00030702846137843F001031370BDE8F081AD
:102AC00000252846BDE8F08182F068FF214681F0AC
:102AD00021FEA7F5C04008F05BFC444B1C710B24A1
:102AE0006DF01CFA6DF01EF9611E11F0FF04F7D1B4
:102AF0003F4801F0DFFB1CF0CDFAD0F80022C7F808
:102B0000582990F87C32DA074DD59B0757D500211C
:102B1000374801F05BFC364817F05AFD014635484E
:102B2000FAF0C0FA344B354C01211B68D86A0368AF
:102B30001B68984794F8E035D7F830096FF34103E4
:102B400084F8E03503689B6A98470121D7F830097B
:102B5000F5F086FF82F022FF8046D7F80C09036863
:102B60001B689847A4F580430146404693F83025FA
:102B700081F0CCFFA4F5004008F0FCFB7DF000FCE8
:102B80007CF078FF0023337001F118FEB7F80239AA
:102B9000C4F87404284623F4087343F02003A7F80C
:102BA0000239BDE8F0811BF0B1FC82F0F7FE3C2158
:102BB00082F0E4FB07F6181300221A60A7E721460B
:102BC0000B4806F0E5FA0E48F4F0D6F9DFED0D7A81
:102BD00007F6181320EE270A83ED000A97E700BFD7
:102BE000ED330024F093002478D5002458D5002438
:102BF000F03300247C94002450D20024F0B300244D
:102C000030B800240AD7233C2DE9F0433E4D87B06D
:102C1000D5F8303993F8D530002B55D01AB1232987
:102C200048D0012946D0E5F0FBFC044620B9002439
:102C3000204607B0BDE8F0831CF02CFA064627F0CA
:102C40003DF8804630461AF0FDFC18B198F928305E
:102C5000022B3ED001212D4808F030FE01212B48E7
:102C600008F05AFD0021D5F83009F5F0F9FE2848A2
:102C70004AF026F882F092FE002181F04BFD254BB0
:102C800000211B68D86A03681B689847D5F80C199F
:102C9000214895F80239091A3C306FF34513B1FA0F
:102CA00081F185F802394909FEF00AFC204607B097
:102CB000BDE8F08395F90039002BB8DAE5F0B0FCF7
:102CC00004460028B3D0B7E70124204607B0BDE88A
:102CD000F08300274FF00009F9B203AA3046CDF87F
:102CE0000C9001910137CDF81090CDF814901BF0A5
:102CF0008FF9019910B9032FEED1ABE703AA404633
:102D000026F014FAF7E700BFF0930024F033002414
:102D10003CC6002450D2002444C9002470B52A4E79
:102D20000D46D6F80C092DED028B036888B0B0EE85
:102D3000408A5B6A9847044600283CD0D6F8303970
:102D400093F8D540BCB3B4EE488AF1EE10FA37D60A
:102D5000DFED1E8ADFED1E7A68EE288A68EEA78A0C
:102D6000D5ED027A02A82A68F1EE677A6B689FEDCA
:102D7000180A02920393CDED047A48F0F9FDB4EEFF
:102D8000488A0022B0EE407A0123F0EE607A9FED8F
:102D9000110AF1EE10FA05A9F0EE680A0E488DED61
:102DA000057ACDED067A8DED071ACDE9002368BFCF
:102DB000134610F005FF204608B0BDEC028B70BD35
:102DC000DFED048ACCE700BFF0930024E02E6542DB
:102DD0000000C8420000000060CC002438B50B4D54
:102DE0000C46D5F80C0903685B6A984758B1D5F8CA
:102DF000303993F8D53033B12146A5F5C040BDE850
:102E0000384000F0FBBB002038BD00BFF093002429
:102E10000148BBF0CBBE00BFBC75002400F5C0402C
:102E200008B590F80039C3F340128A4204D061F328
:102E3000451380F8003901B908BD82F0AFFD0F21BC
:102E4000BDE8084082F09ABA70B500F5C046D6F8E1
:102E500040398B4208D0012905460C4626D002296C
:102E600012D011B1C6F8404970BD82F097FD1B2108
:102E700082F084FA46F29860144A0621284486F0CB
:102E8000DFFCC6F84049EFE7012101F09FFA82F02C
:102E900085FD1D2182F072FA46F298600C4A0621E7
:102EA000284486F0CDFCC6F84049DDE782F076FD87
:102EB0001A2182F063FA46F29860064A06212844F5
:102EC00086F0BEFCC6F84049CEE700BF703A1A084B
:102ED000903A1A08803A1A0800F5C04210B592F8E4
:102EE00025390C4603F00101A14209D064F3000327
:102EF00082F82539DB0704D507F07EFF024B9C7270
:102F000010BD07F0B5FDF9E758D5002400F5C04025
:102F1000044A90F82539117361F3410380F825398B
:102F2000704700BF58D5002410B5044691F020FF2B
:102F3000202193F097F904F5C043003893F8022953
:102F400018BF012060F3820283F8022910BD00BF80
:102F5000704700BF9FED010A704700BF00000000EE
:102F60000346B6EE061AF4EE000A302093ED4B0A43
:102F700042F0D0BC10B504467DF002FA436F04F570
:102F8000C04204F50044D2F83029D360D4F85C2460
:102F90009366D4F86424C2F80833D4F85C04036858
:102FA0005B6D9847D4F85C04044A03689B6D9342B8
:102FB00000D110BDBDE81040184700BF512F0208D6
:102FC00070B500F5C0452DED028BD5F8303993F87A
:102FD000D530002B3AD095F90039002B36DB00F5BF
:102FE0001043044693F8703183BBD5F80C0903688D
:102FF0005B69984750BB3A4BD3F80C0903681B68D0
:1030000098470B2822D004F500469FED367AD6F873
:103010006434D3EDE47AF0EEE77AF4EEC77AF1EEB9
:1030200010FA13D5D5F83009443085F063FD034616
:10303000B7EE001A9F20DFED2C0A93ED000A42F054
:1030400069FCB5EEC00AF1EE10FA02DCBDEC028BB1
:1030500070BD48F240402044F3F09AFFB0EEC00A41
:10306000DFED227AB4EEE70AF1EE10FAEED5D6F8EB
:103070005C0404F500561E4AD6F8783607EE903AFE
:103080000368D3F89830B8EEE78A934224D1B0EEC3
:10309000C88ADFED187AB4EEE78AF1EE10FAD5D5DA
:1030A000D6F87C3640F2E63203F2F3139342CDD8E1
:1030B000D5F830099FED100AF7F082FBD5F83039CA
:1030C00004F5E6509FED0C0AD3ED0C0ABDEC028B23
:1030D000BDE87040D1F06ABC984738EE408AD6E728
:1030E000F093002400000034000000000000704253
:1030F000552F02080000FA430AD7233CF8B500F523
:10310000C0462DED028B96F8251911F0010504D06B
:103110009FED360ABDEC028BF8BDB0EE408A044646
:1031200091F026FE037F002BF2D0DFED318A04F50B
:103130008047DFED2E0AB0EE480AB0EE681A4E2046
:1031400042F0E8FB29464FF4C872B7F95E07B0EECB
:10315000408A42F04BFC03462046A7F85E3716F043
:10316000AFFFB7F95E3707EE100A07EE903AB8EEF8
:10317000C77AF8EEE77A77EE676AB4EEE68AF1EEA0
:1031800010FA15D5B6F9583143BBB7F95637002BAD
:10319000B8BF5B429BB207EE903AF8EEE77A38EEA2
:1031A000668A27EE888A88EE260ABDEC028BF8BD77
:1031B00077EE877AB4EEE78AF1EE10FAA8DDB7F978
:1031C000563738EE678A78EEE77A07EE103AB8EEAF
:1031D000C77A27EE088A88EE270A9BE7002BB8BF3C
:1031E0005B429BB207EE903AD7E700BF00000000B9
:1031F00000007A4400F5C0400F4908B5D0F83039D6
:103200001A6812698A4214D1B6EE061A3020F4EE1A
:10321000000A93ED4B0A42F07DFBF6EE007A20EEB9
:10322000270AB5EEC00AF1EE10FA48BF9FED030A77
:1032300008BD18469047F0E7612F02080000000023
:1032400038B50446B7EE001A7120DFED1A0A04F50E
:10325000004504F5C0442DED028BD5F85C3493EDA8
:10326000370A42F057FBD5F86434D4F83029B0EE71
:10327000408A03F50574104913681B698B4215D108
:10328000B6EE061A3020F4EE000A92ED4B0A42F038
:1032900041FB38EE408A9FED090A204628EE000ADD
:1032A000BDEC028BBDE83840CCF00CBF104698470F
:1032B000EFE700BF00000000612F020800007A4421
:1032C00000F51250D2ED007A91ED006AD0ED946ACB
:1032D000D0ED975A27EEA67A65EEE77AA6EE257A24
:1032E000E6EE267AC1ED007A82ED007A704700BFE3
:1032F00000F5C043B3F9583143B900F58040B0F947
:1033000056070028B8BF404280B2704783EAE37096
:10331000A0EBE37080B27047704700BF704700BFFA
:10332000704700BF704700BF002070470020704703
:103330000020704700207047002070470020704731
:10334000002070470020704700207047704700BF82
:10335000034644F26C701844704700BF0048704741
:10336000BC781A0800F5C040D0F80C0903681B6847
:10337000184700BF10B4044C39200C6008211070AD
:103380005DF8044B1960704744411A0800F500408D
:103390009FED0A7AD0F870340120D3ED0E7AF4EE66
:1033A000C77A9FED077AF1EE10FAB8BFD3ED047A31
:1033B00067EE877AC1ED007A704700BF00000034E5
:1033C0000AD7233C00F5C040DFED047AD0F80C09A1
:1033D00020EE270A03685B6E184700BF0000C84252
:1033E00000F5104393F81D35002B14BF1B2003205C
:1033F000081AB0FA80F04009704700BF00F5C040DD
:1034000090F82509C0F38000704700BF00F5C04068
:10341000D0F80C0903685B6D184700BF00F5C04089
:10342000D0F80C090368DB6C184700BF00F5C040FA
:10343000D0F80C0903689B6C184700BF00F5C04228
:1034400049F210230344D2F80C09C01AB0FA80F0F4
:103450004009704700F5C04010B5D0F80C090C4683
:103460000368DB6D984707EE900A9FED057A01200F
:10347000F8EE677A67EE877AC4ED007A10BD00BF78
:103480000AD7233C00F5C04010B5D0F80C090C4613
:1034900003689B6D984707EE900A9FED057A01201F
:1034A000F8EEE77A67EE877AC4ED007A10BD00BFC8
:1034B0000AD7233C00F5C04010B5D0F80C090C46E3
:1034C00003681B6E9847DFED047A012020EE270A7F
:1034D00084ED000A10BD00BF0AD7233C9FF06CB8F2
:1034E000FAF0E0B918F0D6B805F0BABAB1F012BEE9
:1034F00094F09CBC7CF086BE3FF0D8BA81F0C6BA8E
:1035000021F034B895F04EBA8EF0E6BB8FF050BA89
:1035100016F020BA16F0F0BE08F05CBC18F050B8F7
:1035200007F0D6BA06F0D6BF06F0C6BE16F0BABB94
:10353000ACF0EEBDBAF056BF13F070BAFFF740BD65
:1035400016F04CBBE2F006B8B6F00AB916F008BEA9
:1035500004F072B916F0C8BA16F044BA91F08ABAFB
:103560006FF050B931F096BA07F08CBF03F03EBC53
:1035700095F028BA16F036BE08F0E2BB05F0F4BDAF
:1035800008F06ABD06F05EBF08F03CB816F062B9FC
:10359000FFF7F0BC3FF07EBE00F5004008B5D0F864
:1035A0007004F1F065F9012008BD00BF49F2102C4C
:1035B000844400F5C040D0F80C09604501D00020DB
:1035C00070470AF051BD00BF49F2102300F5C04218
:1035D0000344D2F80C09984200D070470AF062BD4B
:1035E000012100F512501BF019BC00BF07F0ACBC64
:1035F0000CF048BE0CF07ABB0CF002BB00F5C043E7
:1036000030B50446D3F80C0983B00D4603685B6AF5
:10361000984760B10023DFED070A49F6700029469C
:10362000B0EE600A1A462044009310F0F1FB03B09C
:1036300030BD00BF0000000000F5C04310B50446D7
:103640002DED028BD3F80C09B0EE408A03685B6A5B
:10365000984720B900242046BDEC028B10BD9FED99
:10366000080A49F6700028EE000A20440FF09EF880
:1036700004460028EED001210248FFF7CFFBEAE71D
:103680000000C842F033002470B584B005460C46F3
:103690001646684624F068F805F5C0436946D3F835
:1036A0000C0903685B6D98476946204624F096FF35
:1036B00010B9002004B070BD6946204624F09CFF7C
:1036C0000028F6D0204624F0A5F80446304624F021
:1036D000A1F88442EDD12B68314628461B6A9847F1
:1036E00004B070BD2DE9F0431F4600F5C043044609
:1036F0000D4616462DED028BD3F80C0987B0B0EEBF
:10370000408A0368F0EE608A9DF840805B6A9DF80D
:103710004490984718B39FED140A49F67000CDF80D
:1037200004903B46D5ED006A68EE800A95ED017A7B
:103730002044D5ED027A66EE806A27EE007A3246A2
:1037400067EEC07A03A928EE000ACDF80080CDED1F
:10375000036A8DED047ACDED057A10F049FA07B0D1
:10376000BDEC028BBDE8F0830000C84200F5C04309
:1037700070B50446D3F80C098EB00E4603681546A2
:103780005B6A9847D8B3DFED1F7A0020D6ED004A78
:103790000BAB96ED015A08AAD6ED025A64EEA74A81
:1037A00095ED006A25EE275AD5ED016A65EEE75AD8
:1037B00095ED027A26EE276ADFED130A66EEA76A18
:1037C000009067EE677AB0EE600A05A9CDED054A74
:1037D0008DED065ACDED075A8DED086ACDED096ADB
:1037E000CDED0A7ACDED0B0ACDED0C0ACDED0D0A2B
:1037F000CDE9010049F67000204410F04DFC0EB0F8
:1038000070BD00BF0000C842000000002DE9F04775
:103810001D4600F5C04304468A4616462DED028B30
:10382000D3F80C098EB0F0EE408A0368B0EE608ADF
:103830009DF860705B6A9DF864809DF86890984779
:10384000002846D09FED250A49F670000BAB08AA68
:1038500068EE000A204405A9CDE901899AED003AF5
:10386000DAED013A9AED024A23EE003AD6ED004A2B
:1038700063EE803A96ED015A24EE404AD6ED025AA4
:1038800064EE804A95ED006A25EE005AD5ED016A96
:1038900065EEC05A95ED027A26EE006A66EE806A01
:1038A000009727EE407A8DED053A28EE800ACDED9F
:1038B000063A8DED074ACDED084A8DED095ACDED5A
:1038C0000A5A8DED0B6ACDED0C6A8DED0D7A10F074
:1038D000E3FB0EB0BDEC028BBDE8F0870000C842F0
:1038E00000F5C04370B50546D3F80C0986B00E4606
:1038F00003685B6A9847044610B39FED136A002380
:10390000D6ED006A012196ED017A49F67000D6EDF8
:10391000027A66EE866A27EE067ADFED0C0A67EE1B
:10392000C67A0191B0EE600A1A46284403A90093B2
:10393000CDED036A8DED047ACDED057A10F040F9F6
:10394000204606B070BD00BF0000C8420000000065
:103950002DE9F047984600F5C04305460F46164648
:103960002DED028BD3F80C098AB0B0EE408A0368C3
:10397000F0EE608A9DF850905B6A9DF854A09847DD
:103980000446A8B39FED1D0A012149F67000434685
:1039900068EE800A07AA2844CDE9009AD7ED004ACC
:1039A00097ED015AD7ED025A64EE804A96ED006A0F
:1039B00025EE005AD6ED016A65EEC05A96ED027A00
:1039C00026EE006A66EE806A029127EE407A04A92C
:1039D00028EE000ACDED044A8DED055ACDED065ACC
:1039E0008DED076ACDED086A8DED097A10F072F859
:1039F00020460AB0BDEC028BBDE8F0870000C8424B
:103A000000F5C04370B505462DED048BD3F80C09C5
:103A100088B0F0EE409A0368F0EE608AB0EE419A0A
:103A20005B6AB0EE618A9847044600B3DFED120A84
:103A300000264FF07E5304A829EEA00A079629EE2F
:103A4000201A049368EEA00A0696059646F05EF9E1
:103A50009FED0A0A49F67000002304A928EE000A27
:103A6000284401AA0196029603960FF0A9F9204670
:103A700008B0BDEC048B70BD35FA8E3C0000C84226
:103A800000F5C04330B505462DED048BD3F80C0985
:103A900089B0F0EE409A0368B0EE609AF0EE418A89
:103AA0005B6AB0EE618A98470446F0B100234FF09C
:103AB0007E5204A8049207930693059346F0A0FB58
:103AC0009FED0C0A01A8CDED019A8DED029ACDED86
:103AD000038A47F0A1FF49F67000B0EE480A0123BF
:103AE00001AA04A928440FF06BF9204609B0BDECE7
:103AF000048B30BD35FA8E3C0A4B93F900290B46F6
:103B0000002A09DB00F50040D0F85C24783207CAAF
:103B100083E8070001207047002201208A604A6084
:103B20000A607047F0930024F8B54D4A00F5104341
:103B30000546026093F8F42042B9D3F8F0402CB166
:103B400020463CF043FD204624F07CFE05F5C043B2
:103B5000444AD3F89408C3F8982608B124F076FEB6
:103B6000414B44F24C102B60284423F079FD05F5BD
:103B7000405393F8582842B9D3F854482CB1204602
:103B80003CF024FD204624F05DFE42F2503041F628
:103B9000DC6441F6C46628442C442E44DFF028FF40
:103BA00014F8043C083C3BB92768384627B13CF080
:103BB0000DFD384624F046FEB442F1D141F6C8303E
:103BC00041F2847441F2247628442C442E4494F02B
:103BD000A3FD2046183C3BF091FFA642F9D141F2EB
:103BE000B01441F26817214B2C442F44C5F8883C8F
:103BF00014F8043C083C3BB92668304626B13CF03A
:103C0000E5FC304624F01EFEBC42F1D105F64C60C6
:103C100084F02CFC05F5626084F028FC05F6F45075
:103C200084F024FC05F6485084F020FC05F61C5076
:103C300084F01CFC05F54F6084F018FC0C4A95F8E4
:103C40001032C5F8FC2043B9D5F80C422CB12046FF
:103C50003CF0BCFC204624F0F5FD2846F8BD00BF32
:103C6000C8451A08BCB71B0834921B0854321B08FD
:103C7000D40F1E0810B5044607F066FD204616F066
:103C8000D5FC204605F04EF82046BDE8104005F072
:103C9000D9B900BF10B516F085F991F069F803683D
:103CA000BDE810405B68184710B5044607F05CFAA1
:103CB000204607F001F8204607F0ACFA204617F03E
:103CC0000FFD2046BDE8104004F004BEF8B5714B6E
:103CD0000546002744F2405440F8043B44F2C066D5
:103CE000AAF070F805F110001FF082FF05F1B00096
:103CF000E4F0F2FC05F528707CF066F805F55670E6
:103D00002EF0CEFF05F5F4601DF0D0FD05F63C1059
:103D100024F0F4FD05F688403EF0C0FB41F2187037
:103D20002C442E4428449EF01DFB41F2E8702844A8
:103D300074F050FE41F69820284480F001FC41F6D2
:103D4000AC302844B9F0FAFC41F6C830284494F06D
:103D5000CBFC41F60440284422F08AFD05F5E650EC
:103D6000CFF0BEFC42F250302844DFF02DFE42F28C
:103D70006C3028447CF036FC42F2DC302844ABF056
:103D800083FC05F5005342F23040434A83F8207427
:103D900042F2204328442B4413606BF017FD394650
:103DA00005F5125018F0DEFF42F678302844B1F0E5
:103DB000C1F942F6A8302844CEF054FB43F23460F7
:103DC0002844D7F0FFFB43F24C702844D6F0B8F8F3
:103DD00043F274702844DAF045F805F56050DEF0DF
:103DE00073FD43F664002844DFF0F6FA43F6BC00A6
:103DF00028449EF035FD43F6EC302844CCF0F2FB2D
:103E000043F69440284417F0BDFF05F57850CFF0F5
:103E1000B3F943F658602844E1F00CF944F2AC10D1
:103E20001E49284472F05CF844F2C4102844E6F0BD
:103E3000BFFD44F2CC102844BAF0FAFB44F28C20C7
:103E40002844E0F0A7FF44F2E420284400F1D6FC27
:103E500005F5804383F8307520460C3484F046FE27
:103E6000B442F9D144F2CC600D4C2844E0F0ECFFB0
:103E700044F2F060284484F0F3F8236833B928460C
:103E8000084972F02DF828462560F8BD064800F173
:103E900063FC00BF34921B080CE4002470AB1D08C7
:103EA00084D600244C901B08A43A1A0870B546F634
:103EB0005C150446054428461FF0AEFA25F0FEFEC8
:103EC00090F9253093B390F844337BB304F5C043A5
:103ED00004F63C16D3F83009443084F00BFE034658
:103EE000B7EE001A9F20DFED120A93ED000A41F0B1
:103EF00011FD94F9743928460021012B04F69834F9
:103F000008BF86ED0F0A1FF063F89FED0A7ADFED18
:103F10000A7A304620EE070A94ED287AA7EE270A9F
:103F200084ED280ABDE8704025F046BB70BD00BF97
:103F300000000000CDCCCC3D6666663FFFF7B6BF03
:103F400010B50121044616F0B7FB30B1124BD3F87F
:103F50000C0903689B6A9847B8B14FF400112046DA
:103F600016F0AAFB60B94FF48021204616F0A4FB9E
:103F700000B910BD40F04CFFBDE810403DF03EBB25
:103F800040F046FF3DF06AFCEDE7204602F02AFED5
:103F9000204602F037FEE0E7F0930024FFF7D0BFA1
:103FA00070B500F50045044684B09FED6F0AD5F862
:103FB0005C046C3047F0DCFC01A904F512508DED77
:103FC000010ACDED020A8DED031A18F08DFD0221D4
:103FD000204616F071FB002874D10121204616F00E
:103FE0006BFB40B9614BD3F80C0903689B6A984797
:103FF000002800F0AC800121204616F05DFB00286F
:104000005CD04FF40031204616F056FB30B104F579
:10401000C043D3F8300903685B6C984740212046C1
:1040200016F04AFB00286ED14FF48061204616F04E
:1040300043FB002861D12021204616F03DFB58B1FA
:1040400004F5C046D6F80C0903681B69984740B3CD
:10405000D5F86404EDF0F4FF8021204616F02CFB27
:1040600030B94FF48021204616F026FB002872D08C
:1040700040F0CEFE3DF0E8FA1021204616F01CFB81
:10408000002855D14FF6FF71204616F015FB002889
:1040900048D14FF40041204616F00EFB28BB04B077
:1040A00070BD204610F004FA0028D1D1D6F80C09D2
:1040B00003685B6998470028CAD0CDE7204602F024
:1040C000FBFD9EE70121204616F0F6FA002884D178
:1040D000264BD3F80C0903689B6A984700287FF4A5
:1040E0007CAF204602F07EFD77E748F2FC4020449A
:1040F00004B0BDE8704095F03FB841F698202044E8
:104100007FF0C6FC97E741F6982630197FF014FC43
:1041100004F5805393F9C83B002B85D030197FF00C
:10412000EFFD81E746F23C102044F9F0C5FBB0E713
:10413000D5F85C04E9F04CFB44F69C002044B5F053
:10414000EFFC44F2E0702044E1F028FA9AE72046C0
:1041500002F058FD4FE74FF40021204616F0ACFA6C
:10416000002885D188E700BFE02E6542F093002447
:10417000FFF716BF10B50121044616F09DFA58B995
:104180008021204616F098FA78B94FF400112046A5
:1041900016F092FAD8B910BD204602F08DFD8021AC
:1041A000204616F089FA0028EFD04FF480212046EF
:1041B00016F082FA0028E8D140F02AFE3DF01EFAFF
:1041C0004FF40011204616F077FA0028E3D004F5EA
:1041D000E650BDE81040D0F03FBD00BFFFF7CABFBA
:1041E00070B504464FF6FF7116F066FA04F5C04547
:1041F00080BBD5F8303993F8D530BBB393F05AF87B
:1042000004F5004692F058FA204617F05BFA95F84C
:10421000003904F51044234ADB43C3F3C01384F888
:104220008D30D6F85C5453712B681C6F7CF0A8F865
:104230007BF02CFD1C4B9C4225D1D6F864447CF0CD
:104240009FF87BF023FD04F505742046BDE870401F
:10425000CBF0E6BC07212046D5F8002902F062FD2C
:10426000D5F8303993F8D530002BC7D12046FEF76A
:104270005BFED5F830090D4A03681B6A934205D1ED
:10428000F6F060FABAE72846A047D6E704F5804280
:1042900004F5A04192F8722791F844129847D5F896
:1042A0003009EDE758D500241D3302081933020800
:1042B000FFF796BF2DE9F04100F5125300F5C04419
:1042C00000F500580546D3F8502204F6441704F6CA
:1042D000481644F250603A60D3F85C323360D8F844
:1042E0008036184441F0C4FAC4F84C0904F515634B
:1042F0003A6804F654144FF6FF711A602846336882
:10430000236016F0D9F908B9BDE8F081D8F8802605
:1043100028460921BDE8F04102F0D6BC00F5C041B5
:10432000D1F84029002A48D091F8013913F0010F43
:1043300043D06FF30003012AD1F8902481F80139AA
:10434000D1F88C34B2F9082007EE902AB3F908208E
:10435000F8EEE77A07EE102A30D0B8EEC77A01F609
:10436000541C01F515629CED006A00F51250D2ED67
:10437000005A66EE676A65EEA77AE7EE256AE7EE11
:10438000067A90ED977A90ED946A27EE877AA6EEFA
:10439000867ABDEEC77A17EE102A1A8190ED946ADC
:1043A00090ED977A67EE867AD1F89034E6EEC77A88
:1043B000FDEEE77A17EE902A1A817047B8EEC77AB9
:1043C00001F6481C01F64412CDE700BF38B504469B
:1043D00000F5C0452DED028B59B9D5F84039022BB7
:1043E00002D0BDEC028B38BD15F0FCFBB0F57A7F36
:1043F000F7D3204615F01AFCD5F84C3940F2E632D6
:104400001B1A03F2F3139342EBD944F25063174A99
:10441000C5F84C09034482FB0312DB17C3EB62139C
:1044200006EE903A9FED0F7BB8EEE60B20EE070B01
:10443000B7EEC08BB0EE480A76F128FBF0EE407A7A
:1044400005F5156305F65415B0EE480AC3ED007A7C
:1044500077F1B8F985ED000ABDEC028B38BD00BFDD
:10446000AFF30080000000A046DF913F1F85EB51B5
:1044700010B5044615F02AFE1021204616F01CF94E
:1044800000B910BD204602F0E3FA4FF400112046B7
:1044900016F012F90028F4D140F0BAFC3DF0DEF934
:1044A00004F5E650BDE81040D0F0D6BBFFF7E0BF02
:1044B0002DE9F04F89B00446FFF708FCDB4B44F2CE
:1044C000987004F5C046236046F2A84520444FF09A
:1044D0007C5802F0FBFD44F26073254405A9234497
:1044E000CDF8148005F1080048F24047C6F8A03422
:1044F0000623274446F2986986F8A43484F00CFC1D
:1045000005F12000FFF096F90023CDF8108046F267
:10451000F04886F8E0341923A04404A986F8EC3466
:1045200046F2B05508F10800C6F8E87484F0F4FBD0
:1045300008F12000FFF07EF94FF00108182346F241
:104540004850254486F8288586F834352044C6F836
:10455000307546F2687793F01DFA2846E2F05CF871
:10456000B34B8DF818800DF11808C6F8B035281D2A
:104570004146B04D73F02CFD46F21060A144274433
:1045800020446EF0C9F846F250602044E0F068FD27
:10459000A94B46F268604146C6F85036204406955D
:1045A00084F0BAFB46F2746041460695204484F0DC
:1045B000B3FB4146069504F5CD4046F2C86584F04C
:1045C000ABFB9E4B09F10C002544C6F89836FFF072
:1045D00031F9284614358BF0D9FBBD42F9D11E23A1
:1045E00040F2CC60C6F898380023A6F89C3824F036
:1045F00023F9C6F8940846F6A0002044FFF01AF903
:1046000046F6E4002044FFF015F98D4B1A68002AA5
:1046100000F05D8249F65C278A4B46F610104FF099
:104620007E552744C6F898362044C6F80C79E4F045
:1046300039F806F6441346F65C1006F515661D605B
:104640004FF40071804B2044356048F20C660793AC
:104650007E4B26440694009398E80C001EF032FA34
:1046600046F6F4602044C1F0D9FF48F2104003A997
:104670000395204484F07AFB48F2244003A9039573
:10468000204404F5004584F047FB48F230402044C4
:1046900023F06AF8002305F5886248F27C404FF465
:1046A0000041136020445360936005F24C42136054
:1046B0005360936004F51253C5F85834002385F80D
:1046C00079341FF0EFFB48F2FC40204494F052F99B
:1046D00048F280502044BDF025F948F2BC502044F7
:1046E00073F0A6FD5A4B48F2D050C5F8BC352044B3
:1046F000B9F01EFE48F2EC50564B20445649186063
:1047000071F0EEFBFF235549304685F81C3685F8DD
:10471000243671F0E5FB524B1D68002D40F0DD8121
:1047200048F22C601E6048F6D07804F5104620440C
:104730007DF014FB48F6D460A0442044EEF0D4FE93
:1047400048F6C8702044EEF0B9FC4046CAF0DCFAE6
:10475000414604F51140F7F0D5F8424B424949F281
:104760006010C6F800310623204486F854313F4BD0
:1047700019600B7C4BB12B4601339BB203EB8302D8
:1047800001EB8202127C002AF6D13949394A0B80AA
:10479000D2F8009038490B80B9F1000F40F09A81AF
:1047A000106049F27410354B03A9204449F21028D7
:1047B000039384F0B1FA49F29410A0444FF6FF7AC3
:1047C0004FF0FF3B2044002507F048FB2C4B49F2FB
:1047D000D410C6F89431204407F040FB294B4046E2
:1047E000C6F8D43107F03AFB274B49F29020C6F8BF
:1047F0006882C6F81032254B2044C6F87082C6F88D
:104800006C32234BC6F8788208F13C08C6F8743243
:10481000204BC6F87C3222F0A7FF49F2AC2020449E
:1048200022F0A2FF49F2C82036E000BFC8451A08AE
:10483000183A1A080000A0405C3A1A08BCB71B08D6
:1048400014DB0024AC461A08ED350208B8451A08F6
:104850006C3A1A0818E400244C071C08A8A91D0883
:10486000DCE40024B4A11A0844971A083CD60024BA
:1048700038D60024D4D5002408D60024CDCC4C3D15
:10488000F8A61A08A0A71A0818AB1A08F1350208EA
:10489000F5350208F9350208204422F065FF904BF7
:1048A00049F2E420A6F8E0A2C6F8DC32204422F067
:1048B0005BFF8C4B8C494046C6F894B4C3F800802B
:1048C00071F00EFB49F2A840A6F888B2A6F8A4A29F
:1048D00049F6102820444FF0010A22F045FF49F222
:1048E000C440A044DFF850B2204422F03DFF49F21A
:1048F000E040204422F038FF49F2545086F8F49406
:104900002044C6F8189507F0A9FA784B49F2905060
:10491000C6F854352044FBF0EBF8754B49F214709F
:10492000C6F89035204407F099FA724B49F2587056
:10493000C6F81437204407F091FA6F4B49F298708B
:1049400086F89497C6F85837204407F087FA6B4BDF
:1049500049F2D470C6F89837204407F07FFA684AC5
:1049600006F5016349F62800C6F8D42720441D60E7
:104970005D609D6007F072FA624B49F67000C6F800
:104980006498C6F82838204407F068FA5E4B49F668
:10499000B400C6F8AC98C6F87038204407F05EFA48
:1049A0005A4B49F6FC00C6F8B438204407F056FAD2
:1049B000574B49F63C10C6F8FC38204407F04EFA35
:1049C000544A06F6B41349F6D010C6F83C292044E0
:1049D0001D605D6007F042FA4046A6F80CAAC6F8D2
:1049E000D0B922F0C1FE08F1100022F0BDFE08F19E
:1049F000200022F0B9FE08F1300022F0B5FE384662
:104A000007F02CFA444B49F6982049F66C47C6F853
:104A10005C3A2044274412F0DBF949F65430204434
:104A200007F01CFA3D4B49F69830C6F8909BC6F843
:104A3000543B204407F012FA394B49F6E830A6F807
:104A4000D49BC6F8983B204407F008FA354B49F64A
:104A50002C40C6F8249CC6F8E83B204407F0FEF939
:104A60003846C6F82CBCA6F868AC22F07DFE07F1EB
:104A7000100022F079FE07F1200022F075FE07F108
:104A8000300022F071FE06F6BC43274A49F6C840C2
:104A900086F8B5ACC6F82C2C20441D605D609D6086
:104AA0000CF0F6FE49F69C50204413F0BDFD49F68B
:104AB0001460204407F0D2F906F654631B4A2046DE
:104AC000C6F8142E1D605D6009B0BDE8F08FC3F814
:104AD00000909FE51648FFF03FFE1648FFF03CFEB1
:104AE0000000FFFF20D5002408441B08C0AB1A08B3
:104AF00054AC1A08B8AD1A085CAE1A0800AF1A0810
:104B00009CAF1A08ECB11A0890B21A08D8B31A0868
:104B10007CB41A0820B51A0804B81A0814AD1A088B
:104B20004CBC1A083CB31A085CB71A0814BD1A0822
:104B3000DC3A1A08B83A1A08A0B61A0838B5054C73
:104B40000A46054B01462468256820462C68A04784
:104B5000002038BD50D20024F033002410B5084C9A
:104B6000FFF0D4F9074B024620461A60FFF7A0FC7D
:104B70002046054A0549BDE8104075F181BF00BFD8
:104B8000F033002450D20024588A0124293B020823
:104B90000120704790F8D0308B4204D900EB81009F
:104BA000D0F8D40070470020704700BF90F8D03094
:104BB0008B4204D900EB8100D0F8D400704700206C
:104BC000704700BFFA207047014B93F822077047E7
:104BD000F0730024044BD3F84009A0F10100B0FAAF
:104BE00080F04009704700BFF0930024044BD3F8D5
:104BF0004009A0F10200B0FA80F04009704700BF00
:104C0000F0930024034BD3F8300908B1F3F08EBFC2
:104C100001487047F093002498461A08F8B5D0E987
:104C20000912C36A0446534D41F4E05043F4E05383
:104C300042F4E0526062C4E90A23D5F86434ABB1AF
:104C400041F4F8416162D5F86404ECF039FA38B106
:104C5000D4E90A2342F4804243F48043C4E90A239E
:104C6000D5F86404ECF06CFD00286FD14248B4F034
:104C7000D7FE18B1636A43F0806363623E48B4F0C4
:104C8000F7FE18B1A36A43F08063A3623A48B4F018
:104C9000F5FE18B9E36A43F08063E362374B1F689F
:104CA000002F5CD01921384674F0CCFC18B1636A2F
:104CB00043F480736362324E96F8A834002B35D1EA
:104CC000A36A95F9D42EEAB9626A95F8D01E013923
:104CD000012907D8E16A42F4800243F4800341F4D9
:104CE0008001E16243F0804342F08042C4E909233D
:104CF000D6F8303993F8C1301BB9E36A43F08043EA
:104D0000E362F8BD626A43F0800342F08002C4E9C6
:104D1000092395F9D41E0029D7D095F8BC1F002986
:104D2000D3D0E16A41F08001E162CEE7A36A384660
:104D3000192143F48073A36274F0D6FC0028BFD01D
:104D4000D4E90A3242F48072E262BAE7D4E90A2373
:104D500042F4005243F40053C4E90A2386E7084EA4
:104D600096F8A834002BABD0A36A43F48073A362F7
:104D7000A7E700BFF0B300248C7C00244CD60024AD
:104D8000F093002470B54FF444700D46164623F09E
:104D90004DFD044628B13246294688F065FA024B9B
:104DA0002360204670BD00BF0C491A0800207047E0
:104DB000704700BF0320704708207047014B93F8ED
:104DC00024077047F0730024034B93F9380200382E
:104DD00018BF0120704700BFF0830024014B93F9F6
:104DE00026077047F0730024704700BF08B50C4BCE
:104DF000D3F8640410B1ECF063F968B950201022C4
:104E0000084BD3F8303923B193F8D5300BB142F0C9
:104E1000C00040F0010008BD58201822F0E700BF94
:104E2000F0B30024F093002400B5002389B002936E
:104E3000039304930593069307931AF02BF902A9A1
:104E40001AF0C4F810B909B05DF804FB1AF022F9A1
:104E500000F55A7005AB07C883E80700184647F00D
:104E60002BFAF1EE047A20EE270AFCEEC07ACDEDA3
:104E7000017A9DF8040009B05DF804FB10B5194CE7
:104E800084B094F8EA1D04F6944017F0ADFB30B1FD
:104E900094F8EA1D04F6944017F0BCFBC8B900234F
:104EA0000193029303931AF0F5F801A91AF08EF812
:104EB00050B92FF017FFB02290F80C3302FB03001B
:104EC00090ED410A04B010BD01A847F0F5F904B017
:104ED00010BD94F8EA1D04F6944004B0BDE81040FB
:104EE00017F036BDF063002408B50D4BD3F8300938
:104EF000A8B1443083F0FEFD0346B7EE001A9F20B0
:104F000093ED000ADFED070A40F004FDDFED067ABD
:104F100020EE270ABDEEC00A10EE103A18B208BD06
:104F2000F0930024000000000000C8422DE9F04F7B
:104F3000354C8DB0354E4FF0010B0546E71C06F59C
:104F40008049B6F97C370BF1FF3A43FA0AF3DB07E5
:104F500033D5287C85F07CFE8046287C86F0A8FE30
:104F600000F12103984548D3BAF1030F25D8DFE8B3
:104F70000AF03C342C02D9F8643403F52D735968D7
:104F80001A680491D968586A069119690392212216
:104F900007919969059159691B6A089162210092EC
:104FA00003AA0191C221CDF82500CDF8293019239B
:104FB000287C8DF824B085F0CBFEA74202D014F8EF
:104FC00001BBBEE70DB0BDE8F08FD9F85C04036803
:104FD0001B69984700F1A003D1E7D9F85C04036886
:104FE000DB68984700F1A003C9E7D9F85C040368BF
:104FF0009B68984700F1A003C1E7287C0DB0BDE88D
:10500000F04F84F0F5BE00BFFD491A08F07300248C
:1050100010B50446F8F060FC20B12146BDE8104010
:10502000F8F01CBC10BD00BF38B5044606480D465C
:105030000AF01EFD28B929462046BDE8384087F011
:10504000E5B8042038BD00BF00C60024014809F0BF
:105050006DBB00BF00C600240E4B30B50D46D3F823
:105060003C1283B00446C9070CD411460A48019289
:10507000F9F0AAFB019A2946204603B0BDE830406A
:105080008DF0FABA114603F582400192F7F054F818
:10509000019AEAE7F08300245095002410B588B007
:1050A000044688F0C1FF0C4BD3F8300958B169466B
:1050B0001E22F3F097FC6B46084A0621204688F032
:1050C0009BFF08B010BD064A0621204608B0BDE887
:1050D000104088F091BF00BFF09300245C011E08CF
:1050E000E4461A08034A92F88834013382F8883477
:1050F00087F09EBAF09300240148EEF04FBC00BF49
:10510000C4C2002400B583B00846019123F0B4FA6C
:1051100038B10199054803F0A9F9002003B05DF802
:1051200004FB042003B05DF804FB00BF5CD2002444
:1051300070B58B8B82B00C460546CD2B06D0214630
:10514000284602B0BDE8704087F012BBD1ED067A68
:10515000FCEEE77ACDED017A9DF80430022BEED11A
:105160000D4E019296F8751506F2FC4093F044FC42
:10517000019A0028E3D096F8751506F2FC4093F0EA
:1051800045FC019A0028DAD194ED020A034803F0A5
:105190004DF9019AD3E700BFF0B300245CD200249C
:1051A000542A18BF162A0CBF0123002303D103225F
:1051B00018460A70704787F045B800BF70B50C46B6
:1051C0004B7A897A0546E27A43EA012343EA0243AD
:1051D0009D2B05D021462846BDE8704087F084B954
:1051E000124E96F8751506F2FC4093F005FC002867
:1051F000F0D096F8751506F2FC4093F013FC0228E7
:10520000E8D196F8751506F2FC4093F0FFFB0028F4
:10521000E0D1D4ED057A9FED060AF8EEE77A05486D
:1052200027EE800A03F002F9D4E700BFF0B30024B0
:105230000AD7233C5CD20024074A40F6CD1310B5B0
:1052400040F6CD3492F92C26002A08BF1C4687F080
:10525000A3F9204310BD00BFF0B3002410B584B003
:1052600019F018FF0446684622F07EFA6946204687
:1052700019F094FE0E4B93F8010910F0200014D0A1
:1052800003F50053DDED017A9FED0A7AD3F864341B
:10529000F8EEE77AD3ED0F6A77EEA67A67EE877AB3
:1052A000FDEEE77A17EE903A18B204B010BD00BFD9
:1052B000F09300240AD7233C10B5044623F0C2FA29
:1052C000204610BD10B50C4C94F90039002B0FDBB3
:1052D000D4F80C090368DB6C984758B9D4F80C096A
:1052E00003689B6C984700280CBF0220032010BD68
:1052F000012010BD042010BDF093002408B5134B0D
:1053000093F8010910F020001CD0D3F80C090368B1
:10531000DB6D984707EE100ADFED0D6AB8EE477AAD
:10532000DFED0C7A27EE267AB4EEE77AF1EE10FA8A
:1053300009D5F2EE046AC7EE267AFCEEE77A17EE9C
:10534000903A98B208BD41F6991008BDF093002438
:105350000AD7233C00FF7F4710B44C69012C03D0CF
:105360005DF8044B87F07EB901465DF8044B0148B7
:1053700003F050BFF0330024B1F90430002B3EDBC2
:105380009FED1F0A4FF47A732DE9F041DFF8788022
:1053900082B000270C461546009201970646B1F9E7
:1053A0000220D8F88C148DF043FC0123D8F8901417
:1053B000304601934FF47A7300959FED110AB4F9CA
:1053C00000208DF035FC3B46D8F8941430469FED14
:1053D0000D0ACDE90057B4F904208DF029FCB4F989
:1053E00006209FED070A3046D8F898144FF47A73D8
:1053F000019700958DF01CFC02B0BDE8F08170476C
:105400000000FA4400007A44F093002408B50A4BE7
:1054100093F8010910F020000DD0D3F80C090368AF
:105420009B6D984740F024FA044B83FB0023C01780
:10543000C0EBA310C0B208BDF09300241F85EB5150
:10544000044B187820B9044B93F80209C0F380107C
:10545000704700BFE8D30024F093002400B5002378
:1054600087B003930493059319F014FE03A919F070
:10547000ADFD10B907B05DF804FB19F00BFED0EDDF
:10548000DA0A90EDDB0AF1EE600AB1EE400A76F13D
:1054900095FBDFED097A20EE270A40F0ABF9F6EE36
:1054A000007A20EE270AFCEEC07ACDED017A9DF855
:1054B000040007B05DF804FBE02E6542144B93F83E
:1054C000010910F0200000D1704703F5005300B52A
:1054D000D3F8640483B000F5657046F0EDFE9FEDEF
:1054E0000D7ADFED0D7A20EE070AB4EEE70AF1EE51
:1054F00010FA03D4FF2003B05DF804FBFCEEC07A81
:10550000CDED017A9DF8040003B05DF804FB00BF07
:10551000F0930024CDCC4C3D00007F430B4B93F81F
:10552000F12E7AB993F8252992060BD193F9002927
:10553000002A09DB93F8013913F0200F14BF04206F
:10554000012070470520704703207047F093002426
:1055500030B52DED028B89B0054619F09BFD00F5A5
:105560005A7002AC2D7C07C884E80700DDED020A02
:105570009DED030AF1EE600AB1EE400A76F11EFBE2
:105580002046B0EE408A46F097FEDFED0B7A0C2302
:105590000499012228EE278A28460791A8218DED3B
:1055A000060A8DED058ACDE9003205AA85F0D0FB0B
:1055B00009B0BDEC028B30BDE02E654208B5074B4B
:1055C00093F97037032B03D0BDE8084088F0B8BDCD
:1055D000034A022188F010FD042008BDF073002466
:1055E000FC461A08094BD3F83C2292070CD503F568
:1055F0004053DFED077A03F2344393ED000AB8EE2F
:10560000C00A20EE270A704786F010BEF0830024FF
:105610000AD7233C30B595B0044603A822F0A4F87D
:105620001E4B03A9D3F80C0903685B6D984708B9B2
:1056300015B030BD002103A822F0A0F90028F7D052
:10564000257CFFF0BBF8DDED047A9621059C002255
:10565000F8EEE77A9FED127A01914FF6F85108942F
:10566000002467EE877A3323079028460B920C922A
:105670000D920E920F9210921192129207AAADF80B
:105680004C1057218DF84E40069C0093CDED0A7AC0
:10569000099485F05DFB15B030BD00BFF093002488
:1056A0000AD7233CF0B5884C05462DED0A8BD4F87B
:1056B0000C3999B01A681846536A9847002864D084
:1056C00004F54054D4F8AC38062B00F2E880DFE84B
:1056D00003F004040460A3C95C007C480BAC0EF02A
:1056E000FBFD03469FED7A8A20469FED7A0A40F63D
:1056F000F8579FED799AF0EE489AF0EE48AAF0EE4E
:10570000498AF0EE48BA93ED025B93ED046B93ED9A
:10571000007BB7EEC55BB7EEC66BB7EEC77B8DED12
:105720000C5A8DED0D6A8DED0B7A46F021F9B0EE35
:1057300040CAB0EE60BAB1EE41AA2E7CFFF03EF84E
:105740008C22002133230546019222460124159123
:105750001691304655210093ADF85C700B958DED98
:105760000CCA8DED0DBA8DED0EAACDED0FBACDEDB3
:1057700010AACDED118ACDED129A8DED138A8DED23
:10578000149A8DF85E4085F0E3FA19B0BDEC0A8BEF
:10579000F0BD4E480BAC0EF09FFD03469FED4D0A49
:1057A00020464FF4406793ED025B93ED046B93ED5D
:1057B000007BB7EEC55BB7EEC66BB7EEC77B8DED72
:1057C0000C5A8DED0D6A8DED0B7A46F0D1F83F48FD
:1057D000B0EE41AAB0EE60BAB0EE40CA0EF080FD65
:1057E0009FED3C0AB1EE4AAA46F0C2F83748F0EE07
:1057F000418AF0EE40BAF0EE60AA0EF075FD9FED22
:10580000350AF1EE688A46F0B3F8B1EE419AF0EE4F
:10581000409AB0EE608A90E72C4840F607470EF0B9
:105820005FFD9FED2C0A46F0A3F82848F0EE418A70
:105830009FED27BAF0EE40BA9FED27AAF0EE60AADE
:105840000EF052FD9FED230AF1EE688A46F090F8C3
:10585000B0EE4BCAF0EE409A0BACB1EE419AB0EE0E
:10586000608A6AE7194840F63F470EF03DFDDFEDDC
:1058700018AA9FED180A0BACDFED178A46F078F8EE
:10588000F0EE6ABAB0EE68AAF0EE409AB0EE608A26
:10589000B1EE419AB0EE6ABAB0EE6ACA4DE79FED3A
:1058A0000C8A00279FED0C9A0BACF0EE489AF0EEB4
:1058B000498AB0EE49AAF0EE48AAF0EE48BAB0EE36
:1058C00048BAB0EE48CA38E7F093002460CC002410
:1058D000000000000AD7233C000000802DE9F043BF
:1058E000404D2DED048B95F801398DB09B0604D405
:1058F0000DB0BDEC048BBDE8F08305F500580446FF
:105900009FED398AD8F85C049FED380A6C3046F078
:105910002FF861EE087AD5F80C6920EE089A8DED23
:10592000020A60EE888AFDEEE77A3368CDED030A5D
:1059300030469B6D17EE902A8DED041A94F8109066
:1059400017B2984707EE900A3046F8EEE77A67EE0E
:10595000887AFDEEE77A17EE903A1CB23368DB6D79
:10596000984707EE900A9FED227AF8EE677A67EE85
:10597000887AF4EEC77AF1EE10FA30D5FCEEE77AC9
:1059800017EE903A9DB2D8F864343046DFED169A9F
:1059900093ED0F8A336828EE298A1B6E98471A23E5
:1059A000B72220EE290A48463E21ADF828708DED39
:1059B000059ACDED068A8DED078A8DED090AADF8C1
:1059C0002A40ADF82C50CDE900320022089205AAF9
:1059D00085F0BEF90DB0BDEC048BBDE8F0834FF649
:1059E000FF75D0E7F09300240AD7233C9F0CB34502
:1059F00000FF7F471D4B2DE9F04F2DED028BD3F8B3
:105A00005C348DB0077CD3F88480D3F88860D3F8F9
:105A10008C50D3F8904093ED258AD3F898B0D3F802
:105A20009CA0D3F8DC90FEF0C9FE162225234FF08F
:105A3000000C02900192384602AA532100938DED8A
:105A4000078ACDF820B0CDF824A0CDF82890CDF865
:105A50000C800496059506948DF82CC085F078F995
:105A60000DB0BDEC028BBDE8F08F00BFF0B3002499
:105A7000B0EEC00ADFED157A10B5B4EEE70AF1EE2C
:105A800010FA0ED4124CD4F80C0903681B6898471E
:105A900004281AD0D4F80C0903681B689847142806
:105AA00013D0022211210B4806F048FE30B140F617
:105AB000C4110948BDE810400BF05AB8022205484D
:105AC0001146BDE8104006F039BE10BD000000349C
:105AD000F0930024F033002404CB0024A1F11B0335
:105AE00070B5044684B0282B16D8DFE803F01A15E9
:105AF000151515151515155915151E4F15151515CF
:105B00001515151515151515151515151515151545
:105B100015151529151A1A0004B0BDE870408DF04E
:105B20006DBE0125284604B070BD122184F072F9C3
:105B3000054600284AD0217C26487BF0C3F9F1E7CE
:105B4000262184F067F9054600283FD0217C2248B1
:105B5000C9F046FA214B1E68002EE3D026212046CC
:105B600084F058F905460028DCD0002301AA402122
:105B70002046ADF804308AF0D5FB0028D2D0BDF81D
:105B800004203046217CBFF059FDCBE7162184F07C
:105B900041F90546D0B1217C0E487BF0ABFAC1E754
:105BA0000C2184F037F9054680B10023019302935C
:105BB000039319F06FFA01A919F008FA03460028B7
:105BC000B0D020461D46FFF7C3FCABE700252846B2
:105BD00004B070BD1CBA0024C0C30024D8E4002463
:105BE000054BD3F830392BB193F8CA00002808BF11
:105BF0000220704702207047F093002408B5034B41
:105C0000D3F80C0903681B68984708BDF09300247B
:105C1000024B93F80109C0F340107047F093002441
:105C2000F0B52A4F87B0D1ED017A0646D7F80C3986
:105C30000C46FDEEE77A1A68184617EE905A536A3A
:105C40009847EB0700D440B3D4E9040141F072FB5C
:105C500018B302A821F088FD02AA214630468BF035
:105C6000EDF9D0B11A4902A822F0F2FBA8B9DFED94
:105C7000190A034602460090B0EE600A02A91648CF
:105C80000EF0C6F890B1D7F80C0903685B6A984724
:105C9000044628B1002007B0F0BD022007B0F0BDD7
:105CA000022204210D4806F049FD08B90420F5E759
:105CB000DFED080A2346224602A9B0EE600A064834
:105CC00000940EF0A5F80028E4D1EFE7F09300244B
:105CD00020B800240000000060CC0024F033002431
:105CE00091ED000AB5EEC00AF1EE10FA1EDBDFED11
:105CF0001F7AB4EEE70AF1EE10FA17D89FED1C7A7E
:105D000010B5D1ED037A82B00C46F0EEE76AF4EEFE
:105D1000C76AF1EE10FA0FD4F7EE000AB0EE670A88
:105D20003FF032FC20B9042002B010BD04207047BF
:105D300094ED000AD4ED037ADFED0D6A94ED027A5A
:105D4000F4EEE67AD4ED010AFDEEC77A0948F1EEE9
:105D500010FACDED017A9DF90410ACBF01220022AA
:105D600002F0C0FA002002B010BD00BF0000B44332
:105D7000000000345CD20024D1ED017AF5EEC07A47
:105D8000F1EE10FA30DD91ED007ADFED186AB4EE35
:105D9000E67A08B5F1EE10FA0CDD154B9FED150A09
:105DA000D3F80C0927EE800A0368DB6E9847A0B190
:105DB000002008BDDFED106A0D4BB4EEE67A9FEDD2
:105DC0000D0AD3F80C0927EE800AF1EE10FA0368E9
:105DD00005DD9B6E98470028EAD1042008BD5B6E64
:105DE00098470028E4D1F8E7042070479A99394091
:105DF000F09300240000C8423333F33FD1ED007A22
:105E00009FED167AF0EEE77AF4EEC77AF1EE10FA2B
:105E100011D5D1ED017AF0EEE77AF4EEC77AF1EE22
:105E200010FA08D5022203210D4808B506F086FCB9
:105E300018B9042008BD0220704709480121FCF769
:105E4000EDFF084890F85032012B05D000F5137093
:105E50004AF0A2F8002008BD002008BD0000003470
:105E6000F0330024F0C3002410B5154882B00C466E
:105E7000F7F030FC60B1D4ED017AFCEEE77ACDEDBD
:105E8000017A9DF80400012805D002280BD090B1BA
:105E9000042002B010BD94ED020A0948F7F07EFC20
:105EA000002002B010BD94ED030A0548F7F0BAFCDB
:105EB000002002B010BD034B83F84A0102B010BDB0
:105EC0002C950024F093002410B5D1ED007A0446FF
:105ED000FCEEE77A17EE903A13F0FF0308D1114B6E
:105EE000D3F80C0903689B6F9847A0B1002010BD40
:105EF000012B01D0022010BD0A4BD3F80C09036816
:105F0000DB6F98470028F1D12046074A062188F028
:105F100073F8042010BD2046044A062188F06CF86E
:105F2000042010BDF093002430471A0820471A08B7
:105F300038B5194C94F82539DB070ED4D4F830392C
:105F400093F8D5305BB194F90039002B0FDB0222B6
:105F50000921A4F5C04006F0F1FB002038BD012264
:105F600004F5B6601146FCF78DFD002038BD0D46E6
:105F700002220521A4F5C04006F0E0FB0028ECD089
:105F800095ED000A0121DFED057AD4F80C0920EE29
:105F9000270A14F0ADFFE0E7F09300240000C842A8
:105FA000F6EE007A91ED007AB4EEE77AF1EE10FAAF
:105FB00001DC0420704701220521034808B5FCF7E5
:105FC00023FE002008BD00BFA099002430B58B8BB4
:105FD00085B08C460446D12B12D8B12B2DD8202B5E
:105FE00022D8102B5AD9113B0F2B57D8DFE803F0DA
:105FF0005D565668894F56565656565656565670E2
:106000004AF2124E734500F0F0802BD94AF2134E3B
:10601000734500F0D3804AF2686E73453ED105B0F7
:10602000BDE83040FFF720BF552B6AD0732B2CD131
:1060300005B0BDE83040FFF753BEB23B1F2B2DD853
:10604000DFE803F06D2C2C2C2C2C2C2C2C2CA3AA50
:106050002C2CB1672C2C2C2C2C2C2C2C2C2C2C2CC0
:106060002C2C7386B3F5967F00F0A3804AF2114E74
:10607000734513D17B4D95F8254914F0010400F0C8
:10608000B9800024204605B030BD542B06D19CF8C1
:106090002030032B00F0BE800224F3E76146204647
:1060A00005B0BDE830408DF085BF022205216E4865
:1060B00006F044FB0028E4D10424204605B030BD9E
:1060C00002220621684806F039FB0028D9D1F3E7FF
:1060D000DCED007AF5EEC07AF1EE10FADCDD9FED32
:1060E000637AF4EEC77AF1EE10FAD5D8FCEEE77ACF
:1060F0005C4A0024CDED027A9DF80830A2F86231A6
:10610000C0E702220921584806F018FB0028B8D140
:10611000D2E7614605B0BDE83040FFF7D5BE614625
:1061200005B0BDE83040FFF727BEDCED007AFCEE9D
:10613000E77A17EE903A99B2012904D0022900F0CB
:1061400085800029B8D14A480024ACF055FB99E776
:106150009CED017A0146DCED007ABCEEC77A9CF832
:106160001030FCEEE77ADCED030A9CED020A8DEDBF
:10617000027ACDED037A00933B489DF808309DF8F4
:106180000C2013F0BFFA04467CE70221394807F0DF
:10619000F7FE002890D074E70221364807F0BAFED7
:1061A000002889D06DE7614605B0BDE83040FFF7B3
:1061B00037BD05B0BDE83040FFF720BE294890F854
:1061C000254914F001047FF45CAFD0F8302992F82F
:1061D000D520002A3FF455AF90F90029002A3ADB78
:1061E00091ED000AFFF744FC4CE705B0BDE83040F4
:1061F000FFF79EBE02220521A5F5C04006F09EFADB
:1062000000287FF43EAF0222A5F5C040114606F0FB
:1062100095FA37E7DCED027A9FED177AF0EEE77A30
:106220009CED060ADFED156A0E4BF4EEC77A20EE00
:10623000260AD3F80C09F1EE10FA4CBF0121002117
:1062400014F056FE00287FF41CAF35E70648002402
:1062500003F022FE16E70122082100F5B660FCF7E4
:10626000D3FC0FE7F0930024F033002400007F43B9
:10627000DCB9002400C60024000000340000C8423D
:1062800030B50C46272200212DED028BE57893B026
:10629000954208A828BF154678F16EFB04F10C0161
:1062A00008A82A4678F11EFB4C4BD3F80C0903686A
:1062B0005B6A9847002841D09DF8464061063DD46E
:1062C0004FF07E5200230492220607930693059313
:1062D00040D40A9804AD0B9A0C9B09990590284666
:1062E00004910692079343F091FF38B30023E243F1
:1062F00084F0020004F00401019302F00102029311
:10630000C0F340000393A3071CD052EA000329D135
:1063100041B333480CF04CFDB7EE001A044648B3C5
:10632000FFEE000A40F2ED409DED100A3FF0F2FA58
:10633000234601AA29462A480CF042FD13B0BDECC1
:10634000028B30BD59B90D990E9A0F9B01910292A3
:106350000393DEE704AD284643F052FFC6E70AB9CF
:106360000028D6D001211E480CF0C0FC13B0BDECB3
:10637000028B30BDDFED1B0A4FF49E609DED100ACD
:106380003FF0C8FAF6EE000AB0EE408A3FF0FCF8A3
:1063900090B9B6EE000AB4EEC08AF1EE10FA0EDD46
:1063A00038EE408A104BD3F8683438EE088A93ED03
:1063B000070A28EE000ABBE79FED0A0AB8E70A4B76
:1063C00030EE488AD3F8683438EE088A93ED080A2C
:1063D000B0EEC00A20EE480AAAE700BFF0930024FE
:1063E00060CC002400000000F0B300242DE9F04749
:1063F0000C46352200212DED028BE5789CB09542AC
:106400000EA828BF154678F1B7FA04F10C010EA8C2
:106410002A4678F167FAB94BD3F80C0903685B6A2E
:106420009847002800F0CA809DF86C50EB1F012DA2
:10643000DBB202D0022B00F2D180BDF8684014F428
:10644000E0780CBF0122002212EA542640F0B68008
:10645000002214F007090592069207921BD19FEDC6
:10646000A86AA5F10802DDED106ADDED117A012AB6
:106470009DED0F7A66EE866A67EEC67A27EE067A9B
:10648000CDED066ACDED077A8DED057A40F22E81CD
:10649000022B40F22281002714F0380A089709974E
:1064A0000A9740D1DDED127ADDED146AF4EE677AD9
:1064B0009DED137AB1EE666ACDED087A8DED097A1D
:1064C000F1EE10FA8DED0A6A80F18880F0EEE77A3D
:1064D0009FED8C6AF4EEC67AF1EE10FA7EDCB4EE33
:1064E000477AF1EE10FA79D6B0EEC77AB4EEC67AF2
:1064F000F1EE10FA72DCF4EE666AF1EE10FA6DD687
:10650000F0EEE66AF4EEC66AF1EE10FA66DC9FED94
:106510007C8A08A8B0EE480A45F07EFAA5F1080387
:10652000012B40F2A88000230B930C930D93B8F13C
:10653000000F18D19FED726AA5F10803DDED166A10
:10654000DDED177A012B9DED157A66EE866A67EE12
:10655000C67A27EE067ACDED0C6ACDED0D7A8DED7B
:106560000B7A40F2A68014F4806040D014F40063EB
:106570009FED650A4ED1DDED190AA2069FED637A03
:10658000DFED5F7A60EE870A60EEA70A46D0B9F1C8
:10659000000218BF0122BAF1000F14D19AB1B3FA68
:1065A00083F40121B0FA80F30BAA640958485B090F
:1065B0000094CDE9016108A90DF08CFA1CB0BDEC86
:1065C000028BBDE8F087BAF1000118BF0121002A53
:1065D00038D0002936D0B8F1000F70D001214C48D6
:1065E0000CF084FB1CB0BDEC028BBDE8F087A5F17C
:1065F00008029DED180A9FED457A012ADFED407AE9
:1066000020EE070A8CBF0026012614F4006320EE5A
:10661000270AB0D0A206DFED3C0AB8D1B3FA83F165
:10662000B0FA80F00BAB08AA49094009CDE9011680
:1066300005A9009036480DF02FFD1CB0BDEC028B73
:10664000BDE8F087B9F1000F14BF002101F001018E
:106650000029C3D0B8F1000FC0D00024B0FA80F2F6
:10666000B3FA83F305A9520929485B09CDE900640F
:106670000DF0BEFAA2E708A909AA2648FCF720FEF9
:106680000B970C970D97B8F1000F7FF46CAFDDED11
:10669000166A9DED177ADDED157A66EE886A27EEAB
:1066A000487A67EE887ACDED0C6A8DED0D7ACDEDE6
:1066B0000B7A0CAA0BA91748FCF702FE53E701243A
:1066C000B0FA80F2B3FA83F30BA9520910485B09C0
:1066D000CDE900640DF08CF970E705AF0E48F0F0DD
:1066E00047FC0146384645F063F9D4E605AF06AAF3
:1066F00008483946FCF7E4FDF0E700BFF0930024BA
:106700000000C84200007A4400000000E02E65420C
:1067100060CC0024F033002430B800242DE9F04789
:106720000C463522002106462DED028BE578A0B0FF
:10673000954212A828BF154678F11EF904F10C0104
:1067400012A82A4678F1CEF8A04BD3F80C090368BA
:106750005B6A984730B1BDF87840A30504F4E07552
:1067600005D525B920B0BDEC028BBDE8F0870AAF96
:1067700004F00708384620F0F7FFB8F1000F00F0EA
:10678000A580002314F038060493059306933CD1AA
:10679000DDED167ADDED186AF4EE677A9DED177A75
:1067A000B1EE666ACDED047A8DED057AF1EE10FA60
:1067B0008DED066A80F19980F0EEE77A9FED846AAC
:1067C000F4EEC67AF1EE10FA00F38F80B4EE477A59
:1067D000F1EE10FA80F18980B0EEC77AB4EEC67A95
:1067E000F1EE10FA00F38180F4EE666AF1EE10FA31
:1067F0007BD6F0EEE66AF4EEC66AF1EE10FA74DCCF
:106800009FED740A04A845F007F900230793089345
:1068100009939DB99FED6F6ADDED1A6ADDED1B7A74
:106820009DED197A66EE866A67EEC67A27EE067ADD
:10683000CDED086ACDED097A8DED077A14F4806A02
:1068400034D014F400699FED648A3CD1DDED1D8ADB
:10685000DFED627ADFED5F0A68EEA78A68EEA08A54
:1068600014F03F044AD0B8F1000318BF01230EB959
:10687000002B64D1003E18BF0126002B00F08B8056
:10688000002E00F0888085BB0120B9FA89F3BAFA9E
:106890008AF2F0EE680AB0EE480A5B09520907A9CD
:1068A000CDE900504E480DF0A3F85BE79DED1C8A42
:1068B00014F40069DFED497A9FED460A28EE278A35
:1068C00028EE008AC2D0DFED448AC9E7DDE9139AD9
:1068D0004846514640F02EFD38B1304607AA9DF893
:1068E0007C108CF08DF900283ED101213C480CF041
:1068F000FDF920B0BDEC028BBDE8F087384620F0F2
:1069000089FF0328F1D0002338460EA90E930F9378
:10691000109321F0F9F80028E7D0B9FA89F0BAFA13
:106920008AF3F0EE680A04AA4009B0EE480A5B094F
:106930000EA9CDE900042A480DF032FC12E7B9FA9D
:1069400089F401200021BAFA8AF36409F0EE680A9A
:10695000B0EE480A5B0907AA0094CDE9011004A92A
:106960001F480DF0B7F8FDE6DDED157A0EAE9FED90
:10697000197A5246079B494667EE877A304600935C
:10698000FDEEE77A17EE903A20F006FF96E80F004A
:1069900087E80F00F5E6B8F1000F14BF002606F0F7
:1069A0000106002EA1D0002D9FD00020B9FA89F356
:1069B000BAFA8AF2F0EE680A0090B0EE480A5B0973
:1069C0003946520906480DF023FACBE6F09300242D
:1069D00000007A440000C84200000000E02E65423A
:1069E00060CC002400B591F80AE04B7A43EA0E230C
:1069F00091F80BE043EA0E43562B16D00A46844624
:106A000007D8522B1BD0542B13D15DF804EBFFF7A2
:106A1000EDBC0D49194421F07F41012909D8017CC1
:106A20005DF804EB09487AF025BC5DF804EBFFF74C
:106A300075BE114660465DF804EB8CF06BB95DF8ED
:106A400004EBFFF71DBC00BF7AFFFF001CBA002457
:106A50002DE9F041044648F22C6000230122204435
:106A60002DED028B90B0694600937BF01DFB08B9B9
:106A7000584B009304F5C045D5F80C0903685B69D1
:106A80009847002840F0968004F500489FED528A10
:106A9000D8F8643493EDE07BD3EDE76AFDEEE66A67
:106AA000B7EEC77B16EE903A27EE088A1FB246F281
:106AB000385601A92644304613F0B4FC00287FD094
:106AC0003722002102A877F157FFA3238DF8083061
:106AD00095238DF80930FDF079FED8F85C34CDF8B7
:106AE0000B00D5F83009D3F8DC20D3F8E03044307F
:106AF000CDF81320CDF81730CDF80F1081F0FAFF44
:106B0000B7EE001A90ED000ADFED340A9F203EF048
:106B100001FFD5F8300910EE103A314ACDF81B309C
:106B200003681B69934250D190ED4B0AB6EE061AEA
:106B3000F4EE000A30203EF0EDFE10EE103A48F27E
:106B40004045CDF81F3018EE103A2819CDF8233003
:106B5000F0F012FADFED207A3046D8F80C3420EE4F
:106B6000270ACDF82B3010EE103ACDF82730019BD4
:106B7000CDF82F3013F07AFC009A10EE103A281955
:106B8000ADF83B70CDF83330CDF83720F0F000FA97
:106B9000BDEEC00A41F69820372202A9204410EE2B
:106BA000103AADF83D307DF0D5FD10B0BDEC028B54
:106BB000BDE8F08100279FED098A04F5004876E7DB
:106BC0007EF0ECFE034B01937AE7984710EE103A03
:106BD000B5E700BF2292CA7F0AD7233C000000001D
:106BE000612F020810B500F50044D4F85C04E5F00C
:106BF0001FFDD4F86414D4F85C04BDE81040E5F03F
:106C00007DBD00BF70B54FF48051044613F054FDB4
:106C100000284FD004F5004641F69825D6F85C04CC
:106C2000254403689B689847692100F1A002284623
:106C30007DF090FBD6F85C040368DB6898476A2116
:106C400000F1A00228467DF085FBD6F85C040368BD
:106C50001B6998476B2100F1A00228467DF07AFB62
:106C6000D6F864246C21284602F52D727DF072FB63
:106C70002021204613F020FDE0B104F5C043D3F8F5
:106C80000C0903681B69984778B1D6F86424284634
:106C90006E2190327DF05EFBD6F8642428466F2189
:106CA000BC32BDE870407DF055BB20460DF000FCC5
:106CB0000028EAD170BD00BF08B518F0EBF9BDE8B7
:106CC000084018F041B900BF70B50D4684B04FF6CA
:106CD000FF710646144613F0EFFC08B904B070BD0E
:106CE0000023CDE90033CDE90233A3238DF8003032
:106CF00095238DF8013003238DF80230FDF066FDF9
:106D0000CDF8030041F698200B4610223044694626
:106D10008DF80B50CDF8073003947DF0B1FD04B031
:106D200070BD00BF70B50D4684B04FF6FF710646CA
:106D3000144613F0C1FC08B904B070BD0023CDE9BE
:106D40000033CDE90233A3238DF8003095238DF86D
:106D5000013004238DF80230FDF038FDCDF803003A
:106D600041F698200B461022304469468DF80B50AE
:106D7000CDF8073003947DF083FD04B070BD00BFF3
:106D800030B50023A32204460D462DED048B87B0B9
:106D9000B0EE409AF0EE608A0093B0EE418A05931F
:106DA0008DF800209522CDE90133CDE90333062388
:106DB0008DF801208DF80230FDF008FDCDF80300BC
:106DC00041F698200B461822694620448DF80B5056
:106DD000CDF807308DED039ACDED048A8DED058A4F
:106DE0007DF0B8FC07B0BDEC048B30BD10B54FF49E
:106DF0008011044613F060FC00B910BD04F5125078
:106E0000BDE8104015F04EBF2DE9F04F2DED028B7F
:106E10008DB080462F2200216846F0EE408AB0EE09
:106E2000608A11EE10BA11EE90AA12EE109A12EECC
:106E3000907A13EE106A13EE905A14EE104A77F11E
:106E40009BFDA3238DF8003095238DF80130092395
:106E50008DF80230FDF0BAFC18EE903ACDF8030040
:106E600041F69820CDF80710CDF80B302F2218EE00
:106E7000103A69464044CDF813B0CDF80F30CDF844
:106E800017A0CDF81B90CDF81F70CDF82360CDF87A
:106E90002750CDF82B407DF05DFC0DB0BDEC028B92
:106EA000BDE8F08F30B52DED088B8BB0282204465D
:106EB0000D4668460021B0EE40BAF0EE60AAB0EE92
:106EC00041AAF0EE619AB0EE429AF0EE628AB0EE1C
:106ED000438A77F151FDA3238DF8003095238DF877
:106EE00001300A238DF80230FDF070FCCDF803006C
:106EF00041F698200B462822694620448DF80B5015
:106F0000CDF807308DED03BACDED04AA8DED05AABD
:106F1000CDED069A8DED079ACDED088A8DED098AA3
:106F20007DF018FC0BB0BDEC088B30BD2DE9F043B3
:106F30008FB01446074689463122002101A8169ECB
:106F4000179D984677F118FDA3238DF804309523FB
:106F50008DF8053008238DF80630FDF037FC2368E6
:106F60003122CDF8070041F6982004936368384435
:106F7000CDF80B1001A90593A3686C6806933368DC
:106F80008DF80F90CDF81D3073688DF81C80CDF80A
:106F90002130B368CDF82D40CDF825302B68CDF8E1
:106FA0002930AB68CDF831307DF0D4FB0FB0BDE8AF
:106FB000F08300BFF0B52C27144605460E463A462E
:106FC00000212DED068B8DB0B0EE409AF0EE608A78
:106FD00001A8B0EE418AB0EE61AAF0EE429A77F1D4
:106FE000CBFCA3238DF8043095238DF805300B23BB
:106FF0008DF80630FDF0EAFBDFED1A7A0B4694EDD2
:10700000006A3A46D4ED016A29EE279A94ED027A95
:1070100026EE276ACDF8070041F6982066EEA76AAB
:1070200001A968EEA78A284428EE278A8DF80F6008
:1070300067EE277ACDF80B308DED049ACDED058AF9
:107040008DED068A8DED076ACDED086ACDED097AE2
:107050008DED0AAACDED0B9A7DF07CFB0DB0BDEC59
:10706000068BF0BDE02E6542B020704730B5044677
:1070700041F6982589B0134B25441E22D3F83009D8
:107080006946F1F0AFFC6A460F4928467DF0D2FA16
:1070900004F5C043D3F80C0903681B68984704F54E
:1070A00080430146284693F830257DF02FFD04F5F6
:1070B000125018F06FFA04F556702CF065FF09B005
:1070C00030BD00BFF09300245C011E08F8B54FF0FE
:1070D000804105460023404A404C05F66867404819
:1070E000A96340496B61AB61EB61EB6329646A643E
:1070F0006C6305F66834686005F14800DEF036F828
:1071000005F58270B2F0C0F805F52B608DF0C2FB7A
:10711000354E364BC5F8B03A20468DF031FE44F876
:10712000306BBC42F8D1204605F580568FF0BEFE8C
:1071300041F6F40000212E4C2844F5F0F1FA41F616
:10714000A4102844F6F0B4FA41F6C810C6F8C449B1
:107150002844F7F063F9A4F5E76341F66420C6F824
:10716000583A2844B9F00EFFA4F50C7341F62C40B0
:10717000D434C6F81C3C9FED1F1A2844DFED1E0ACC
:107180009FED1E0AC6F8284CE6F0AAFA9FED191AE0
:1071900041F644409FED1A0AF0EE410A2844E6F019
:1071A0009FFA9FED141A41F65C409FED150AF0EE30
:1071B000410A2844E6F094FA41F6AC402844EBF04A
:1071C000C9FD28460F496EF08BFE28460E496EF029
:1071D00087FE2846F8BD00BF0000E0400000C8411F
:1071E000084B00240AD7233C7CA11A0890A11A0856
:1071F000B8D00024000000009A99993E0000B443E2
:1072000000804A43C4931A08B4961A082DE9F04343
:10721000ADF50F7D504DD022504981465AA877F1E7
:1072200061FB0DF1380C5AAC8EAE0FCDACE80F00FF
:107230000FCDACE80F000FCDACE80F0095E80F00C4
:107240008CE80F0020461034B7EE000A00216FF0E2
:1072500079FCB442F6D1424B02AC0FCB84E80F006C
:1072600001A920466FF01EFC002844D10EAC0DF1A0
:10727000780820461034B7EE000A00216FF062FC57
:107280004445F6D136AF90223649384677F12AFB8D
:107290000022092138466FF011FD99F9D46D002EB6
:1072A0003DD0314D06AE9FED310A44460FCD0FC69D
:1072B00095E80F0086E80F0006A800216FF042FC59
:1072C000002130469FED290A6FF03CFC602205F159
:1072D0001001404677F106FB20461034B7EE000A55
:1072E00000216FF02FFCA742F6D18FF0A5FD0DF520
:1072F0000F7DBDE8F0839DF90430F0EE007ADFEDFC
:107300001C6AB7EE000A07EE103AE068B8EEC77ADA
:10731000E7EE267A80EE270A70F0CAFAA6E7154D46
:1073200044460FCD0FC40FCD0FC40FCD0FC495E849
:107330000F0084E80F003246042140466FF0BEFC87
:107340009FED0D0A0D4870F0B3FAB7EE000A0C4835
:1073500070F0AEFAA5E700BF002C1A08302B1A080F
:10736000402C1A08502C1A08202D1A08000034420C
:10737000CDCCCC3DE02C1A0800000000A8921A08E1
:10738000B8921A0830B5B5B0D0220849684634AD75
:10739000044677F1A7FA20461034B7EE000A002120
:1073A0006FF0D0FBAC42F6D135B030BDA02D1A083D
:1073B0002DE9F04391B01D200DF106018FF0E6FBA1
:1073C00010B911B0BDE8F0839DF8063011216F4A65
:1073D0000BA80133DBB28DF80630FCF0FFFA002277
:1073E0000DF107010BA86EF07DF99DF80630684A93
:1073F000112104460BA8FCF0F1FA00220DF107015F
:107400000BA86EF06FF99DF80630624A112105460F
:107410000BA8FCF0E3FA00220DF107010BA86EF0B7
:1074200061F99DF806305C4A112103F03F030746DD
:107430000BA8FCF0D3FA0DF107010BA800226EF0A7
:1074400051F90646002CBCD0002DBAD0002FB8D080
:107450000028B6D020466EF0FBFC0028B1D12846AB
:107460006EF0F6FC0028ACD138466EF0F1FC002836
:10747000A7D130466EF0ECFC0028A2D1474B0DF1AD
:107480000C0C0DF11C0803F1100E0FCB8CE80F0053
:107490009EE80F0088E80F0002A960466FF002FB2B
:1074A00002A968B3BDF9089040466FF0FBFA1FFAD5
:1074B00089F3002857D1002B83D040F2D66842468A
:1074C0009A4232D228460DF10A01ADF80A9070F0C6
:1074D000FFFD20460DF10A01ADF80A8070F0F8FDBD
:1074E0000DF10A013846ADF80A8070F0F1FD012374
:1074F0000DF10A013046ADF80A3070F003FE60E786
:1075000040466FF0CFFA00283FF45BAFBDF908802A
:107510001FFA88F2002A3FF454AF40F2E2494B468A
:10752000CEE740F2E24940F2D66828460DF10A0162
:10753000ADF80A8070F0CCFD20460DF10A01ADF8DF
:107540000A9070F0C5FD0DF10A013846ADF80A90B9
:1075500070F0BEFD00230DF10A013046ADF80A308F
:1075600070F0D0FD2DE7BDF908801FFA88F253EACC
:1075700002013FF426AF23B1002A9ED00FFA83F90F
:107580009EE7002ACDD040F2E243F7E7C8921A08FE
:10759000D4921A08E0921A08F0921A08702E1A086B
:1075A00044F22071782230B5014483B004467AF069
:1075B000DDFE00220C21294801256FF07FFB2046CB
:1075C000FFF7F6FE44F23470B7EE000A0022022103
:1075D00020446FF027FC44F2CC110023204A2144C0
:1075E000452000956FF084FB1E4B1A68D1070CD420
:1075F0001D4A04F578511D6041F6AC33116044F228
:10760000E421234421449361D16044F29870032221
:107610001549012520446FF0CDFB41F69821002348
:10762000124A2144FD2000956FF062FB104B1A684E
:10763000D20705D442F26C320E491D6022440A6022
:1076400001210C486FF0D4FB70F02AF90A4A138824
:1076500043F00103138003B030BD00BF04931A0848
:1076600000A21D0854D20024C4250024689A1B08D7
:1076700058D20024E825002414D600240F2904D869
:10768000302303FB0100B83070470020704700BF73
:10769000014B93F967077047F0730024024B93F88E
:1076A000250900F001007047F0930024054BB3F862
:1076B0002C37DB0703D40069C0F34010704700206B
:1076C000704700BFF0730024014BD3F89804704753
:1076D000F093002438B50C1E05DB1C4DE3B295F881
:1076E000A4249A4200D238BDD5F8A0340122A5F5D1
:1076F000C040195D05F022F80028F4D08DF038FB69
:1077000003218EF0AFFD0028EDD18DF031FB0D216E
:107710008EF0A8FD0028E6D1A5F5005292F94C376D
:10772000E340DB0706D5A5F5C0400221BDE838409F
:10773000FBF78ABB92F96617A5F5C040E140BDE8AA
:10774000384001F00101FBF77FBB00BFF09300243C
:10775000022910B5044608D00A4BD3F80C09036877
:107760001B689847844207D010BD01463522064861
:10777000BDE8104004F0E2BF8DF0FAFABDE8104019
:107780008DF0F0B9F0930024F033002408B50368BD
:107790000A4A9B6893420ED1094B93F8250900F0E1
:1077A000010030B9064B93F92409B0FA80F0400982
:1077B00008BD002008BD9847F3E700BF9D7602088A
:1077C000F093002400F5C0439FED186ADFED186ABE
:1077D000012110B5D3F890240446D3F88C3400F579
:1077E0001250B2F90820B3F9083007EE102A07EE5C
:1077F000903AB8EEC77AF8EEE77AC7EE060A87EE57
:10780000860A60EEA60A20EE260A17F0EDFC7EF04E
:10781000C5F826217DF0B2FD46F29860054A0621A2
:107820002044BDE8104082F00BB800BF0000C84201
:1078300035FA8E3C289F1A0870B500F5004595F87A
:10784000781400294BD0324B0446324AD3F80C0945
:10785000904245D1D3F830392F4E93F8D530002BD4
:107860003FD0012295F87934327243B904F5C04310
:1078700093F90009002832DB85F8792405E004F546
:10788000C04393F90029002A2BDB01399FED236ABD
:10789000DFED236A04F51250C9B285F87814B1FA05
:1078A00081F1D3F89024D3F88C344909B2F9082037
:1078B000B3F9083007EE102A07EE903AB8EEC77A0F
:1078C000F8EEE77AC7EE060A87EE860A60EEA60AA9
:1078D00020EE260A17F088FC95F8783473B170BD55
:1078E0000D4E002346F298600E4A0621204485F88A
:1078F00078343372BDE8704081F0A2BF46F29860E0
:107900003372094A06212044BDE8704081F098BFD7
:10791000F09300244CCE002458D5002400007A4572
:1079200035FA8E3C349F1A08489F1A088B1ED92BB3
:107930006ED8DFE803F06F706F6F6D6F6D6D706DF7
:107940006F70706D6F6F6F6D6D706F706D70706D4B
:107950006D6D6D6D706F6D6D6D6F6D706D6D6F7048
:10796000706F6D6F6F6F6D6D6F6D6D6F6F6F6D6D34
:107970006F6F6D6D6D6D6D6D6F6F6F6F6F6F6D7024
:10798000706D6D6D6D6D6D6F706D6D6D6D6D6D6D1F
:107990006D6D6D6D6D6D6D6F6D6D6D6D6D6D6D6D15
:1079A0006D706D6D6D6D6D6D6D6D6D6D6D6D6D6D04
:1079B0006D6D6D6D6D6D6D6D6D6D6D6D6D6D6D6DF7
:1079C0006D6D6D6D6D6D6D6D6D6D6D6F6F6D6F6DE1
:1079D0006D6D6D70706F6D6D6D6D6D6D6D6D6D6DCF
:1079E0006D6D6D6D6D6D6F6D6F6D6D6D6D6D6D6DC3
:1079F0006D6D6D6D6D6D6D6D6D6D6D6D6D6D6D6DB7
:107A00006D6D6D6D6D6D6D6D6D6D6D6D6D6D6D70A3
:107A10008EF060BA704700238EF022BA8B1E70B5CC
:107A20008AB0D92B00F22281DFE813F00603F702B7
:107A30000003DE022001DA0020012001D50220012E
:107A40002001CA02B7022001B102AB02A502200147
:107A500020019B029302840220017802500220013F
:107A60002001200120012001FD01F701200120015A
:107A70002001F1012001E50120012001DF012001A9
:107A8000D6011C012001200120012001200120013C
:107A9000D001200120014A0244023E0220012001BF
:107AA00038021D02200120012001200120012001B7
:107AB000170211020B02BE01B801C4012001A90185
:107AC00095012001200120012001200120018701D2
:107AD0007A01200120012001200120012001200144
:107AE000200120012001200120012001200174013A
:107AF000200120012001200120012001200120017E
:107B0000200120012001200120012001200120016D
:107B1000200120012001200120012001200120015D
:107B2000200120012001200120012001200120014D
:107B3000200120012001200120012001200120013D
:107B4000200120012001200120012001200120012D
:107B50002001200120016E01500120015D01200162
:107B600020012001200145013A01200120012001CE
:107B700020012001200120012001200120012001FD
:107B800020012001200120012001200125012001E8
:107B9000CA01200120012001200120012001200133
:107BA00020012001200120012001200120012001CD
:107BB00020012001200120012001200120012001BD
:107BC00020012001200120012001200120012001AD
:107BD00020012001200120012001200120011C01A1
:107BE000022A3FD1BF4CC04BD4F80C299A4239D05D
:107BF000D4F8303993F8D530A3B304F54055B5F92E
:107C0000803223B9D4F89434B3F9083053B305AEB5
:107C1000002330460993CDE90333CDE90533CDE99F
:107C200007331FF0A1FDB5F98032B04D002B00F0F5
:107C30008C8205F58663D4F894440FCB86E80F0058
:107C4000B4F9083003A9AA48002BCCBF1023152390
:107C5000ADF80E3045F058FB20B17DF09FFE272196
:107C60007DF08CFB012420460AB070BD0AB0BDE84F
:107C700070408DF061BC002A00F00E82022AF1D122
:107C8000984BD3F80C0903689B6F98470028E9D1FB
:107C90008BF002FC974A0421012481F0D1FDE2E738
:107CA000002A00F00182022ADCD101238D4A1C4601
:107CB00082F87034D7E7002A00F0E981022AD1D196
:107CC0000123884A1C4682F80839CCE7022AC9D128
:107CD00089480124FCF7EEFA8BF0DEFB874A062187
:107CE00081F0AEFDBFE711468DF098FB8448DEF0D1
:107CF000FBFC04460028B5D07A4A92F8033943F0D9
:107D0000020382F80339AEE711461C200124FFF775
:107D10001FFDA8E711461B200124FFF719FDA2E76C
:107D2000002A00F0AF81022A02D16E4BC3F8042969
:107D30007448012405F0B4FA95E76A49724BD1F80A
:107D40000C0998428ED1022A4FF0010400F0EE8116
:107D500011F018FB87E7022A00F082816B4B0022AA
:107D6000012483F870217DF019FE4B217DF006FB84
:107D70008BF092FB664A062181F062FD73E7012ACF
:107D800000F0A281022A00F09981002A7FF46AAFF4
:107D9000012160480C4612F07FFB64E71146072082
:107DA0000124FFF7D5FC5EE7114616200124FFF7FA
:107DB000CFFC58E711460B200124FFF7C9FC52E71E
:107DC000114655480124F9F055FD4CE701201146B4
:107DD0000446FFF7BDFC46E7012A00F23781414B1C
:107DE0000022012483F84A213DE711461520012491
:107DF000FFF7AEFC37E7002A00F05B81022A7FF430
:107E000031AF0123414A1C4682F838392BE711462D
:107E100012200124FFF79CFC25E7114611200124C4
:107E2000FFF796FC1FE7013A01242E4BA24293F87C
:107E300002198CBF0022012262F3041183F8021997
:107E400011E7114602200124FFF782FC0BE71146DF
:107E500010200124FFF77CFC05E7114600200124D7
:107E6000FFF776FCFFE61F49274BD1F80C499C42EF
:107E70007FF4F8AE2046019211F094FA019A012A9B
:107E800000F05D81022A00F05481002A7FF4EAAEFE
:107E900020461146012410F071FEE4E61146182038
:107EA0000124FFF755FCDEE6114617200124FFF7F9
:107EB0004FFCD8E6114605200124FFF749FCD2E625
:107EC000114604200124FFF743FCCCE6A2F1020195
:107ED000064B0124B1FA81F1D3F85C044909E8F0BA
:107EE000C7F8C0E6F093002400C60024F0B30024D5
:107EF0003CC60024889F1A08F0330024A49F1A0867
:107F0000A099002484C500248CD10024F0C300244F
:107F1000749F1A082899002480C90024A2F1020243
:107F2000954B0124B2FA82F2D3F85C34520983F8FB
:107F3000202098E6012A00F0E680022A00F0DE8088
:107F4000002A7FF48FAE11468C480124AAF054FC1D
:107F500089E6022A7FF486AE8948012401F09CFF5D
:107F600081E6A2F1020185480124B1FA81F14909B3
:107F7000AAF042FC77E6114609200124FFF7E8FB4E
:107F800071E611460F200124FFF7E2FB6BE6114674
:107F900003200124FFF7DCFB65E6012A00F0A48042
:107FA000022A00F09780002A7FF45CAE754B012412
:107FB00083F890277DF0F2FC2B217DF0DFF952E66B
:107FC000012A5DD0022A14BF002102216C4801243D
:107FD000FAF73AFF47E6022A00F09B806A4B00223C
:107FE000012483F8A8243EE6022A7FF43BAE664DC6
:107FF000D5F80C090368DB6A9847044600283FF46B
:1080000031AED5F89434B3F90830002B7FF42AAEA2
:10801000A5F5C040FFF7D6FB25E6111E58484FF0E6
:10802000010418BF0121FAF70FFF1CE611460620D4
:108030000124FFF78DFB16E6022A7FF413AE3522EA
:108040000E214F48012404F079FB0CE6022A7FF44C
:1080500009AE9FED4E0A01244D48F5F0E3FB02E620
:108060004C4B012483F870417DF098FC4A217DF04F
:1080700085F98BF011FA484A062181F0E1FBF2E51F
:108080001146A3E7404B0122C3F8042950E63E4BBA
:10809000012483F80829E6E53B4B0124D3F80C09B9
:1080A0000368DB6F9847DEE5374B012483F87024C3
:1080B000D9E5384B012483F83829D4E511463748EF
:1080C000012412F0E9F9CEE500213448144612F0FB
:1080D000E3F9C8E52B4B012483F890277DF05EFC83
:1080E0002D217DF04BF9BEE5264B144683F89027F1
:1080F0007DF054FC2C217DF041F9B4E501211F48AD
:10810000AAF07AFB28E711461C481446AAF074FB33
:10811000A9E51921224871F095FA044600283FF498
:108120005DAF194B012283F8A8249CE511F0AEF84D
:1081300099E5012120460C4610F020FD93E52046EC
:108140000021144610F08EFA8DE5162303A9154878
:10815000ADF80E30D5F83434642BB8BF64230693E1
:1081600045F0D2F800283FF464AD7DF017FC2721DC
:108170007DF004F95DE500BFF0B30024DCB9002414
:10818000F0330024F0730024F0930024000000007A
:108190002C950024F0C30024609F1A08289900241D
:1081A000D84B00243CC600240120704700207047B3
:1081B00038B5044614482DED028BEEF0E1FE05467D
:1081C00042F0C4FF1148B0EE408A12F001FA30B11B
:1081D000DFED0F7AB4EEE78AF1EE10FA04DC94EDED
:1081E000080ABDEC028B38BDD5ED000A95ED010AF9
:1081F00073F1E4FCDFED077A20EE270A84ED080A2C
:10820000BDEC028B38BD00BF30B80024F033002431
:1082100000401C46E02E6542174A92F94D37022B6A
:1082200009D0032B15D073B10368012B0AD00122AA
:10823000C0E9002370470029F6D0036813B100227B
:10824000C0E9002370470268002AFBD0C0E9003271
:1082500070470368042BF5D043600421A2F5CC538A
:108260009FED067A0160D3ED007AF8EEE77A67EECB
:10827000877AC0ED087A7047F07300240AD7233C50
:10828000074B93F94D07022807D0032803D0003885
:1082900018BF012070470420704781F0010070472B
:1082A000F073002403688B4208D00429C0E900134E
:1082B00005D0072900D07047002383627047074B21
:1082C0009FED077A03F5D063D3ED007AF8EEE77AF5
:1082D00067EE877AC0ED087A704700BFF05300243C
:1082E0000AD7233C70B5044616460D462DED028B89
:1082F000F0EE408AB0EE608AFCF060FAE061002E99
:1083000040D0236843B9334B03F5D063D3ED007AF3
:10831000F8EEE77AC4ED097A9FED2F0A002D28EEDA
:10832000800A2CDB84ED050ADFED2C7A2C4BB4EEB1
:10833000E78AD3F85C04F1EE10FA10DAE5F01EFBE0
:10834000DFED257A20EE270A84ED060A2368032B49
:1083500002D00322C4E90023BDEC028B70BDE5F01E
:108360000DFBB4EE480ADFED1C0AF1EE10FA48BF2F
:10837000B0EE408A28EE208A84ED068AE6E7B1EE68
:10838000400ACFE794ED090ADFED137A98EEA70AC9
:108390003DF00EFA002D84ED050A0CDBC4D0DFEDB4
:1083A000117AB4EEE70AF1EE10FABDD8DFED0E7ADD
:1083B00030EE270AB6E7DFED097AB4EEE70AF1EE10
:1083C00010FAB1DBDFED087A30EE670A84ED050ABA
:1083D000AAE700BFF05300240000C84200000034A8
:1083E000F0B30024000000B400A00C4710B5044610
:1083F0002DED028BB0EE608AF0EE408AFCF0DEF9E3
:10840000DFED090A236828EEA00AE06168EE200A81
:10841000062B84ED090AC4ED0A0A02D00622C4E93B
:108420000023BDEC028B10BD0000C84210B504460D
:108430002DED028BB0EE408AFCF0C0F994ED090AF4
:10844000DFED097AE061A8EE270A3DF0FBF9236829
:10845000002284ED090A062BA26202D00622C4E99A
